:020000040000FA
:1000000018F09FE518F09FE518F09FE518F09FE5C0
:1000100018F09FE50000A0E1F0FF1FE518F09FE554
:10002000400000004C4D0100EC370100484D01003C
:10003000444D010000000000404D01003C4D010016
:10004000C0009FE5C0009FE50210A0E3001080E51E
:10005000B8009FE5AA10A0E35520A0E32330A0E359
:10006000043080E50130A0E3003080E50C1080E52D
:100070000C2080E5083090E5013B13E2FCFFFF0A0D
:100080000330A0E3003080E50C1080E50C2080E513
:100090007C009FE50410A0E3041080E50210A0E3BB
:1000A000001080E56C009FE5DBF021E300D0A0E1CB
:1000B000040040E2D7F021E300D0A0E1040040E2D8
:1000C000D1F021E300D0A0E1040040E2D2F021E32E
:1000D00000D0A0E1800040E2D3F021E300D0A0E115
:1000E000040040E210F021E300D0A0E128009FE5E9
:1000F000010010E324E09F0524E09F1510FF2FE18D
:10010000FEFFFFEAFEE7C0460000E0FF00C11FE07F
:1001100080C01FE000C01FE090040040D9680000CC
:10012000000100000501000020000000095200004D
:10013000D15100007552000041520000070000003C
:100140000700000005000000070000000700000095
:100150000500000000000000010000000100000098
:100160000100000007000000010000000A0000007C
:0B0170000A00000001020408102040FB
:10017C00520000003D51000009510000A151000047
:10018C0071510000460000004600000032000000E3
:10019C004600000046000000320000000000000095
:1001AC000A0000000A0000000A00000046000000DF
:1001BC000A0000006400000064000000A0060000BB
:1001CC0005050000A005000005040000A0040000C7
:1001DC0005030000A0030000050200000506000056
:1001EC0000000000500600000A0500005005000049
:1001FC000A040000500400000A0300005003000031
:10020C000A020000300200000A0600000000000094
:10021C00102122232425262711121314151617003A
:07022C0001020304050607AF
:0602340002402010080446
:10023C00121422132324152550000000095200002B
:10024C00D15100007552000041520000070000001F
:10025C000700000005000000070000000700000078
:10026C00050000000000000001000000010000007B
:10027C000100000007000000010000000A0000005F
:10028C000A00000000052595A00000003D5100006B
:10029C0009510000A151000071510000070000003D
:1002AC000700000005000000070000000700000028
:1002BC00050000000000000001000000010000002B
:1002CC0001000000070000000100000060EA0000CF
:1002DC000A00000020537572726F756E64205072A4
:0902EC006F636573736F722000EB
:1002F800000000403C483F00003E001D1C301F4AE3
:100308003A3B00001E4931004733414243444546C9
:100318003D353834242E2F23000037002B2C2D2276
:100328000032360028292A210039000025262720F6
:100338004C004B0000000000504D4F4E00000000E4
:1003480053000052000000005C0000510000000053
:10035800545556570000000058595A5B00000000D9
:100368000000000000000000000000000000000085
:100378000100000009000000020000000B0000005E
:10038800040000000D000000080000000C00000040
:10039800100000000A0000004000000004000000F7
:1003A800000100000E000000000200000F00000025
:1003B8000004000010000000000800001100000008
:1003C80000100000060000000020000005000000EA
:1003D8000040000008000000008000000700000046
:1003E80000000100160000000000020017000000D5
:1003F80000000400180000000000080019000000B8
:10040800000010001200000000002000130000008F
:1004180000004000140000000000800015000000EB
:100428004100000062000000000000000000000021
:10043800526573746F72652044656661756C7420CB
:100448004F4B2020002E2E2E2E2E2E2E2E2E2E2ED0
:100458002E2E2E2E2E2E2E2E2E0054657374204DE9
:100468006F6465202020202020204155544F002013
:1004780020436172792043696E656D6120313120B6
:02048800200052
:10048C0025630050617373776F7264204D69736DCF
:10049C0061746368210050617373776F72642053C9
:1004AC00657421005265456E7465722050617373DA
:1004BC00776F72643A0050617373776F7264206562
:1004CC0072726F722100456E746572204E657720D2
:1004DC0050617373776F72643A002A00456E7465CD
:1004EC0072204F6C642050617373776F72643A00A2
:1004FC00456E7465722050617373776F72643A0045
:10050C005F0025332E31666442002534646442005A
:10051C002533646D73002538730025332E316666E0
:10052C00742025322E31664D00257300F31C00001B
:10053C0000000600F4150000771B00000300070004
:10054C0008080000F71B000004000900A4080000C4
:10055C000A1C00000500090058090000171C0000C7
:10056C0006000A00240A0000231C000007000900F2
:10057C00EC0A0000381C000008003900A00B000039
:10058C00441C000009000200241000007F1B000026
:10059C000A0004004C100000BB1B00000B000A00FA
:1005AC009C100000CE1B00000C0009006411000020
:1005BC00E21B00000D000B0028120000851B000040
:1005CC000E000300241300008B1B00000F0003001F
:1005DC00B8130000921B000014000D008C140000D6
:1005EC00D81C000016000200CC150000681C00008E
:1005FC001700030090150000000070C1000068C1D6
:10060C00000060C1000058C1000050C1000048C18A
:10061C00000040C1000038C1000030C1000028C1FA
:10062C00000020C1000018C1000010C1000008C16A
:10063C00000000C10000F0C00000E0C00000D0C00D
:10064C000000C0C00000B0C00000A0C0000090C0FE
:10065C00000080C0000060C0000040C0000020C04E
:10066C00000000C00000C0BF000080BF000000BF41
:10067C00000000000000003F0000803F0000C03F71
:10068C00000000400000204000004040000060409E
:10069C0000008040000090400000A0400000B040EE
:1006AC000000C0400000D0400000E0400000F040DE
:1006BC0000000041000008410000104100001841FA
:1006CC00000020410000284100003041000038416A
:1006DC0000004041000048410000504100005841DA
:1006EC000000604100006841000070410000000003
:1006FC000D1B000001000000081B000002000000A0
:10070C00031B000003000000FE1A000004000000A0
:10071C00F91A000005000000F41A000006000000A1
:10072C00EF1A000007000000E91A000008000000A2
:10073C00E31A000009000000DD1A00000A000000A6
:10074C00D71A00000B000000D11A00000B000000AB
:10075C00000000000C000000000000000D00000074
:10076C000000000003000000000000000400000076
:10077C000000000005000000000000000600000062
:10078C00000000000700000000000000080000004E
:10079C000000000009000000000000000000000044
:1007AC00000000000E000000000000000F00000020
:1007BC00000000001000000000000000110000000C
:1007CC0000000000120000000000000013000000F8
:1007DC00000000000A0000000000000014000000EF
:1007EC0000000000150000000000000016000000D2
:1007FC00000000001700000000000000F71B0000C4
:10080C00010100007807000000000000CD79000015
:10081C000A1C00000101000080070000000000001D
:10082C00CD790000171C00000101000088070000B2
:10083C0000000000CD790000231C00000101000025
:10084C009007000000000000CD790000381C00006B
:10085C00010100009807000000000000CD790000A5
:10086C00441C000001010000A00700000000000073
:10087C00CD790000AC1B000001010000A8070000AE
:10088C0000000000CD79000000000000CE1A00002E
:10089C0001000000CA1A00005C1B000002020000EC
:1008AC009408000000000000056E00005F1B0000B3
:1008BC00020200009408000001000000056E000018
:1008CC00631B0000020200009408000002000000FC
:1008DC00056E0000661B0000020200009408000078
:1008EC0004000000056E0000691B000002020000FD
:1008FC009408000007000000056E00006D1B00004E
:10090C00020200009408000006000000056E0000C2
:10091C00711B00000202000094080000030000009C
:10092C00056E0000741B0000020200009408000019
:10093C0005000000056E0000A71B0000010100006F
:10094C007007000000000000CD7900005C1B000067
:10095C000565000000000000000000007D6E000036
:10096C005F1B000005650000000000000100000096
:10097C007D6E0000631B0000056500000000000098
:10098C00020000007D6E0000661B00000565000083
:10099C0000000000040000007D6E0000691B0000D8
:1009AC000565000000000000070000007D6E0000DF
:1009BC006D1B000005650000000000000600000033
:1009CC007D6E0000711B000005650000000000003A
:1009DC00030000007D6E0000741B00000565000024
:1009EC0000000000050000007D6E0000A71B000049
:1009FC00010100007007000001000000CD7900002B
:100A0C0000000000191B000001000000C31A0000C8
:100A1C0002000000BE1A0000B41A0000020300001D
:100A2C000C0A000000000000DD6E00005C1B0000E2
:100A3C00093D000004060000000000000D700000DD
:100A4C005F1B0000093D00000406000001000000CF
:100A5C000D700000631B0000093D0000040600003F
:100A6C00020000000D700000661B0000093D000034
:100A7C0004060000040000000D700000691B00005B
:100A8C00093D000004060000070000000D70000086
:100A9C006D1B0000093D000004060000060000006C
:100AAC000D700000711B0000093D000004060000E1
:100ABC00030000000D700000741B0000093D0000D5
:100ACC0004060000050000000D700000A71B0000CC
:100ADC00010100007007000002000000CD79000049
:100AEC005C1B0000020C0000F80600000000000077
:100AFC00797000005F1B0000020C0000F80600007B
:100B0C000100000079700000631B0000020C000063
:100B1C00F80600000200000079700000661B00005F
:100B2C00020C0000F80600000400000079700000C0
:100B3C00691B0000020C0000F80600000700000012
:100B4C00797000006D1B0000020C0000F80600001C
:100B5C000600000079700000711B0000020C000000
:100B6C00F80600000300000079700000741B000000
:100B7C00020C0000F806000005000000797000006F
:100B8C00A71B00000101000070070000030000001B
:100B9C00CD790000AB1A0000093D000004060000EE
:100BAC000000000049710000A11A0000093D00007E
:100BBC00040600001000000049710000971A0000A4
:100BCC00093D0000040600002000000049710000EF
:100BDC008C1A0000093D00000406000030000000E3
:100BEC0049710000811A0000093D00000406000054
:100BFC004000000049710000751A0000093D00001A
:100C0C00040600005000000049710000691A000041
:100C1C00093D00000406000060000000497100005E
:100C2C00601A0000093D00000406000001000000ED
:100C3C0049710000561A0000093D0000040600002E
:100C4C0011000000497100004C1A0000093D000021
:100C5C00040600002100000049710000411A000048
:100C6C00093D00000406000031000000497100003D
:100C7C00361A0000093D0000040600004100000087
:100C8C0049710000291A0000093D0000040600000B
:100C9C0051000000497100001C1A0000093D0000C1
:100CAC00040600006100000049710000131A0000E6
:100CBC00093D00000406000002000000497100001C
:100CCC00091A0000093D0000040600001200000093
:100CDC0049710000FF190000093D000004060000E6
:100CEC002200000049710000F4190000093D0000C9
:100CFC00040600003200000049710000E9190000F0
:100D0C00093D00000406000042000000497100008B
:100D1C00DD190000093D000004060000520000002F
:100D2C0049710000D1190000093D000004060000C3
:100D3C006200000049710000C8190000093D000064
:100D4C00040600000400000049710000BE190000F8
:100D5C00093D000004060000140000004971000069
:100D6C00B4190000093D0000040600002400000036
:100D7C0049710000A9190000093D0000040600009B
:100D8C0034000000497100009E190000093D00006C
:100D9C000406000044000000497100009219000094
:100DAC00093D0000040600005400000049710000D9
:100DBC0086190000093D00000406000064000000D4
:100DCC00497100007D190000093D00000406000077
:100DDC00070000004971000073190000093D000074
:100DEC00040600001700000049710000691900009A
:100DFC00093D0000040600002700000049710000B6
:100E0C005E190000093D00000406000037000000D8
:100E1C004971000053190000093D00000406000050
:100E2C00470000004971000046190000093D000010
:100E3C000406000057000000497100003919000039
:100E4C00093D000004060000670000004971000025
:100E5C0030190000093D00000406000006000000E7
:100E6C004971000026190000093D0000040600002D
:100E7C0016000000497100001C190000093D00001B
:100E8C000406000026000000497100001119000042
:100E9C00093D000004060000360000004971000006
:100EAC0006190000093D0000040600004600000081
:100EBC0049710000F9180000093D0000040600000B
:100ECC005600000049710000EC180000093D0000BC
:100EDC00040600006600000049710000E3180000E1
:100EEC00093D0000040600000300000049710000E9
:100EFC00D9180000093D0000040600001300000092
:100F0C0049710000CF180000093D000004060000E4
:100F1C002300000049710000C4180000093D0000C6
:100F2C00040600003300000049710000B9180000ED
:100F3C00093D000004060000430000004971000058
:100F4C00AD180000093D000004060000530000002D
:100F5C0049710000A1180000093D000004060000C2
:100F6C00630000004971000098180000093D000062
:100F7C000406000005000000497100008F180000F5
:100F8C00093D000004060000150000004971000036
:100F9C0086180000093D0000040600002500000032
:100FAC00497100007D180000093D00000406000096
:100FBC00350000004971000074180000093D000064
:100FCC000406000045000000497100006A1800008A
:100FDC00093D0000040600005500000049710000A6
:100FEC0060180000093D00000406000065000000C8
:100FFC0049710000A71B00000101000070070000F0
:10100C0004000000CD79000000000000571800001B
:10101C00010000004E1800004218000002020000FF
:10102C001410000000000000E5700000A71B000079
:10103C00010100007007000005000000CD790000E0
:10104C00BB1B00000101000058070000000000005D
:10105C00CD790000CE1B00000101000060070000EC
:10106C0000000000CD790000E21B0000010100002F
:10107C006807000000000000CD790000AC1B0000E8
:10108C0001010000A807000001000000CD7900005C
:10109C001D1B0000040C0000FC2100400800000097
:1010AC0041730000241B0000040C000009220040C6
:1010BC0000000000417300002B1B0000040C00001A
:1010CC00162200400100000041730000321B00009A
:1010DC00040C0000232200400200000041730000B9
:1010EC00391B0000040C00003022004003000000FB
:1010FC0041730000401B0000040C00003D22004026
:10110C000400000041730000471B0000040C0000A9
:10111C004A22004005000000417300004E1B0000F5
:10112C00040C000057220040060000004173000030
:10113C00551B0000040C0000642200400700000056
:10114C0041730000A71B000001010000E007000034
:10115C0000000000CD790000241B0000081F0000D7
:10116C0040170000000000000D7200002B1B000057
:10117C00081F000040170000010000000D72000065
:10118C00321B0000081F0000401700000200000086
:10119C000D720000391B0000081F000040170000F2
:1011AC00030000000D720000401B0000081F00002F
:1011BC0040170000040000000D720000471B0000E7
:1011CC00081F000040170000050000000D72000011
:1011DC004E1B0000081F0000401700000600000016
:1011EC000D720000551B0000081F00004017000086
:1011FC00070000000D720000A71B00000101000099
:10120C00E007000001000000CD79000000000000A4
:10121C003B1800000100000037180000241B0000E0
:10122C00020200001812000000000000957200007D
:10123C002B1B00000202000018120000010000002D
:10124C0095720000321B0000020200001812000010
:10125C000200000095720000391B00000202000021
:10126C00181200000300000095720000401B0000E3
:10127C000202000018120000040000009572000029
:10128C00471B0000020200001812000005000000BD
:10129C00957200004E1B00000202000018120000A4
:1012AC000600000095720000551B000002020000B1
:1012BC001812000007000000957200001D1B0000B2
:1012CC0002020000181200000800000095720000D5
:1012DC00561C000002020000181200000900000059
:1012EC0095720000A71B000001010000E007000040
:1012FC0002000000CD790000000000002F18000053
:10130C000100000029180000000000002018000057
:10131C00010000001B1800000F1800000202000062
:10132C000413000000000000D57400000318000036
:10133C00020200001413000000000000657500009C
:10134C00AC1B000001010000A80700000200000017
:10135C00CD79000000000000241B000001000000FB
:10136C002B1B000002000000321B000003000000D9
:10137C00391B000004000000401B000005000000A9
:10138C00471B0000060000004E1B00000700000079
:10139C00551B0000080000001D1B00001900000078
:1013AC000018000029000000FD170000F0170000D5
:1013BC00020B00006013000000000000D16A000066
:1013CC00E2170000086A00006C1600000000000024
:1013DC00656B0000AC1B000001010000A8070000B9
:1013EC0003000000CD79000000000000191B000074
:1013FC0001000000DD17000002000000D8170000FB
:10140C0000000000191B000001000000A41B0000DC
:10141C0000000000191B000001000000D4170000A0
:10142C0002000000D017000003000000CB170000E2
:10143C0000000000A41B000001000000191B0000AC
:10144C0000000000C517000001000000C0170000DC
:10145C0002000000BB17000000000000B4170000E1
:10146C0001000000AD17000000000000A6170000EE
:10147C0001000000121B0000020000009B1700007E
:10148C00681C0000010100000008000000000000C2
:10149C00CD790000CA1C00000765000000000000A8
:1014AC000000000099690000611C000002040000AB
:1014BC001C14000000000000356A0000D81C00005D
:1014CC0001010000F807000000000000CD790000C9
:1014DC00961C0000020300004C14000000000000E9
:1014EC00CD6B0000A21C0000020300004C14000095
:1014FC0000000000196C00008E17000002020000B2
:10150C006414000000000000D96C0000801700007B
:10151C00020200006414000000000000696C00006E
:10152C00B11C000002030000741400000000000055
:10153C00496D0000861C0000020200003C140000F3
:10154C0000000000916A00005C1C00000203000017
:10155C00F413000000000000E9690000BA1C000050
:10156C00030000000000000000000000996D000066
:10157C00AC1B000001010000A807000004000000E3
:10158C00CD790000711C0000020200000C14000058
:10159C0000000000097600007F1C00000A04000017
:1015AC0000000000000000007D760000A71B00007A
:1015BC0001010000E807000000000000CD790000E8
:1015CC007E17000004120000712200400000000091
:1015DC0065740000A71B000001010000E807000073
:1015EC0003000000CD790000771B00000101000012
:1015FC007007000000000000CD7900007F1B000088
:10160C0001010000E007000000000000CD7900009F
:10161C00851B000001010000B00700000000000065
:10162C00CD7900008B1B000001010000B807000001
:10163C0000000000CD790000921B000001010000A9
:10164C00E807000000000000CD790000E91C000054
:10165C00010000000000000000000000B179000053
:10166C00A6FFA7FFA8FFA9FFAAFFABFFACFFADFF2A
:10167C00AEFFAFFFB0FFB1FFB2FFB3FFB4FFB5FFDA
:10168C00B6FFB7FFB8FFB9FFBAFFBBFFBCFFBDFF8A
:10169C00BEFFBFFFC0FFC1FFC2FFC3FFC4FFC5FF3A
:1016AC00C6FFC7FFC8FFC9FFCAFFCBFFCCFFCDFFEA
:1016BC00CEFFCFFFD0FFD1FFD2FFD3FFD4FFD5FF9A
:1016CC00D6FFD7FFD8FFD9FFDAFFDBFFDCFFDDFF4A
:1016DC00DEFFDFFFE0FFE1FFE2FFE3FFE4FFE5FFFA
:1016EC00E6FFE7FFE8FFE9FFEAFFEBFFECFFEDFFAA
:1016FC00EEFFEFFFF0FFF1FFF2FFF3FFF4FFF5FF5A
:10170C00F6FFF7FFF8FFF9FFFAFFFBFFFCFFFDFF09
:10171C00FEFFFFFF000001000200030004000500B3
:10172C0006000700080009000A000B000C000D0061
:10173C000E000F00EEFFEFFFF0FFF1FFF2FFF3FFE3
:10174C00F4FFF5FFF6FFF7FFF8FFF9FFFAFFFBFFD9
:10175C00FCFFFDFFFEFFFFFF000001000200030085
:10176C000400050006000700080009000A000B0031
:10177C000C0020005A4F4E4532204952204D4F4408
:10178C00450052454152204952204D4F4445005A84
:10179C004F4E45203120262032005A4F4E452031E5
:1017AC0000496E76657274004E6F726D616C00420A
:1017BC006F746800526561720046726F6E740048F7
:1017CC00696768004D6964004C6F770046756C6CF6
:1017DC000048616C66005A6F6E65203220766F6C23
:1017EC00756D65005A6F6E65203220696E70757468
:1017FC0000464D00414D0053657420414D207374DB
:10180C0065700053657420464D2046726571003931
:10181C004B487A0055534131306B487A004A61701D
:10182C00616E0055532F4575726F00445350004242
:10183C00797061737300416C6C20537065616B65DA
:10184C0072004F7574706861736500496E20706822
:10185C006173650053572020313235487A00535755
:10186C002020313030487A00535720203830487AC5
:10187C0000535720203633487A00535720203530F8
:10188C00487A00535720203430487A005357202090
:10189C003235487A00534C20203136303030487A7B
:1018AC0000534C20203132353030487A00534C20D4
:1018BC002038303030487A00534C202032353030CC
:1018CC00487A00534C2020383030487A00534C2052
:1018DC0020323530487A00534C20203830487A007A
:1018EC0053424C20203136303030487A0053424C31
:1018FC0020203132353030487A0053424C20383079
:10190C003030487A0053424C2032353030487A001F
:10191C0053424C20383030487A0053424C203235F8
:10192C0030487A0053424C203830487A00534252A7
:10193C0020203136303030487A005342522020314A
:10194C0032353030487A00534252203830303048EB
:10195C007A005342522032353030487A005342528A
:10196C0020383030487A0053425220323530487A91
:10197C0000534252203830487A00535220203136DE
:10198C00303030487A0053522020313235303048D4
:10199C007A005352202038303030487A005352208D
:1019AC002032353030487A005352202038303048BD
:1019BC007A0053522020323530487A00535220207E
:1019CC003830487A00465220203136303030487A50
:1019DC0000465220203132353030487A00465220B1
:1019EC002038303030487A004652202032353030A2
:1019FC00487A0046522020383030487A004652202F
:101A0C0020323530487A00465220203830487A004F
:101A1C0043454E20203136303030487A0043454E15
:101A2C0020203132353030487A0043454E20383052
:101A3C003030487A0043454E2032353030487A00F9
:101A4C0043454E20383030487A0043454E203235DD
:101A5C0030487A0043454E203830487A00464C20B6
:101A6C00203136303030487A00464C202031323527
:101A7C003030487A00464C202038303030487A00DC
:101A8C00464C202032353030487A00464C202038E5
:101A9C003030487A00464C2020323530487A0046A7
:101AAC004C20203830487A0054455354204D4F4434
:101ABC0045004155544F004D414E55414C00596520
:101ACC0073004E6F00313530487A00313330487A2C
:101ADC0000313230487A00313130487A00313030C0
:101AEC00487A003930487A003830487A0037304824
:101AFC007A003630487A003530487A003430487AEB
:101B0C000046554C4C005A4F4E452032004F6666ED
:101B1C0000372E3120496E00494E50555431004942
:101B2C004E5055543200494E5055543300494E5086
:101B3C0055543400494E5055543500494E50555467
:101B4C003600494E5055543700494E5055543800C4
:101B5C00464C0043454E00465200535200534252ED
:101B6C000053424C00534C00535700535045414BCB
:101B7C00455200494E50555400524144494F005A69
:101B8C004F4E45203200414456414E43454420536C
:101B9C00455454494E4753004F6E004241434B004D
:101BAC00474F544F204D41494E204D454E55004313
:101BBC0068616E676520696E707574206E616D6505
:101BCC00730053657420416E616C6F6720496E2001
:101BDC006C6576656C0053657420416E616C6F6743
:101BEC0020496E20436F6E666967005365742053FD
:101BFC007065616B657220436F6E66696700536533
:101C0C00742044697374616E63650053657420427B
:101C1C00616C616E6365005365742043726F7373FE
:101C2C006F76657220506F696E7473005365742003
:101C3C00526F6F6D20455100536574205370656170
:101C4C006B65722050686173650054756E65720027
:101C5C004C617465004272696768740050617373FB
:101C6C00776F72640050617373776F7264204D6F7D
:101C7C006465004368616E6765004175746F204947
:101C8C006E707574205365656B00495220436F6EFE
:101C9C0074726F6C73005A4F4E4532204952204378
:101CAC0074726C7300545249474745525300526545
:101CBC0073746F72652044656661756C740041566F
:101CCC002053594E432044656C6179004564697416
:101CDC0020437573746F6D204E616D6500455849D6
:101CEC0054204D454E55005345545550204D454EAE
:021CFC00550091
:101D0000FE200000659D0000FB200000F99D000002
:101D1000F92000002D9E0000F5200000699E0000C3
:101D2000F1200000CD9E0000ED200000D19E0000BB
:101D3000E9200000559F0000E5200000B99F000049
:101D4000E1200000BD9F0000DE2000004DA000004B
:101D5000DA200000C5A00000D720000031A100005B
:101D6000D320000065A10000CF200000418E0000BC
:101D7000CB200000158F0000C7200000718F0000ED
:101D8000C3200000A18F0000BF20000005940000C8
:101D9000BA200000FD920000B5200000F191000083
:101DA000B020000011910000AB200000F994000069
:101DB000A720000099900000A32000003D900000A3
:101DC0009E200000F58F000099200000B98F0000D0
:101DD00093200000A58F00008F200000BD8D000023
:101DE0008A200000FD94000084200000419600003D
:101DF0007E200000B19600007820000021970000AE
:101E000071200000919700006920000001980000F7
:101E100061200000759800005A200000E998000039
:101E2000532000005D9900004E200000D199000071
:101E30004A200000159A000046200000C19A0000C8
:101E400042200000899B00003E200000359C0000DD
:101E50003A200000799C000036200000319D0000EF
:101E600032200000619D00002E20000001A2000031
:101E70002A20000055A2000026200000A9A2000090
:101E800021200000FDA200001C20000051A3000042
:101E900017200000A5A3000012200000F9A30000F5
:101EA0000D2000004DA4000009200000F1A4000056
:101EB0000520000029A500000120000095A50000D4
:101EC000FD1F000001A60000F81F00006DA6000025
:101ED000F31F0000D9A60000EE1F000045A7000078
:101EE000E91F0000B1A70000E51F00001DA80000C9
:101EF000E11F000089A80000DC1F0000F5A8000019
:101F0000D71F000035A90000D21F000075A90000EE
:101F1000CD1F0000B5A90000C81F0000F5A90000F2
:101F2000C31F000035AA0000BF1F000075AA0000F3
:101F3000BA1F0000B5AA0000B61F0000A5AB000044
:101F4000B01F000019AC0000AA1F00008DAC0000FB
:101F5000A41F000001AD00009E1F000075AD000031
:101F6000981F0000E9AD0000911F00005DAE000069
:101F70008A1F0000D1AE0000861F000045AF0000A0
:101F8000404552520A0053485000535A5853424C4D
:101F900000535A5853425200535A58534C00535A04
:101FA00058535200535A58465200535A5846430009
:101FB000535A58464C00535A5800535A53570053DB
:101FC0005A4300535A425200535A424C00535A53F8
:101FD0005200535A534C00535A465200535A464CDF
:101FE0000053504700535073005350424C0053501D
:101FF0004252005350534C005350535200535052CE
:10200000005350430053504C0053505500534C5311
:102010005700534C424C00534C425200534C534CCB
:1020200000534C535200534C5200534C4300534CFA
:102030004C005A323F005A324D005A325A005A323E
:1020400058005A3256005A3253005A3250005A3110
:102050004551005A3145515357005A314551534C5F
:10206000005A31455142534C005A31455142535266
:10207000005A3145515352005A31455152005A319C
:10208000455143005A3145514C005A31564D005A82
:10209000313F005A3141443F005A314153005A31D7
:1020A000413F005A3143005A3144005A31454D00F6
:1020B0005A314544005A314546005A314558005A74
:1020C0003145005A314C005A314D005A3150005AB6
:1020D00031530052534E0046500054543F00544870
:1020E0000054465400544653005446500054415442
:1020F0000054415300544150005400484D0048568C
:10210000004054415425640A004054465425642E2E
:102110002531640A0040544825640A00405A32566A
:102120007325640A00405A325325640A00405A322B
:1021300050300A00405A3250310A00405A31564D50
:102140007325640A00405A314525640A00405A311B
:10215000455825640A00405A31454625640A004026
:102160005A314544300A00405A314544310A004052
:102170005A314425640A00405A314325640A00401C
:102180005A314125640A00405A3150300A00405A01
:0D2190003150310A00405A315325640A00D5
:1021A00001000000FDCE000003000000A57D00003E
:1021B000040000004DB200000200000059C40000FD
:1021C00005000000EDD000000600000025D1000051
:1021D00053746572656F004D6F6E6F004D75746559
:1021E0000073746572656F206D6F64653A204D6F82
:1021F0006E6F0073746572656F206D6F64653A2051
:102200004175746F002020202053415645205025F1
:102210003032643F20202020202020002020202059
:1022200053415645205025642D3F2020202020205A
:1022300020005A313A20414D20257320205025306E
:102240003264005A313A20414D2025732020502518
:10225000642D00202534644B487A005A313A2046D8
:102260004D20257320205025303264005A313A2009
:10227000464D20257320205025642D002533642EE3
:10228000253031644D487A00000000000000000055
:10229000000000000000000000000000000000003E
:1022A000000000000000000020202020202020202E
:0122B000002D
:1022B400253364004D757465005A323A2025730045
:1022C4005A323A20414D202534644B487A2020204C
:1022D400005A323A20464D202533642E253031648D
:1022E4004D487A2020005A323A202020202D4F4693
:0B22F400462D2020202020202020006C
:10230000000100005C1B0000010200005F1B0000D8
:1023100002040000631B000003080000711B0000A2
:1023200004100000661B0000062000006D1B00006A
:1023300007400000691B000005800000741B0000BE
:10234000B4290000CDDB0000082A0000BDDC00003D
:102350001D2A000009E00000322A0000EDE1000023
:10236000472A0000CDE400005C2A0000EDE60000F2
:10237000712A000089E900000000000039F800001F
:102380000100000055F800000200000091F8000074
:102390000300000029F900000000000021100000E7
:1023A000422000006330000084400000A55000007F
:1023B000C6600000E770000008810000299100005D
:1023C0004AA100006BB100008CC10000ADD100003B
:1023D000CEE10000EFF10000140015001600180017
:1023E00019001B001C001E002000220024002600F3
:1023F00028002A002D002F003200350038003C0054
:102400003F00430047004B004F00540059005E005E
:1024100064006A00700077007E0085008D009600E1
:102420009F00A800B200BC00C800D300E000ED008F
:10243000FB000A011A012B013C014F0163017801E5
:102440008E01A601BF01D901F50113023302540226
:1024500077029C02C402EE021A0349037B03B00315
:10246000E80323046204A504EB0436058505D805BA
:1024700031068F06F2065C07CB074208BF08430906
:10248000D009650A020BA90B5A0C160DDC0DAE0E15
:102490008D0F791073117C129413BD14F715451725
:1024A000A6181B1AA81B4B1D071FDE20D122E124F2
:1024B00010276129D42B6D2E2D3117342D37723A08
:1024C000E93D944177459549F14D4C4154452046AD
:1024D000554C4C004C4154452048414C46004C4121
:1024E0005445204F4646004551204F4E004551204F
:1024F0004F464600526573746F726520446566618D
:10250000756C742E2E2E202000564F4C202D0A0064
:10251000564F4C202B0A00434553372E310A004EAC
:10252000454F3A360A005355522E4D4F44450A0046
:1025300050524F4C4F474943204949780A00494E71
:10254000505554380A00494E505554370A00494EE8
:10255000505554360A00494E505554350A00494EDC
:10256000505554340A00494E505554330A00494ED0
:10257000505554320A00494E505554310A005345C3
:102580005455500A002B0A002D0A00760A005E0AF4
:1025900000505245534554203E0A003C20505245BD
:1025A0005345540A00414D0A00464D0A00504F570A
:1025B00045520A0025733A2573005A313A20417575
:1025C000746F205365656B2E2E2E202533640041D9
:1025D0004E414C4F4700434F415849414C00544FE6
:1025E000534C494E4B004661696C206D616C6C6FB9
:1025F000632073656E5F627566004661696C206D6D
:10260000616C6C6F6320726563765F6275660055FE
:1026100070646174696E672E2E2E004F4B004572F8
:102620006173653A253035580050726F6772616D7D
:102630003A2530355800746F205365747570204DFD
:10264000656E752020202020202000507265737355
:1026500020454E54455220726573746F7265200098
:1026600072756E204175746F2053657475702061AA
:102670006761696E00436F7272656374206F757471
:1026800070686173652053504B00496E207068611B
:102690007365004F7574207068617365005345540D
:1026A00000253364487A0025332E316664420025C4
:1026B000332E316666742025322E31664D00546FFC
:1026C00074616C2025316420537065616B65727391
:1026D000202020200059657300204E6F004E2F41AE
:1026E000002E00504C4541534520434845434B2E56
:1026F0002E2E202020202000535045414B455220B3
:102700004E4F5420464F554E44202020005A313A17
:10271000202020202D4F46462D2020202020202024
:1027200020002020202020002D4F46462D005A3129
:102730003A202573004454532039362F3234004D4B
:1027400061747269780044697363726574650043EB
:10275000455320372E31204F4E004454532D4553BE
:1027600000445453004454532043455320372E31E2
:10277000204F4E00444F4C42592044494749544150
:102780004C20455800444F4C425920455820434561
:102790005320372E31204F4E00444F4C4259204495
:1027A00049474954414C204558204F464600444F24
:1027B0004C4259204449474954414C20352E310060
:1027C000444F4C4259204449474954414C204558B4
:1027D000204F4E00444F4C425920352E3120434566
:1027E0005320372E31204F4E00444F4C4259204445
:1027F00049474954414C20322E3000444F4C4259F5
:1028000020504C204949782000444F4C42592050D8
:102810004C204949202000444F4C42592043455305
:102820000048616C6C004C697665002000444F4C98
:102830004259204865616470686F6E652000416C84
:102840006C2053746572656F00416C6C204D6F6E27
:102850006F0043455320372E310043696E656D612B
:1028600000445453204E454F3A3600444F4C425991
:1028700020504C20494978004D75736963004D6FB5
:1028800076696500444F4C425920504C204949001C
:102890003139326B487A002039366B487A0020345F
:1028A000342E316B487A002034386B487A0050431C
:1028B0004D004E4F205349474E414C0050434D2050
:1028C0002020202020202034386B487A0053746563
:1028D00072656F00427970617373004D75746500A5
:1028E000253364004D617920333020323030370099
:1028F00056312E312E380025732020257300372EB7
:1029000031434820494E2020202000494E50555444
:102910002038202020202000494E505554203720B8
:102920002020202000494E505554203620202020C1
:102930002000494E505554203520202020200049A9
:102940004E5055542034202020202000494E505510
:10295000542033202020202000494E50555420324E
:10296000202020202000494E505554203120202086
:0329700020200024
:102974000000000000000000000000000000000053
:102984000000000000000000000000000000000043
:102994000000000000000000000000000000000033
:1029A4000000000000000000000000000000000023
:1029B4004175746F20536F756E64205345545550A0
:1029C4003F20202000507265737320454E544552B9
:1029D40020746F2053746172740050726573732095
:1029E400454E544552206E6F77202020202000430E
:1029F4006F6E6E656374204D6963726F70686F6E7D
:102A0400653F2000537065616B65722043686563A0
:102A14006B202020202020200053657420446973FB
:102A240074616E63652020202020202020005365DF
:102A3400742042616C616E63652020202020202078
:102A44002020005365742043726F73736F76657230
:102A540020506F696E74730053657420526F6F6DEC
:102A64002045512020202020202020200053657460
:102A740020537065616B65722070686173652020F6
:022A8400200030
:102A88000000000000000000FF000000000000003F
:102A9800000000000000000000000000000000002E
:102AA800000000000000000000000000000000001E
:102AB800000000000000000000000000000000000E
:102AC80000000000000000000000000000000000FE
:102AD80000000000000000000000000000000000EE
:102AE80000000000000000000000000000000000DE
:102AF80000000000000000000000000000000000CE
:102B080000000000000000000000000000000000BD
:102B180000000000000000000000000000000000AD
:102B2800000000000000000000000000000000009D
:102B3800000000000000000000000000000000008D
:102B4800000000000000000000000000000000007D
:102B5800000000000000000000000000000000006D
:102B6800000000000000000000000000000000005D
:102B7800000000000000000000000000000000004D
:102B880000000000000000000C01C03B6FE9E23BC0
:102B9800FA97243CC748763CDCB9B03CABB2EF3C72
:102BA8000A0F1A3D80D63C3DD2005E3D15747B3D30
:102BB80036AC893D6A14923DE86B963DE86B963DCC
:102BC8006A14923D36AC893D15747B3DD2005E3D5A
:102BD80080D63C3D0A0F1A3DABB2EF3CDCB9B03CA5
:102BE800C748763CFA97243C6FE9E23B0C01C03BAE
:102BF8000000000080150000002B0000404300008A
:102C0800003D0300C06E00004087000000B10000D6
:102C180000C30000C0DC000080F20000400E01008C
:102C2800401201000022010080330100C05701005A
:102C3800405F0100406D0100008C010000AB010005
:102C4800C0CA010000EA010080090200C029020090
:102C580000440200405E020080790200C08D02003C
:102C680080980200C09C0200809D020080AE020095
:102C780040C3020000D8020040EA020080000300BE
:102C880000170300402E030000800300408E03005D
:102C98000A0500000300020000000000A000000078
:102CA80000007041A100000000006041A200000087
:102CB80000005041A300000000004041A4000000B3
:102CC80000004041A500000000004041A6000000AF
:102CD80000004041A700000000003041A8000000AB
:102CE80000002041A900000000002041AA000000C7
:102CF80000001041AB00000000001041AC000000D3
:102D08000000F040AD0000000000E040AE00000010
:102D18000000D040AF0000000000C040B00000003C
:102D28000000A040B10000000000A040B200000078
:102D38000000A040B30000000000A040B400000064
:102D480000008040B500000000006040B6000000B0
:102D580000004040B700000000000040B80000003C
:102D68000000C03FB90000000000803FBA0000002A
:102D780000000000BB00000000000040BC00000094
:102D8800000000C0BD000000000000C0BE00000040
:102D98009A99D93F0000000000000000190028009F
:102DA80032003F00500064007D000A000A000A005B
:102DB8000A000A000A000A005000FA002003C409A9
:102DC800401FD430803E28007D009001E204A00F0F
:102DD8006A18401F15001A001F00240029002E0041
:102DE800330038003D00420047004C0051005600B7
:102DF8005B00600065006A006F00740079007E0067
:102E0800830088008D00920097009C00A100A60016
:102E1800AB00B000B500BA00BF000A010F011401F1
:102E280019011E0123012801C400C900CE00D300E6
:102E3800D800DD00E200E700EC00F100F600FB003E
:102E4800000105012530385820000A000A52656142
:102E5800643A253036580A000000000000000000DF
:072E6800286E756C6C290057
:102E700090040040910400409404004095040040F8
:102E8000980400409F040040A0040040A8040040B3
:102E9000A8040040AD040040B0040040CE0400404F
:102EA000D0040040D2040040D4040040F8040040A4
:102EB000F8040040080500400805004014050040E3
:102EC000140500406B0500406C050040850500407E
:102ED000880500408C1D00408C1D0040B41D004042
:102EE000B41D0040D11D0040D41D0040331F0040E0
:102EF000341F00403C1F00403C1F0040591F004051
:102F00005C1F0040911F0040941F0040981F00402C
:102F1000981F0040AD220040B0220040B422004083
:102F2000B4220040BE240040C0240040C72400401A
:102F3000C8240040CC240040000000000000000035
:102F4000A8040040AC0400408A841201040500403B
:102F50000505004001000000180500406B05004019
:102F60000120202020202020202020202020202080
:102F70002020202020202020202020202020202051
:102F80002020202020202020200020202020202061
:102F90002020202020202020202020202020202031
:102FA0002020202020202020202020202020202021
:102FB000202000007C0500407D050040010000004D
:102FC000880500408C050040C18B0000C91D0040F1
:102FD000CA1D004003000000D81D00401C1F004017
:102FE000E81D0000F01D0000F81D0000001E00009C
:102FF000081E0000101E0000181E0000201E000009
:10300000281E0000A81D0000901D0000981D000053
:10301000A01D0000881D0000E01D0000681D0000CC
:10302000701D0000781D0000801D0000B01D000014
:10303000B81D0000C81D0000D01D0000C01D00000C
:10304000D81D0000301E0000381E0000401E000089
:10305000481E0000501E0000581E0000601E0000A8
:10306000281D0000181D0000201D0000401D00004C
:10307000301D0000381D0000481D0000501D0000DC
:10308000101D0000681E0000701E0000781E000069
:10309000801E0000881E0000901E0000981E000088
:1030A000A01E0000A81E0000B01E0000B81E0000F8
:1030B000C01E0000C81E0000D01E0000D81E000068
:1030C000E01E0000E81E0000F01E0000401F00008F
:1030D000481F0000501F0000581F0000601F000024
:1030E000681F0000701F0000381F0000F81E00005D
:1030F000001F0000081F0000101F0000181F000024
:10310000201F0000281F0000301F0000781F000053
:10311000001D0000081D0000581D0000601D00007B
:1031200000000000301F0040311F0040010000007F
:103130003C1F0040591F0040A0210000B8210000A2
:10314000A8210000B0210000C0210000C82100001B
:1031500000000000010000005C1F0040741F0040E0
:1031600012020000A406000012020000CC5501006B
:10317000E0A50100CC550100821F0040831F0040E4
:103180000A000000851F0040891F00400101010165
:103190008A1F00408B1F004001000000981F004064
:1031A0000420004008200040282100403820004032
:1031B00098200040F8200040C820004068200040CF
:1031C0005821004000000000662900005929000035
:1031D0004C2900003F290000322900002529000069
:1031E000182900000B290000FE28000009220040D9
:1031F0001622004023220040302200403D220040A1
:103200004A2200405722004064220040FC21004036
:1032100008200040A821004000000000000000003D
:10322000000000000000000000000000000000009E
:10323000000000000000000000000000000000008E
:10324000000000000023000000000000000000005B
:10325000000000000000000000000000000000006E
:10326000000000000000000000000000000000005E
:10327000000000001023000000000000000000001B
:10328000000000000000000000000000000000003E
:10329000000000000000000000000000000000002E
:1032A00000000000182300000000000000000000E3
:1032B000000000000000000000000000000000000E
:1032C00000000000000000000000000000000000FE
:1032D00000000000202300000000000000000000AB
:1032E00000000000000000000000000000000000DE
:1032F00000000000000000000000000000000000CE
:103300000000000028230000000000000000000072
:1033100000000000000000000000000000000000AD
:10332000000000000000000000000000000000009D
:10333000000000003023000000000000000000003A
:10334000000000000000000000000000000000007D
:10335000000000000000000000000000000000006D
:103360000000000008230000000000000000000032
:10337000000000000000000000000000000000004D
:10338000000000000000000000000000000000003D
:103390000000000038230000402300004823000004
:1033A0005023000058230000682300006023000021
:1033B0007023000000000000B0210040D021004038
:1033C0008823000078230000902300008023000061
:1033D00000000000DE250000D6250000CF250000FB
:1033E000882200409D2200402020202020202020F4
:1033F000202020202020202020202020000000004D
:10340000E6230040E823004001010000A52400401D
:10341000A724004001010000C3240040C424004050
:1034200003000000000000000000000000B5011CC7
:10343000081C002803D0044800F060F802E00348AC
:1034400000F05CF800BDC0465112000050120000B0
:1034500000B5074800F052F8064800F04FF806485B
:1034600000F04CF80548007800F00AF800BDC046AE
:10347000FF100000FF11000050120000A21D0040CC
:1034800000B5011C081C002803D0044800F036F8E1
:1034900002E0034800F032F800BDC046801300008F
:1034A0000013000030B5051C1048002101F00EFE8D
:1034B000002411E00E48002101F0EAFD291C0D480E
:1034C00001400D4801F0E4FD0948012101F0E0FD53
:1034D0006D0001342406240E201C0006000E102866
:1034E000E8DB0248012101F0F1FD30BD00004000A1
:1034F00000100000008000000020000000B5011C4A
:10350000081CFFF7CFFF00BD00B5021C101C0549C9
:1035100009780143034801700248007800F066F81A
:1035200000BDC0469004004000B5011C081C000608
:10353000000E02061216D2431206120E044801783B
:10354000114001700248007800F050F800BDC046FC
:103550009004004000B5011C081C0006000E00F09D
:103560001DF80448012101F0B1FD0248002101F0DD
:10357000ADFD00BD0000001000B5011C081C0006D8
:10358000000E00F00BF80448012101F09FFD0248F5
:10359000002101F09BFD00BD0000040030B5051CBA
:1035A000002415E0281C0106090E802001400D486A
:1035B00001F08CFD0C48002101F06AFD6D002D0624
:1035C0002D0E0948012101F063FD01342406240E6B
:1035D000201C0006000E0828E4DB0248012101F04F
:1035E00075FD30BD000000200000100000B5011C7A
:1035F000081C0006000EFFF7D1FF0448012101F06E
:1036000047FD0248002101F043FD00BD000080009D
:1036100070B5051C002412E00C2000F033F8061CE5
:10362000301C0006000E1021084203D0012002F0D9
:1036300047FA01E000200BE001342406240E281C88
:103640000106090E201C0006000E8842E4D301206A
:1036500070BDC04630B50C1C051C094893B06946C6
:10366000132304C804C15B1EFBD1281C0006000EF6
:10367000211C0906090E01F05DFA13B030BDC046E9
:103680002801000010B5041C094893B069461323B3
:1036900004C804C15B1EFBD1201C0006000E01F013
:1036A000D5F913B00006000E0006000E10BDC0468E
:1036B0002801000000B50021081CFFF7CBFF012006
:1036C0008421FFF7C7FF05208521FFF7C3FF0620F0
:1036D0001021FFF7BFFF04209821FFF7BBFF00BDBB
:1036E00000B51820FFF7CEFF011C081C0006000ED5
:1036F0001E2801DA0C210EE0081C0006000E22280C
:1037000001DA042107E0081C0006000E422801DA55
:10371000002100E00121081C0006000E00BDC0468B
:1037200010B4031C1B0AFF2423401B061B0E1A1C8B
:103730001206120E072A20DC021C22401206120E6C
:10374000081C002809D0141C181C0106090E0C487E
:1037500040180178214301700FE0101C0006000E94
:1037600002061216D2431206120E181C0106090E8A
:103770000348401801781140017010BC7047C046E2
:103780009804004010B5002418E0201C0106090E22
:103790000D48405C0006000E00060016C043FFF70F
:1037A000EBFE201C0106090E0848405C00F010F8F2
:1037B000FF20FFF7E1FE01342406240E201C000642
:1037C000000E0728E1DB10BD7401000098040040E2
:1037D00030B5051C1048002101F05AFC002415E00A
:1037E000281C0106090E802001400C4801F06EFCE7
:1037F0000948012101F04CFC6D002D062D0E0648F4
:10380000002101F045FC01342406240E201C000692
:10381000000E0828E4DB30BD000020000000000896
:1038200001B500990348405C011C022000F0BAF881
:1038300001B000BD1C02000011B500980C490968D8
:10384000814208D089000A4C0A4840580021FFF7FD
:1038500067FF0098206006480168890005484058C5
:103860000121FFF75DFFFFF78DFF01B010BDC046DE
:10387000A0040040C801000010B500240BE0201C8B
:103880000106090E8900094840580021FFF748FF4A
:1038900001342406240E201C0106090E8900034869
:1038A00040580028EBD1FFF76DFF10BDC8010000A4
:1038B00011B5009811490968814208D089000F4C60
:1038C0000F4840580021FFF72BFF009820600B485D
:1038D000016889000A4840580121FFF721FFFFF7DE
:1038E00051FF0098012804DB072802DC00F088F86B
:1038F00002E0002000F084F801B010BDA4040040F4
:10390000F001000001B512480021FFF709FF11483E
:103910000021FFF705FFFF200021FFF701FF0098BE
:10392000012808D002280BD000280DD10848012119
:10393000FFF7F6FE08E007480121FFF7F1FE03E07C
:10394000FF200121FFF7ECFEFFF71CFF01B000BDD7
:10395000C0020000FF01000070B5051C0124FFF744
:103960008BFF281C0006000E002800D1022412E064
:10397000281C0006000E211C0906090E00F090F814
:10398000061C301C002803D0201C0006000E08E096
:1039900001342406240E201C0006000E0328E7DD57
:1039A000002070BD30B50C1C051C094893B0694659
:1039B000132304C804C15B1EFBD1281C0006000EA3
:1039C000211C0906090E01F0B5F813B030BDC04640
:1039D0007C01000030B50C1C051CFFF74DFF281CB6
:1039E0000006000E211C0906090E00F059F8011C02
:1039F000081C002801D0012000E0002030BDC04696
:103A000001B500990348405C011C0320FFF7CAFF81
:103A100001B000BD2B02000000B5011C081C0028ED
:103A200004D00121081CFFF7BDFF03E001200021A5
:103A3000FFF7B8FF00BDC04630B5051C00240CE000
:103A4000281C02F03DF8084801F050FB002801D185
:103A5000012008E001342406240E201C0006000E7C
:103A60000A28EDDB002030BD0000010030B5051C48
:103A700000240CE0281C02F023F8084801F018FB91
:103A8000002801D1012008E001342406240E201C66
:103A90000006000E0A28EDDB002030BD00000020EB
:103AA00030B50D1C021C101C0006000E082800D1A9
:103AB0008CE0101C0206120E12011206120EF020EB
:103AC0000240291C0A43101C02282DD003282DD0A7
:103AD00011282DD012282DD013282DD021282DD0FB
:103AE00022282DD023282DD031282DD032282DD09A
:103AF00033282DD041282DD042282DD043282DD039
:103B000051282DD052282DD053282DD061282DD0CA
:103B100062282DD063282DD071282DD072282DD069
:103B200073282DD001282CD100242AE0002428E07D
:103B3000012426E0082424E0012422E0022420E0DD
:103B400009241EE002241CE003241AE00A2418E0E1
:103B5000032416E0042414E00B2412E0042410E0F3
:103B600005240EE00C240CE005240AE0062408E0FD
:103B70000D2406E0062404E0072402E00E2400E001
:103B80000724281C0006000E03280FD1201C000665
:103B9000000EFFF751FE3220FFF768FF0006000E0F
:103BA00000281CD1281C0006000E19E0201C00066D
:103BB000000EFFF735FE1E20FFF72AFD0006000E5F
:103BC00000280CD1281C0006000E09E03220FFF767
:103BD00033FF0006000E002801D1012000E0002084
:103BE00030BDC04600B5011C081C002803D0802051
:103BF000FFF78AFC02E08020FFF796FC00BDC0467C
:103C000000B5011C081C0006000E012803D100208D
:103C100000F072F802E0012000F06EF800BDC0462E
:103C200000B5011C081C0006000E012803D100206D
:103C300000F054F802E0012000F050F800BDC0464A
:103C400000B5011C081C0006000E012803D101204C
:103C500000F036F802E0002000F032F800BDC04667
:103C600000B5011C081C0006000E012803D100202D
:103C700000F050F802E0012000F04CF800BDC04612
:103C800000B5011C081C0006000E012803D100200D
:103C900000F05CF802E0012000F058F800BDC046DA
:103CA00000B5011C081C0006000E012803D10020ED
:103CB00000F03EF802E0012000F03AF800BDC046F6
:103CC00000B5011C081C002803D00120FFF71CFCD4
:103CD00002E00120FFF728FC00BDC04600B5011C32
:103CE000081C002803D00220FFF70EFC02E002208F
:103CF000FFF71AFC00BDC04600B5011C081C0028D7
:103D000003D00420FFF700FC02E00420FFF70CFCC6
:103D100000BDC04600B5011C081C002803D00820C7
:103D2000FFF7F2FB02E00820FFF7FEFB00BDC046F4
:103D300000B5011C081C002803D03020FFF7E4FB6D
:103D400002E03020FFF7F0FB00BDC04600B5011CCB
:103D5000081C002803D04020FFF7D6FB02E04020DB
:103D6000FFF7E2FB00BDC04630B5051C081C00F0A3
:103D70006FF8011C281C0006000EF02210402028BD
:103D80000BD0302811D010280FD1081C0406240EA7
:103D9000194804432404240C0EE0081C0406240ED5
:103DA000164804432404240C06E0081C0406240ED0
:103DB000134804432404240C1248012101F086F91D
:103DC000281C0106090E0F2001400F48405C000628
:103DD000000E00060016C043FFF7BCFB201C0004C9
:103DE000000C00F013F8FF20FFF7B4FB054800219A
:103DF00001F06CF930BDC04600EB000000F300009C
:103E000000CB0000000008003402000030B5051CA3
:103E1000002411E00B48002101F058F9291C0A4840
:103E200001400A4801F034F90648012101F04EF939
:103E30006D0001342406240E201C0006000E1028FC
:103E4000E8DB30BD000008000080000000004000FA
:103E500000B5021C101C07490FF02AFF021C06497E
:103E6000101C0FF07BFE10F0C9F8011C081C0006A6
:103E7000000E00BD000000400000604370B5151C3E
:103E80000E1C031C281C0006000E012808D1244823
:103E90001B18181C322111F093F8081C041C08E0B0
:103EA00020481B18181C0A2111F08AF8081C041C51
:103EB00024011D48002101F009F9282000F00EF925
:103EC0001948012101F002F9201CFF21084000F0EF
:103ED00005F9201C000AFF21084000F0FFF8301C03
:103EE00000280CD0281C0006000E012803D13E201B
:103EF00000F0F4F80FE08C2000F0F0F80BE0281C44
:103F00000006000E012803D13A2000F0E7F802E095
:103F1000882000F0E3F80448002101F0D7F870BDD4
:103F2000CC290000C201000000000200F0B51C1CFA
:103F3000151C0E1C071C1048002101F0C7F8381C86
:103F40000006000E00F0CAF80B48012101F0BEF88F
:103F5000301C0006000E00F0C1F8281C0006000E00
:103F600000F0BCF8201C0006000E00F0B7F8024874
:103F7000002101F0ABF8F0BD0000020030B50024D4
:103F80001548002101F0A2F82A2000F0A7F81248F5
:103F9000012101F09BF8002512E01048002101F0FA
:103FA00077F864000D48012101F072F80C4801F027
:103FB0007FF8002801D00120044301352D062D0E85
:103FC000281C0006000E1828E7DB0348002101F03A
:103FD0007DF8201C30BDC046000002000000000437
:103FE0000000000200B5011C081C01280FD00228A7
:103FF00017D003281DD0002822D162211D4801704E
:10400000007900281CD1E2211A48017018E00A2129
:10401000184801700079002812D18A2115480170D2
:104020000EE001211348017101787F2211400170D7
:1040300006E000210F4801710178802211430170D0
:104040000D480078002806D00A480178DF2001409A
:104050000848017005E00748017820200143054821
:1040600001700448017842788078031C2920FFF70A
:104070005DFF00BDA8040040AB04004000B5011C7A
:10408000081C0006000E012803D10120FFF7AAFF3B
:1040900002E00020FFF7A6FF00BDC04600B5011CEE
:1040A000081C002807D001210B48C1700178DF22CD
:1040B0001140017006E000210748C17001782022FC
:1040C000114301700448017842788078031C29204C
:1040D000FFF72CFF00BDC046A804004030B5051C0A
:1040E000002413E00C48002100F0D2FF281C010638
:1040F000090E01200140094800F0CAFF06480121CD
:1041000000F0C6FF6D0801342406240E201C0006B2
:10411000000E0828E6DB30BD0000000400000008A7
:10412000011C081C0006000E0A2807D10D220E48AB
:1041300002700E48007820221042FAD00A1C0A4869
:1041400002700A48007820221042FAD0081C0006AB
:10415000000E0D2807D10A2103480170034800789A
:1041600020210842FAD0704700C000E014C000E0EF
:1041700000B5021C832109480170111C084810F089
:1041800043FF081C0106090E06480170002106487D
:10419000017003210148017000BDC0460CC000E061
:1041A0000018150000C000E004C000E000B503489E
:1041B00000F036F8024800F091F800BD80250000BC
:1041C00000C201000F592DE940009FE50000D0E535
:1041D0000E0000E2040050E30700001A30009FE5E3
:1041E0000010D0E50100A0E1001CA0E1211CA0E12D
:1041F00020009FE5000090E5A70700EB0010A0E37A
:1042000014009FE5001080E50F59BDE804F05EE260
:1042100008C000E000C000E0D41D004030F0FFFF07
:1042200000B5011C0523154802681A430260081CEA
:10423000FFF79EFF012112480170124912480160E8
:104240002621124801604022114801681143016093
:104250000C2010F0DBFD0F4908600F490D48006885
:10426000018100890004001410F0D0FD011C0948F0
:104270000068016001F0D8FE00BDC04600C002E049
:1042800004C000E0C441000000F1FFFF00F2FFFFA6
:1042900010F0FFFFD41D00400001000003002DE9D5
:1042A00028009FE50000D0E50E0000E2040050E386
:1042B0000100001A18009FE50000D0E50010A0E3FF
:1042C00010009FE5001080E50300BDE804F05EE209
:1042D000080001E0000001E030F0FFFF00B5021C23
:1042E0000B4B0C4801681943016083210A48017097
:1042F000111C0A4810F088FE081C0106090E084827
:10430000017000210748017003210348017000BDBE
:104310000000010000C002E00C0001E000181500E0
:10432000000001E0040001E000C09FE51CFF2FE158
:1043300035430000F0B50A1C071C0023381C0FF0A1
:1043400033FEA34C211C10F01DFE09D3381C0FF0C6
:104350002BFEA04C211C10F015FE01D8012600E018
:104360000026381C0FF020FE9B4C211C10F00AFE8A
:1043700009D3381C0FF018FE984C211C10F002FED7
:1043800001D8012400E0002495480078011C002990
:1043900007D1111C002900D117E1012790490F70A6
:1043A00013E101281AD100218E48018000218E4896
:1043B000017002218A480170301C002803D00021BE
:1043C0008A48017001E1201C002803D001218748A0
:1043D0000170FAE0002182480170F6E0834800781D
:1043E000002821D07F48018849007E480180101CA8
:1043F0000006000E002805D17A48018801200143FB
:10440000784801807848017801310170301C00281B
:1044100003D00021754801700EE0201C0006000E3C
:10442000002809D1012307E0301C002803D0012116
:104430006E48017000E001236B4800780C2810D111
:10444000101C0006000E00280BD1684800780028D8
:1044500007D0644801884900624801800D21624804
:104460000170181C00280AD000215D480170101C42
:10447000002800D1A9E0012159480170A5E05A485F
:1044800000780D2800D0A0E0564801880C1CA00937
:104490001F221040132835D155480578E20A012023
:1044A00002401206120E52480270281C0206120E1A
:1044B0004F480078904206D10A1C3F2002404D48E8
:1044C000007882420DD00A1C3F210A401206120ECB
:1044D00048490A70012248490A70002247490A7077
:1044E00070E000F0C1F900286CD044480178081C45
:1044F000032803DD01224048027063E03F48013198
:1045000001705FE0A0091F210840122844D13848FB
:10451000057834480088011CC90A012001400906B9
:10452000090E33480170281C0106090E3048007836
:10453000884208D12B480088011C3F2001403048A8
:104540000078814213D0274909880A1C3F210A407C
:104550001206120E2A490A702A490978002902D047
:10456000012229490A70002224490A702AE000F039
:104570006BF9002826D021480178081C032807DDA4
:104580002048007800281DD001221F48027019E041
:104590001A480131017015E00221174801701148D5
:1045A0000088011C3F2001400906090E11480170D6
:1045B0000C480088011C89091F2001400906090ECA
:1045C00012480170002106480170F0BC08BC184771
:1045D00098FF28463CBDDE46501EEE46E02D3C4787
:1045E000C5040040B0040040C4040040C6040040BC
:1045F000C7040040B5040040B4040040C8040040B3
:10460000B804004004050040B7040040B604004070
:1046100000C09FE51CFF2FE11D46000070B50A1C7D
:10462000061C0023301C0FF0BFFC7A4C211C10F03C
:10463000A9FC09D3301C0FF0B7FC774C211C10F0FB
:10464000A1FC01D8012500E00025301C0FF0ACFCD6
:10465000724C211C10F096FC09D3301C0FF0A4FC06
:104660006F4C211C10F08EFC01D8012400E00024C6
:104670006C480078002807D1111C002900D1C6E041
:10468000012668490E70C2E001281AD1002166484F
:104690000180002165480170022162480170281CD8
:1046A000002803D0002162480170B0E0201C0028DF
:1046B00003D001215E480170A9E000215948017032
:1046C000A5E05B480078002821D0574801884900C0
:1046D00055480180101C0006000E002805D15248E4
:1046E0000188012001435048018050480178013180
:1046F0000170281C002803D000214D4801700EE0F5
:10470000201C0006000E002809D1012307E0281C08
:10471000002803D001214648017000E001234348EE
:1047200000780C2810D1101C0006000E00280BD1B8
:104730003F480078002807D03B48018849003A48A4
:1047400001800D2139480170181C002809D0002172
:1047500034480170101C002859D0012131480170E3
:1047600055E0324800780D2851D12F480688321C78
:1047700094091F25201C2840122835D12D48017886
:10478000D20A012002401206120E2A480270081CAA
:104790000106090E27480078884206D1311C3F20C7
:1047A00001402548007881420DD0321C3F210A404B
:1047B0001206120E20490A70012220490A700022B6
:1047C0001F490A7020E000F03FF800281CD01C4868
:1047D0000178081C032803DD01221848027013E049
:1047E0001748013101700FE0022114480170311C9B
:1047F0003F2001400906090E0F480170211C294085
:104800000906090E0F48017000210648017070BCAE
:1048100008BC184798FF28463CBDDE46501EEE46B1
:10482000E02D3C47CA040040B2040040C9040040E7
:10483000CB040040CC040040B8040040B704004062
:10484000CD040040B9040040011C081C0006000E05
:10485000132804D0081C0006000E102801D10120E6
:1048600000E000207047C046021C002113E0081C35
:1048700003061B0E0D48C35C181CFF2801D1002045
:1048800012E0101C0006000E984201D101200BE03E
:1048900001310906090E06480078031C081C0006B1
:1048A000000E9842E3D300207047C046BA0400408F
:1048B000C104004000B50448FF21072210F092FA1D
:1048C00000210248017000BDBA040040C10400404C
:1048D00030B5051C0C480078072812DA281C0006A1
:1048E000000EFFF7C1FF0006000E002809D12A1CA8
:1048F0000649C879041C054B1A550130C8710120BE
:1049000000E0002030BDC046C1040040BA040040B1
:1049100010B400231A1C0FE0191C0C06240E2349A6
:10492000095D0C1C011C0906090EA14201D10122DE
:104930000AE001331B061B0E1D4909780C1C191CCB
:104940000906090EA142E7D31BE0181C0006000E61
:1049500001301749097888420ADA181C0106090E45
:104960001448405C191C0C06240E1049085505E03B
:10497000FF20191C0C06240E0C49085501331B0698
:104980001B0E0B4801780C1C181C0006000EA042E0
:10499000DBD3002907D0101C0006000E012802D12D
:1049A00003480139017010BC7047C046BA0400408A
:1049B000C1040040BB040040F0B50E1C051C81B0D2
:1049C00006AC002100A8017035E000211D480170EF
:1049D000201C806900F00CF9201C00F0A5F9201CB7
:1049E0000178201C00F0FCF900270BE0381C0206BF
:1049F000120E301C805C011C201C00F0F1F9013704
:104A00003F063F0E281C0106090E381C0006000E4A
:104A10008842EBD3201C00F0BDF9201C406C00F054
:104A2000E7F808480078002801D1002008E000A835
:104A300001780131017000A800780328C5DB024825
:104A400001B0F0BDD0040040FFFFFFFFF0B5071C30
:104A500082B0391CFF2001400906090E01A801702F
:104A60003E1C31480640F6090E2006403606360E3A
:104A700007AD002450E000212C480170281C8069FB
:104A800000F0B6F8281C00F04FF9381CFF2809D9AF
:104A9000281C0178301C0006000E0143281C00F081
:104AA0009FF904E0281C0178281C00F099F901A85E
:104AB0000078011C281C00F093F9281C00F034F940
:104AC000381CFF280BD9281C0178301C0006000E6A
:104AD000014301200143281C00F082F906E0281C54
:104AE000017801200143281C00F07AF9281C00F00D
:104AF000D1F900A90870281C002100F081F8281CB9
:104B000000F048F909480078002802D100A8007890
:104B100008E001342406240E201C0006000E0328A1
:104B2000A9DB034802B0F0BD00070000D00400403C
:104B3000FFFFFFFFF0B50F1C061C82B0311CFF20E9
:104B400001400906090E00A80170311C25480140EA
:104B5000C9090E2001400906090E01A8017007AD20
:104B6000002436E0002120480170281C806900F0F4
:104B70003FF8281C00F0D8F8301CFF2808D9281C62
:104B8000017801A800780143281C00F029F904E00D
:104B9000281C0178281C00F023F900A80078011CCB
:104BA000281C00F01DF9381C0106090E281C00F015
:104BB00017F9281C00F0EEF8281C406C00F018F8DB
:104BC00009480078002801D1002008E001342406BB
:104BD000240E201C0006000E0328C3DB034802B08D
:104BE000F0BDC04600070000D0040040FFFFFFFFFB
:104BF000011C0138000400140029F9D17047C04697
:104C0000F0B50F1C061C454D45480078002800D023
:104C10007FE0381C022835D0012854D10120311CF6
:104C2000896810F0C6F9301C016B301C406B4018CD
:104C3000FFF7DEFF301C406AFFF7DAFF0120311C6E
:104C4000496810F0B6F9301C806AFFF7D1FF301CBC
:104C5000006910F0ADF9002801D1002511E02F4DB9
:104C60000120FFF7C5FF013424042414301C816C9B
:104C7000201C000400148842E9DB2A480178013135
:104C800001702CE0301C406AFFF7B2FF0020311C9D
:104C9000896810F08EF9301C016B301C806B401855
:104CA000FFF7A6FF301C406AFFF7A2FF0120311C6E
:104CB000496810F07EF9301C816A301C406B401846
:104CC000FFF796FF0BE00120311C496810F071F9E5
:104CD000301C816A301C406B4018FFF789FF0020B0
:104CE000311C496810F065F9301C416A301C806B3A
:104CF0004018FFF77DFF381C0006000E022808D17F
:104D00000120311C896810F054F9301C406BFFF70A
:104D10006FFF281C00040014F0BDC046FFFF000018
:104D2000D1040040D004004010B5041C184800789D
:104D300000282CD10120211C896810F03AF9201C90
:104D4000406AFFF755FF0120211C496810F031F936
:104D5000201C016A201C406B4018FFF749FF00200F
:104D6000211C896810F025F9201CC169201C806B6A
:104D70004018FFF73DFF0020211C496810F019F989
:104D8000201C416A201C806B4018FFF731FF10BDCA
:104D9000D104004010B5041C00211048017000200F
:104DA000211C896810F005F9201C406AFFF720FFDC
:104DB0000120211C496810F0FCF8201CC16B201C4C
:104DC000406B4018FFF714FF0120211C896810F088
:104DD000F0F8201C406BFFF70BFF10BDD104004022
:104DE00070B50E1C041C2948007800284CD1002501
:104DF00036E0201C406AFFF7FBFE301C0006000E68
:104E00008021084205D00120211C896810F0D1F8CA
:104E100004E00020211C896810F0CBF8201C006BF6
:104E2000FFF7E6FE0120211C496810F0C2F8201CA3
:104E3000816A201C406B4018FFF7DAFE0020211C1D
:104E4000496810F0B6F8201CC16A201C806B40181D
:104E5000FFF7CEFE76003606360E01352D062D0EF6
:104E6000281C0006000E0828C3DB201C0121FFF7C8
:104E7000C7FE07480078002803D0012103480170CD
:104E800002E000210148017070BDC046D10400401D
:104E9000D004004070B5061C00240120311C896834
:104EA00010F087F81E480078002835D100252EE044
:104EB00064002406240E301C4069FFF799FE01208F
:104EC000311C496810F075F8301C406BFFF790FEFC
:104ED000301C006910F06CF8002802D00120044357
:104EE000FFE7301C806AFFF783FE0020311C496811
:104EF00010F05FF8301C016C301C806B4018311CC6
:104F0000496A4018FFF774FE01352D062D0E281C46
:104F10000006000E0828CBDB201C0006000E70BD2A
:104F2000D104004030B500241348002100F0B0F84F
:104F30001148012100F0ACF8002512E064000F4890
:104F4000002100F0C3F80E4800F0D0F8002801D08E
:104F5000012004430948012100F0B8F801352D066D
:104F60002D0E281C0006000E1828E7DBE443054838
:104F70008443201C30BDC046000002000000100029
:104F800000000040000000FF00B5011C3120FEF7CA
:104F9000EBFE00BD00B5011C3020FEF7E5FE00BDB4
:104FA00010B5011C081C0FF0A9FD114C20606168B0
:104FB000002000F01FF8E168022000F01BF82169D2
:104FC000032000F017F86169042000F013F8E1698C
:104FD000062000F00FF8216A072000F00BF8A16806
:104FE000012000F007F8A169052000F003F810BDCA
:104FF000D404004030B50B1C021C191C101C050603
:105000002D0EAD000748084C6151191C00680EF0C8
:10501000A5FD011C101C0206120E0448805CFEF760
:10502000A3FE30BDD4040040D80400403C02000080
:1050300030B5051C00240FE0201C0106090E0948AC
:10504000405C01B4281C0FF059FD011C01BCFEF7A7
:105050008BFE01342406240E201C0006000E0828B6
:10506000EADB30BD3C02000000B5011C081C002832
:1050700003D00548FFF794FF05E0044800880004CA
:105080000014FFF78DFF00BD9CFFFFFFD4210040FF
:10509000021C081C002803D0111C0348016002E018
:1050A000111C024801607047048002E00C8002E09D
:1050B000021C05480068111C0840002801D001208E
:1050C00000E000207047C046008002E0021C081C7F
:1050D000002803D0111C0348016002E0111C0248A3
:1050E00001607047148002E01C8002E0021C054849
:1050F0000068111C0840002801D0012000E00020B9
:105100007047C046108002E0011C081C002807D030
:10511000082207480260074801689143016006E0E1
:105120000822054802600348016811430160704786
:10513000048002E0088002E00C8002E0011C081CF0
:10514000002807D0042207480260074801689143FD
:10515000016006E00422054802600348016811432B
:1051600001607047048002E0088002E00C8002E0E9
:1051700009480068082208490B6893430B600749F7
:105180000968114201D0012100E00021021C0248FF
:105190000260081C7047C046088002E0008002E000
:1051A00009480068042208490B6893430B600749CB
:1051B0000968114201D0012100E00021021C0248CF
:1051C0000260081C7047C046088002E0008002E0D0
:1051D000011C081C002807D0074A0848026008483C
:1051E00001689143016006E0034A064802600448F2
:1051F000016811430160704700800000048002E0F4
:10520000088002E00C8002E0011C081C002807D086
:10521000074A08480260084801689143016006E0B7
:10522000034A064802600448016811430160704760
:1052300000002000148002E0188002E01C8002E0E0
:1052400009480068094A08490B6893430B600849FC
:105250000968114201D0012100E00021021C02482E
:105260000260081C7047C046088002E00080000011
:10527000008002E009480068094A08490B68934326
:105280000B6008490968114201D0012100E00021AA
:10529000021C02480260081C7047C046188002E0E9
:1052A00000002000108002E0054A06480168114312
:1052B0000160054A05480168114301607047C04616
:1052C00000009000088002E000000430188002E036
:1052D00000B51020FFF7ECFE00BDC04600B5024847
:1052E000FFF704FF00BDC0460000000200B520200B
:1052F000FFF7DEFE00BDC04600B5011C4020FFF7F1
:10530000C7FE00BD00B5011C0148FFF7DFFE00BD70
:105310000000000100B5011C0148FFF7B9FE00BD07
:105320000002000000B5011C0148FFF7B1FE00BDFE
:105330000004000000B5011C0148FFF7C7FE00BDD6
:105340000000800010B5041C0A480121FFF7BEFED2
:1053500009480121FFF7BAFE201C002804D00548A7
:105360000021FFF7B3FE03E003480021FFF7AEFE84
:1053700010BDC046000000800000000400B5021C03
:1053800000F032F900F010F9101C01280CD00228AE
:1053900013D0002821D11149114801602E21114854
:1053A000016000F0F9F818E00F4910480160312160
:1053B0000F48016000F010F90FE00849084801604B
:1053C0002E210848016000F0E7F80749074801600E
:1053D00031210748016000F0FFF800BDF8550000DA
:1053E00008F1FFFF08F2FFFF0058000014F1FFFF73
:1053F00014F2FFFF00B5021C00F0E6F8101C0128B3
:1054000007D0022811D000281AD101210D480170BF
:1054100016E000210B4801700B490C480160302157
:105420000B48016000F0C8F80AE00121054801704E
:1054300005490648016030210548016000F0BCF8CC
:1054400000BDC04604050040E85600000CF1FFFF17
:105450000CF2FFFF00B5002110480160FFF724FFA8
:105460000020FEF7DDFB00F02BF80020FEF7D4FA59
:1054700000F04CF800F0CEFA00F05CF800F06CF8A8
:1054800000F04AFA00F060FA00F068FA00F08AFAD8
:1054900000F0A4FA00F0E2FA00BDC04614C002E039
:1054A00000B50020FEF756F80020FEF765F800BDB5
:1054B00000B5FF20FEF74EF8FF20FEF75DF800BDB7
:1054C00000B50E4A0E480168114301600D4A0E48AE
:1054D0000168114301600020FFF716FE0120FFF76D
:1054E0002DFE0120FFF710FE0020FFF771FE0120C6
:1054F000FFF78AFE0120FFF76BFE00BD0C80000065
:10550000088002E000002000188002E0054A0648FA
:10551000016811430160054A0548016811430160B3
:105520007047C04600001000188002E00000020032
:10553000088002E0054A0648016891430160054A77
:1055400003480168914301607047C04600000800AD
:10555000088002E00000040000B50B4A0B48016817
:10556000114301600A4A0B480168114301600120A0
:10557000FFF7C2FE0120FFF7C5FE0020FFF7CAFEBD
:105580000020FFF7CFFE00BD40060000088002E0CB
:1055900000008001188002E0014902480160704764
:1055A0000040000010F0FFFF014902480160704711
:1055B0000040000014F0FFFF0149024801607047FD
:1055C0000000010010F0FFFF014902480160704730
:1055D0000000010014F0FFFF01490248016070471C
:1055E0000000020010F0FFFF01490248016070470F
:1055F0000000020014F0FFFF3F5F2DE90000A0E370
:105600000010A0E10120A0E3BC309FE50020C3E52D
:10561000B8309FE50030D3E5010013E30400000A31
:10562000A8309FE50050D3E5FE5005E20050C3E5E9
:10563000040000EA94109FE50030D1E5013083E3D7
:105640000030C1E50210A0E184209FE5003092E522
:1056500080209FE50050D2E5000055E30900000AD4
:1056600074209FE5004092E570209FE5940505E0D9
:105670000340A0E1054084E0005092E5054044E08D
:105680000D00C2E5030000EA50009FE5000090E530
:105690000340A0E1004044E00320A0E13C009FE57E
:1056A000002080E50100A0E1001CA0E1211CA0E198
:1056B0000400A0E11BFBFFEB0010A0E320009FE52E
:1056C000001080E53F5FBDE804F05EE240C11FE0EE
:1056D0004CC11FE0084000E005050040184000E014
:1056E000F804004030F0FFFF3F5F2DE90000A0E329
:1056F0000010A0E10430A0E3E0209FE50030C2E507
:10570000DC209FE50020D2E5040012E30900000A36
:10571000CC209FE50030D2E5FB3003E20030C2E54B
:10572000C0209FE50020D2E5010052E30A00001AE4
:105730000110A0E3080000EAA4209FE50030D2E5B4
:10574000043083E30030C2E598209FE50020D2E5D5
:10575000000052E30000001A0110A0E388209FE53A
:10576000003092E584209FE50050D2E5000055E32B
:105770000900000A78209FE5004092E574209FE52B
:10578000940505E00340A0E1054084E0005092E567
:10579000054044E00A00C2E5030000EA54009FE52A
:1057A000000090E50340A0E1004044E00320A0E1B8
:1057B00040009FE5002080E50100A0E1001CA0E181
:1057C000211CA0E10400A0E190FBFFEB0010A0E38E
:1057D00024009FE5001080E53F5FBDE804F05EE235
:1057E00040C11FE04CC11FE0A41D0040084000E084
:1057F00006050040184000E0FC04004030F0FFFFC8
:105800003F5F2DE90000A0E30010A0E10830A0E315
:10581000E0209FE50030C2E5DC209FE50020D2E5D6
:10582000080012E30900000ACC209FE50030D2E511
:10583000F73003E20030C2E5C0209FE50020D2E54A
:10584000010052E30A00001A0110A0E3080000EA78
:10585000A4209FE50030D2E5083083E30030C2E5A4
:1058600098209FE50020D2E5000052E30000001AD6
:105870000110A0E388209FE5003092E584209FE599
:105880000050D2E5000055E30900000A78209FE5AA
:10589000004092E574209FE5940505E00340A0E1F7
:1058A000054084E0005092E5054044E00700C2E571
:1058B000030000EA54009FE5000090E50340A0E1EA
:1058C000004044E00320A0E140009FE5002080E587
:1058D0000100A0E1001CA0E1211CA0E10400A0E166
:1058E00090FAFFEB0010A0E324009FE5001080E594
:1058F0003F5FBDE804F05EE240C11FE04CC11FE025
:10590000A51D0040084000E007050040184000E0E9
:105910000005004030F0FFFF064A074801681143C8
:105920000160064A06480168114301600F210548DD
:105930000170704700C0000000C002E001000020BC
:1059400004C002E048C11FE0024A03480168114355
:105950000160704700080000088002E000B50B4AB3
:105960000B480168114301600A4A0B480168114362
:1059700001600A480021FFF78BFB09480021FFF76F
:1059800087FB04480021FFF7A1FB00BD00300000A9
:10599000088002E000004000188002E000100000D3
:1059A0000020000000B5094A094801681143016060
:1059B000084809490A6802430A600021FFF786FB8C
:1059C00002480021FFF764FB00BDC0460000400014
:1059D000088002E000000800188002E000B50948D5
:1059E00009490A6802430A60084B09490A681A43D0
:1059F0000A600021FFF74CFB04480021FFF766FB1B
:105A000000BDC04600002000088002E00000000841
:105A1000188002E000B50B4A0B4801681143016091
:105A20000A480B490A6802430A600021FFF74EFB4F
:105A300008480021FFF72CFB07480021FFF728FB4F
:105A400000BDC0460000000C088002E0000002001B
:105A5000188002E0000000080000000400B5044ABD
:105A600004480168114301600120FFF76BFC00BD91
:105A700000000084188002E009490A4801600321FF
:105A8000094801600121094801600949094801608C
:105A90002421094801601021084801607047C04670
:105AA00065560000184000E0144000E0044000E0AB
:105AB000E45A000010F1FFFF10F2FFFF10F0FFFFAB
:105AC000011C00290ADD011C0904090C044801809D
:105AD00003480088000400140028F9D17047C0462C
:105AE0000C0500401F5F2DE90110A0E328019FE590
:105AF000001080E51040A0E320019FE5004080E514
:105B00001C019FE50010E0E3011080E00020D1E5DA
:105B1000012082E20020C1E50010D0E5011081E201
:105B20000010C0E5011080E20020D1E5012082E2F2
:105B30000020C1E5B610D0E10118A0E14118A0E1B4
:105B40000100A0E1000050E3020000DAD4009FE56C
:105B5000011041E2B010C0E1C80200EBC8009FE5AF
:105B60000010D0E5011081E20010C0E5B8009FE50B
:105B70000000D0E50A0050E3060000DA0100A0E3CF
:105B8000A8109FE50B00C1E50C00C1E50000A0E3F3
:105B90000D00C1E52F0200EB94009FE5B010D0E1AD
:105BA000000051E30200000A84009FE5011041E279
:105BB000B010C0E17C009FE50010D0E5011081E24B
:105BC0000010C0E56C009FE50000D0E5640050E3E4
:105BD000090000BA0010A0E348009FE50710C0E5E7
:105BE0000310E0E3010080E0001090E5011081E285
:105BF000001080E5660100EBF21E00EBB20B00EB3B
:105C000034009FE5004080E50010A0E32C009FE5F4
:105C1000001080E51F5FBDE804F05EE2004000E098
:105C200014F0FFFF060500400C050040120500407F
:105C3000050500400E0500401305004010F0FFFF71
:105C400030F0FFFFF0B50F1C061C81B001250020CD
:105C5000FFF760FB0020FFF755FB022000F0A6F8DD
:105C6000832000F0ADF8022000F0A0F8002400A886
:105C700000F0C6F805062D0E381C0106090E201C82
:105C8000884208DA00A80178221C301C81540134B3
:105C9000281C0028EBD10120FFF734FB022000F084
:105CA00085F8201C01B0F0BDF0B50F1C061C81B0BA
:105CB00001250020FFF72EFB0020FFF71DFB02202F
:105CC00000F074F8812000F07BF8022000F06EF8FC
:105CD000002400A800F0C6F805062D0E381C0106A9
:105CE000090E201C884208DA00A80178221C301C0A
:105CF00081540134281C0028EBD10120FFF7FCFA65
:105D0000022000F053F8201C01B0F0BD70B50E1C4D
:105D1000051C0020FFF7FEFA0020FFF7EDFA022035
:105D200000F044F8802000F04BF8022000F03EF82C
:105D3000002408E0211C281C405C00F041F80220EF
:105D400000F034F80134311C201C8842F2D30120C9
:105D5000FFF7D2FA022000F029F870BD70B50E1CD2
:105D6000051C0020FFF7D6FA0020FFF7CBFA02202F
:105D700000F01CF8822000F023F8022000F016F852
:105D8000002408E0211C281C405C00F019F80220C7
:105D900000F00CF80134311C201C8842F2D30120A1
:105DA000FFF7B0FA022000F001F870BD642101395C
:105DB0000A1C002AFBDC011C01380029F6D17047BF
:105DC00030B5051C0020FFF7A5FA002412E0281CBE
:105DD0000006000E80210840FFF7A4FA0120FFF71B
:105DE00099FA6D002D062D0E0020FFF793FA01346D
:105DF0002406240E201C0006000E0828E7DB30BD18
:105E000070B5061C01240025301C057021E001201E
:105E1000FFF780FA281C0006000E062804D1FFF7C1
:105E200057FA002800D00024301C01784900301CAB
:105E30000170FFF75BFA002805D0301C01780120C3
:105E40000143301C01700020FFF764FA01352D0674
:105E50002D0E281C0006000E0828D8DB201C00068A
:105E6000000E70BD70B5061C01240025301C0570A5
:105E700021E00120FFF74EFA281C0006000E06283C
:105E800004D1FFF72BFA002800D00024301C017841
:105E90004900301C0170FFF729FA002805D0301C9A
:105EA000017801200143301C01700020FFF732FA15
:105EB00001352D062D0E281C0006000E0828D8DB03
:105EC000201C0006000E70BD10B50C1C011C081C27
:105ED00002280BD0032812D0012817D10B2000F084
:105EE00045F8201C142100F02BF80FE0072000F0EB
:105EF0003DF8201C1430142100F022F806E00B209D
:105F000000F034F8201C282100F01AF810BDC0461B
:105F100010B5041C201C0006000E04280CDA1F20FB
:105F200000F024F8582000F021F8201C0106090E8A
:105F30000248405C00F01AF810BDC0469002000014
:105F400030B50D1C041C084893B06946132304C8DF
:105F500004C15B1EFBD1281C00040014211CFEF7A9
:105F60002BFD13B030BDC0464402000001B5074808
:105F700093B06946132304C804C15B1EFBD113A967
:105F80000120FEF719FD13B001B000BD440200006E
:105F900030B50D1C041C084893B06946132304C88F
:105FA00004C15B1EFBD1281C0106090E201CFEF754
:105FB000C1FD13B030BDC0469402000010B5041CF2
:105FC000084893B06946132304C804C15B1EFBD183
:105FD000201CFEF73BFD13B00006000E0006000E6D
:105FE00010BDC046940200000EB470B5021CA0B0F3
:105FF00024AB00A8111C1A1C0DF09AFD00AE301C39
:106000000EF0C8FE041C002504E0281C305CFEF7DE
:1060100087F80135211C281C8842F6DB201C20B0A3
:1060200070BC08BC03B01847021C0349101C8180D7
:10603000101CC1807047C046FFFF000000B5021C65
:10604000101C008900040014011C101C808800042E
:1060500000140EF0D9FF011C101CC08800040014AD
:10606000814201D1022000E0002000BD00B5021CE9
:10607000101CC088000400140130111C0989090497
:1060800009140EF0C1FF011C101C808800040014CC
:10609000814201D1012000E0002000BD00C09FE549
:1060A0001CFF2FE1A960000010B50C1C031C181C7C
:1060B000FFF7DCFF00281AD1181CC0880004001468
:1060C0000130191C0989090409140EF09DFF011CF7
:1060D0000904090C181CC180211C181CC08800046C
:1060E0000014021C181C00688154002000E00120EC
:1060F00010BC08BC1847C04610B50B1C041C201C63
:10610000FFF79CFF00281BD1201C8088000400148E
:106110000130211C0989090409140EF075FF011CC6
:106120000904090C201C8180201C808800040014B4
:10613000011C201C0068425C181C0270002000E05A
:10614000012010BD10B5041C201CFFF777FF0228AA
:1061500001D100201DE0201CFFF788FF002804D09B
:10616000201C00890004001413E0201CC0880004D7
:106170000014011C201C808800040014021C8A42A8
:1061800006DD531A201C008900040014C01A00E028
:10619000881A10BD00C09FE51CFF2FE1A16100001F
:1061A0001548018800290FD0134801390180124891
:1061B0000088002808D1012110480170104800789B
:1061C000012801D10F4801700F4801880904091402
:1061D00000290FD00C48013901800B4800880004C9
:1061E0000014002806D106480078012802D10121B8
:1061F000064801707047C04614050040180500406D
:10620000D321004016050040D02100401705004072
:1062100000B502490320FFF757FE00BD19050040F5
:1062200010B5041C201C002808D00648008800284F
:1062300001D0FFF7EDFF002102480180211C024838
:10624000017010BD140500401805004008B4F0B5F9
:106250000D1C071C90B0002415AB00A8111C1A1CC3
:106260000DF066FC00AE301C0EF094FD031C381CD3
:106270000006000E191C4018282805D90124381CD6
:106280000006000E28231B1A381C0106090E0F48B1
:106290004018311C1A1C0EF061FD281C022803D086
:1062A000032801D0012809D109480078002805D029
:1062B000281C0006000E0549FFF706FE201C0006FC
:1062C000000E10B0F0BC08BC01B018471905004022
:1062D0001805004030B50C1C011C0025081C0128C5
:1062E00005D0022805D0002804D1012502E00225AE
:1062F00000E00325281C0006000E0121084204D0FE
:106300000D48202114220EF06DFD281C0006000E01
:106310000221084204D00948202114220EF062FD17
:1063200007480078002805D0201C0006000E02490E
:10633000FFF7CAFD30BDC046190500402D050040DD
:1063400018050040F0B5141C0D1C071C90B015AECC
:1063500000A8191C321C0DF0EBFB00AE301C0EF037
:1063600019FD031C381C0006000E191C40182828B3
:1063700001D901201CE0381C0106090E0E48401806
:10638000311C1A1C0EF0EAFC281C022803D003283A
:1063900001D0012805D1281C0006000E0649FFF790
:1063A00093FD201C0104090C002000F043F800209C
:1063B00010B0F0BC08BC18474205004030B50C1CBA
:1063C000011C0025081C012805D0022805D0002842
:1063D00004D1012502E0022500E00325281C000667
:1063E000000E0121084204D00B48202114220EF097
:1063F000F9FC281C0006000E0221084204D00748C0
:10640000202114220EF0EEFC201C0006000E024992
:10641000FFF75AFD30BDC04642050040560500401A
:10642000011C081C0106090E0148405C7047C0466B
:10643000190500400A1C011C0B1C05480370081CB0
:106440000006000E002802D1111C0248018070478E
:10645000180500401405004000C09FE51CFF2FE117
:106460006564000000B500F0D3F91C4800780028EE
:1064700008D00021194801704078021C0020012139
:1064800006F082FE16480078002810D001280BD1B3
:1064900014480078011C3F2001401348405C021C56
:1064A0000020012106F070FE00210D4801700F4808
:1064B0000078002810D001280BD10D480078011C6D
:1064C0003F2001400B48405C021C0220012106F0E5
:1064D0005BFE00210548017008BC18477D0500409F
:1064E000B4040040B5040040F8020000B7040040C6
:1064F000B80400403803000010B4021C00210EE074
:10650000081C03061B0EDB000A48C458101CA042DE
:1065100002D10948C05C0BE001310906090E081CD4
:1065200003061B0EDB000348C0580028E8D10020FA
:1065300010BC7047780300007C03000010B5041CF9
:10654000201C00281CD01E480078002803D1002100
:106550001C48017030E01B48017801310170194876
:106560000078152804D10122101C111C06F00CFE25
:1065700014480078FF281FD11521124801701BE034
:106580000F480078002803D000210E48017013E066
:106590000C480178013101700A480078152804D1AF
:1065A0000121081C022206F0EFFD06480078FF28B2
:1065B00002D1152103480170211C0148017010BD52
:1065C0007F0500408005004030B5041C81B0FEF717
:1065D000A9FC051C281C20210840FFF7AFFF281C40
:1065E00024490840FFF788FF031C00210A1C181CDF
:1065F00000281CD020480078051C181C0006000E3E
:10660000A84204D01C4841701D1C05701DE01B48A9
:1066100005780135057019480078072800D1012256
:10662000192812D10F221548027002220DE01248DB
:106630000078002807D0114D2D78072D01DB0322AB
:10664000031C0D4801700D480170191C00A8017051
:10665000111C01206844017000A9201C001C06D0F8
:1066600002220B780370491C401C521EF9D101B064
:1066700030BDC046DFFFFF008105004082050040BD
:1066800000C09FE51CFF2FE18D66000010B50024BF
:1066900045480168782903DA43480131016004E084
:1066A000782041490860002048604048FEF700FD1E
:1066B000002800D001243E48FEF7FAFC002801D053
:1066C00002200443201C0106090E3A480078884243
:1066D00066D0201C002859D002282CD0012859D17E
:1066E00035480078002858D000212F4801761B211A
:1066F00081810068782805D03048008800040014A3
:106700001B2807D0002028494860012048741B201E
:1067100088740CE02A48016801310160284800684B
:10672000052804DD0120204948741B2088740021BD
:106730001D48016031E02048007800282DD000215C
:10674000194801761A2181810068782805D01B48F4
:106750000088000400141A2807D00020124948605D
:10676000012048741A2088740CE015480168013132
:10677000016013480068052804DD01200A494874B7
:106780001A20887400210848016006E001210A48A7
:10679000017002E0002108480170211C05480170C9
:1067A00010BC08BC1847C0466C050040000008003B
:1067B0000000040083050040840500407A05004085
:1067C0007005004000B5011C081C0006000E622880
:1067D00006D0081C0206120E0020012106F0D4FC8F
:1067E00000BDC04600B5021C101C0006000E622849
:1067F0000BD1081C0004000C0A2806D1101C02064C
:10680000120E0020012106F0BFFC00BD7047C046FB
:1068100010B581B000AC201CFFF7D6FE0120684403
:10682000007802280AD0032812D0012818D10021AC
:106830000C4801602078FFF7C5FF11E009480168A6
:1068400001310160074801682078FFF7CBFF07E0BE
:10685000044801682078FFF7D9FF00210148016052
:1068600001B010BD7405004000B5011C0948007856
:1068700001280ED1081C0006000E312809D0064858
:106880000078002805D10120FFF742FB32210348A0
:10689000018000BDD2210040DF210040D021004016
:1068A00000B5024802490EF04DFB00BD8C050040CA
:1068B0000018000000B5FEF7CDFDFFF7F1FFFFF770
:1068C000DBF8FDF773FCFDF7F5FF1020FEF700F88D
:1068D0001120FDF7FDFF00BD284806C80B1C13431F
:1068E00005D000230B70491C9142FBD1F5E72448E9
:1068F000C01C0323984306C80B1C134306D003781F
:10690000401C0B70491C9142F9D1F1E700B583B0EE
:10691000FFF7D0FF04F0B2FB0120FDF791F906F07C
:10692000EFFDFEF7BDFD174800680EF041FB00AC1F
:10693000201C04F0EDFB0006000E012802D1201CF3
:1069400004F054FC0CF0A8FE0F480078002804D096
:1069500000210D480170FFF75BFC0C48007800280F
:1069600006D000210A4801700A480078FFF7D0FAE3
:1069700005F056F8D7E703B000BDC046702E000002
:10698000402F000088050040160500401705004014
:1069900017050040DF21004010B50C1C011C081C2D
:1069A00001280CD0022811D0032816D0002816D1B7
:1069B000201C0106090E082000F082FE0FE01820BE
:1069C000FFF7FCFA041C0006000E09E0201C01067B
:1069D000090E1820FFF7DCFA01E0002000E000209B
:1069E00010BC08BC1847C04610B50C1C011C081C84
:1069F00001280BD0022810D0032815D0002815D16B
:106A0000201C0006000E0AF09DFB0FE02120FFF77E
:106A1000D5FA041C0006000E09E0201C0106090E30
:106A20002120FFF7B5FA01E0002000E0002010BCB3
:106A300008BC184710B50C1C011C081C01280CD000
:106A4000022815D003281AD000281AD1201C0006CD
:106A5000000E022106F076FB13E00420FFF7AEFAE9
:106A6000041C211C09480170201C0006000E09E0CE
:106A7000201C0106090E0420FFF78AFA01E002201B
:106A800000E0002010BC08BC1847C046DF210040D1
:106A900010B50C1C011C081C002815D002280AD0B7
:106AA00003280FD001280FD10520FFF787FA041C17
:106AB0000006000E09E0201C0106090E0520FFF764
:106AC00067FA01E0012000E0002010BC08BC184774
:106AD00010B50C1C011C081C01282CD0022831D038
:106AE000032836D0002836D105F0C4FD002832D066
:106AF000201C0006000E0F21084009280DD1201C83
:106B00000006000EF0210840102803D1022005F0F5
:106B1000BBFD02E0012005F0B7FD201C0106090EB7
:106B20000F2001400906090E0D4801700C4800783D
:106B3000FCF7BEFE0FE00620FFF740FA041C00063B
:106B4000000E09E0201C0106090E0620FFF720FABE
:106B500001E0002000E0002010BC08BC1847C0463F
:106B6000DA21004010B50C1C011C081C012817D0AC
:106B7000022821D003281DD000281DD1201C020688
:106B8000120E52000E480F49895A09040914418116
:106B90004089000400140DF0B1FFFEF7F5F90BE099
:106BA000094800880004001400F030FE041C0006B0
:106BB000000E02E03C2000E0002010BC08BC18479A
:106BC000D22100406C160000DC21004010B50C1CE6
:106BD000011C081C01280BD0022810D0032815D056
:106BE000002815D1201C0006000EFEF7C7FB0FE0A1
:106BF0000720FFF7E3F9041C0006000E09E0201C43
:106C00000106090E0720FFF7C3F901E0002000E0AC
:106C1000002010BC08BC184710B50C1C011C081C37
:106C200001280BD0022810D0032815D0002815D138
:106C3000201C0006000EFEF7DDFB0FE00948FFF701
:106C4000BDF9041C0006000E09E0201C0106090E17
:106C50000448FFF79DF901E0002000E0002010BC8F
:106C600008BC18477501000010B50C1C011C081C5D
:106C700001280FD002281DD0032822D0002822D1BD
:106C8000201C002801D0012400E00024211C104811
:106C9000017018E00F48FFF791F9041C002801D09B
:106CA000012400E00024211C09480170201C00067A
:106CB000000E09E0201C0106090E0648FFF768F9DE
:106CC00001E0002000E0002010BC08BC1847C046CE
:106CD000A41D00407301000010B50C1C011C081C11
:106CE00001280FD002281DD0032822D0002822D14D
:106CF000201C002801D0012400E00024211C1048A1
:106D0000017018E00F48FFF759F9041C002801D062
:106D1000012400E00024211C09480170201C000609
:106D2000000E09E0201C0106090E0648FFF730F9A5
:106D300001E0002000E0002010BC08BC1847C0465D
:106D4000A51D00407401000010B50C1C011C081C9E
:106D5000012809D002280ED0032813D0002813D10F
:106D6000211C0B4801700FE00A48FFF727F9041CAB
:106D70000006000E09E0201C0106090E0548FFF779
:106D800007F901E0002000E0002010BC08BC184713
:106D9000A11D00403A01000030B50C1C011C081C6C
:106DA00001281CD0022820D003281CD000281CD188
:106DB0000020104D2870104A14200221FFF746FAD7
:106DC000012000F05DFF0D4A14200221FFF73EFA7A
:106DD0000B48FEF775FE01202870012006E0201CFC
:106DE0000006000E02E0002000E0002030BC08BCDD
:106DF0001847C0467C0500404D04000038040000E0
:106E0000F401000030B5151C0C1C011C081C0128E5
:106E10000ED002281AD0032827D0002827D1281CFA
:106E20000006000E211C0906090E04F0F9F81EE008
:106E3000281C0006000E10494018FFF7BFF8041C7C
:106E4000002801D0012013E0002011E0201C0028C0
:106E500000D00124281C0006000E07494018211C00
:106E60000906090EFFF794F801E0012000E0002078
:106E700030BC08BC1847C0461C01000030B5151CCA
:106E80000C1C011C081C01280ED0022816D0032857
:106E90001ED000281ED1281C0006000E211C090649
:106EA000090E00F00DFC15E0281C0006000E103045
:106EB000FFF784F8041C0006000E0CE0281C0006F6
:106EC000000E1030211C0906090EFFF761F801E0E1
:106ED000002000E0002030BC08BC184730B50C1C76
:106EE000011C081C01286FD0022874D0032879D017
:106EF000002879D1101C0006000E012810D13C4852
:106F00000078002807D000213948017004200022B1
:106F1000111C04F0A1F837480021FFF739F863E0AD
:106F2000201C012807D002280CD000285CD10021A9
:106F30002F48017058E03048FEF732F801212C4804
:106F4000017051E001212A48017000252B4805708D
:106F500022E0281C0106090E890029484058C06A11
:106F600001780022101C04F077F8264A1420002132
:106F7000FFF76CF9281C0106090E890020484058CB
:106F8000C06A42681E200221FFF760F91E48FEF722
:106F900097FD01352D062D0E281C0106090E8900CE
:106FA000174840580028D4D112480021FEF7F0FFBE
:106FB00004200022111C04F04FF801220C480F4954
:106FC0000A70002101700FE00A48FEF7F7FF041C69
:106FD0000006000E09E0201C0106090E0548FEF718
:106FE000D7FF01E0002000E0002030BC08BC1847BB
:106FF000A31D004038010000ECFFFFFF7C050040AE
:10700000981F0040620400008813000030B5151C72
:107010000C1C011C081C012811D0022819D00328BF
:1070200021D0002821D1201C0106090E8900114819
:107030004158281C0006000EFDF7DCFF15E0281C57
:107040000006000E1930FEF7B9FF041C0006000E02
:107050000CE0281C0006000E1930211C0906090E40
:10706000FEF796FF01E01E2000E0002030BC08BCC7
:107070001847C0460406000030B5151C0C1C011C46
:10708000081C012813D002281BD0032823D0002875
:1070900023D1281C0006000E211C0906090E03F04E
:1070A000B1FF281C0006000E0AF06EF815E0281C3F
:1070B0000006000E0830FEF781FF041C0006000EDB
:1070C0000CE0281C0006000E0830211C0906090EE1
:1070D000FEF75EFF01E0002000E0002030BC08BCAD
:1070E0001847C04610B50C1C011C081C01280BD009
:1070F000022817D003281CD000281CD1201C000611
:10710000000EFCF7BDF916E00D48FEF757FF041C12
:10711000211C0C480170201C002801D001200BE02C
:10712000002009E0201C0106090E0548FEF730FF8B
:1071300001E0002000E0002010BC08BC1847C04659
:1071400039010000A21D004070B50C1C011C101C70
:107150000606360E0F2006403606360E101C0506B3
:107160002D0EF02005402D092D062D0E081C01289E
:107170001DD002282CD003283BD000283BD1201C56
:107180000106090E89001E484058291C0906090EEF
:107190008900321C1206120E1C235A435218194938
:1071A0008850301C0006000E09F0EEFF23E0301C72
:1071B0000006000E0521484313494018291C090602
:1071C000090E4018FEF7FAFE041C0006000E13E03C
:1071D000301C0006000E052148430B494018291CAD
:1071E0000906090E4018211C0906090EFEF7D0FEFB
:1071F00001E01E2000E0002070BC08BC1847C0461B
:1072000004060000B42200403B01000070B5151CCC
:107210000C1C061C301C012811D0022826D0032883
:107220002FD000282FD1301C0006000E291C090683
:10723000090E221C1206120E00F00AFB23E0281C85
:107240000006000E12494018FEF7B8FE041C301C60
:107250000006000E291C0906090E221C1206120E39
:1072600000F0F6FA201C0006000E0DE0281C0006B7
:10727000000E07494018211C0906090EFEF788FE7A
:1072800001E0122000E0002070BC08BC1847C04696
:107290002601000070B5141C0D1C061C301C0128B2
:1072A0001BD0022830D0032839D0002840D1301C10
:1072B0000006000E211C0906090E2A1C1206120ED9
:1072C00000F0F2FA201C0006000E1B4909788142EA
:1072D0002ED1012006F02CF82AE0201C0006000E1A
:1072E00016494018FEF76AFE051C301C0006000E09
:1072F000211C0906090E2A1C1206120E00F0D4FAEF
:10730000281C0006000E14E0201C0006000E0B498D
:107310004018291C0906090EFEF73AFE08E0201C59
:107320000006000E002801D1002002E0012000E04C
:10733000002070BC08BC1847D62100402E01000078
:1073400030B5141C0B1C011C081C012829D0022874
:1073500017D0032835D000283ED1201C0106090E85
:1073600089001F4D1F48405829781A1C13061B0E10
:107370000C2200F0D1FA28702878011C0C20401A49
:107380002BE0201C0006000E0C2148432330211C5A
:107390000A06120E920013498A580C2100F026F8B2
:1073A0001AE0201C0006000E0C2148432330211C4B
:1073B0000A06120E92000B498A580C2100F086FA38
:1073C0000AE0201C0206120E920006488058064968
:1073D00089580C220DF0EEFC002030BC08BC184788
:1073E000B21D0040E01F0040BC1F0040F0B5171C5C
:1073F0000E1C051C002415E0201C0106090E381C7B
:10740000415C081C202815DB7F2813DC201C0206A9
:10741000120E281C0006000E8018FEF7B9FD01347C
:107420002406240E301C0106090E201C0006000E46
:107430008842E1D30CE0201C0106090E281C00063E
:10744000000E40182021FEF7A3FD01342406240E6F
:10745000301C0106090E201C0006000E8842EAD3EB
:10746000F0BDC04610B50A1C011C081C01281BD029
:10747000022813D003281DD0002820D1124C2078D8
:10748000011C101C03061B0E1048122200F044FAC7
:1074900020702078011C1220401A11E00B4A8F2026
:1074A0001221FFF7A3FF0AE0084A8F20122100F003
:1074B0000DFA04E00548064912220DF07BFC00207D
:1074C00010BC08BC1847C046B31D004071220040E4
:1074D0007704000010B50C1C011C081C002809D002
:1074E000022824D0032829D0012829D11648FEF7E4
:1074F00065FD041C201C0006000E002808D113485E
:1075000013494860134888600860A120C87607E0E6
:1075100011480F494860114888600860BF20C8764C
:1075200001210F480170201C0006000E09E0201CFC
:107530000106090E0448FEF72BFD01E0002000E0E3
:10754000002010BC08BC184724010000E0A5010081
:10755000681F0040CC55010078630100E02801005D
:10756000A61D004010B50C1C011C081C002809D0E9
:1075700002282ED0032833D0012833D11B48FEF730
:107580001DFD041C201C0006000E00280DD118490A
:1075900018484160184981600160FB22011C2831B4
:1075A0000A700A21263001700CE01449114841602C
:1075B000134981600160DD22011C28310A70092114
:1075C0002630017001210F480170201C0006000EBA
:1075D00009E0201C0106090E0448FEF7D9FC01E071
:1075E000002000E0002010BC08BC18472501000066
:1075F000A40600005C1F00401202000042060000CA
:1076000013020000A61D004010B50C1C011C081C34
:10761000012810D002281FD0032824D0002824D10C
:10762000201C002803D00121124801701DE0002118
:107630001048017019E01048FEF7C0FC041C002837
:1076400003D001210B48017002E0002109480170BC
:10765000201C0006000E09E0201C0106090E064849
:10766000FEF796FC01E0002000E0002010BC08BC02
:107670001847C0468C1D00401901000010B50C1CB5
:10768000011C081C002815D002280AD003280FD09E
:1076900001280FD10948FEF791FC041C0006000EDA
:1076A00009E0201C0106090E0448FEF771FC01E008
:1076B000002000E0002010BC08BC184719010000A1
:1076C000F0B50B1C051C0026321C281C01280FD00D
:1076D00002280DD003280BD0042809D0052807D094
:1076E000062805D0072803D008283AD000283CD126
:1076F000191C281C07063F0E3348C155181C0106EB
:10770000090E32480078884207D2191C2F480170B0
:10771000291C2F480170012227E0281C0106090EB0
:107720002B480078884220D128480670002411E0B8
:10773000201C0106090E2448415C081C234E3678A3
:10774000B04204D921480170211C21480170013444
:107750002406240E201C0006000E0728E8DD012266
:1077600003E0191C1B4801700122101C00281AD0CC
:10777000002412E0201C0106090E1348405C134946
:107780000978091A134800780918201C0006000E11
:1077900003F02CFC01342406240E201C0006000EED
:1077A0000728E7DD0FE0281C0106090E0648405CAB
:1077B00006490978091A074800780918281C0006A4
:1077C000000E03F013FCF0BDA71D0040B01D0040EB
:1077D000AF1D0040B11D004000B5021C0A480078F2
:1077E00001280FD1081C002807D0101C0106090E23
:1077F0000022101C03F030FC04E004200022111CC5
:1078000003F02AFC00BDC046A31D0040021C00215D
:1078100014E0081C03061B0E5B000C48C05A000451
:107820000014031C101C00040014984203D1081C0F
:107830000006000E08E001310906090E081C0006CA
:10784000000E6A28E5DB3C207047C0466C1600003D
:1078500030B5031C081C0006000E09281DDC101C96
:107860000C1C25062D0E0D4C6055081C0106090E3A
:107870000B480078884210D1181C0006000E002822
:107880000BD1101C0106090E49000648405A00049D
:1078900000140DF033F9FDF77DFB30BD8D1D004068
:1078A000D62100404017000010B4141C0B1C181CFB
:1078B0000006000E092805DC201C191C0A06120E01
:1078C0000149885410BC7047971D0040F0B5141C46
:1078D0000F1C061C002510E0281C0106090E301C98
:1078E0000006000E4018FEF769FB291C0B061B0E54
:1078F000211CC85401352D062D0E381C0106090E19
:10790000281C0006000E8842E6D30020291C0B0626
:107910001B0E211CC854F0BD30B4041C181C5E287A
:1079200016D05F2823D0602828D0612833D05D2866
:1079300032D1081C03061B0E201CC05C031C7F2BCD
:107940002ADA0B1C1D062D0E231C0130585523E08E
:10795000081C03061B0E201CC05C031C202B1BDD17
:107960000B1C1D062D0E231C0138585514E0081C55
:10797000002811D001390906090E0DE0101C03067C
:107980001B0E013B081C0006000E984204DA013170
:107990000906090E00E000210023101C0206120E49
:1079A000201C8354081C0006000E30BC7047C046E3
:1079B00000B500F0F7FC03F013FC0006000E0021F8
:1079C00005F018FC002008BC1847C04610B5141C70
:1079D000081C0006000E00F01DF80D4908600C4858
:1079E0000368002B01D101200EE0201C084A90758D
:1079F000907D041C14214C43996809195160011CA5
:107A0000181C00F077FC002010BC08BC1847C046CA
:107A1000B41D004010B4021C002112E0081C030633
:107A20001B0E0C2043430B48C05C041C101C0006BA
:107A3000000E844202D10848C01808E0013109064E
:107A4000090E081C0006000E1128E7DB002010BC00
:107A50007047C0463C0500003805000010B500F036
:107A6000D1F90C4CA08603F0BBFB211C3831087007
:107A7000032003F0A5FB2078012808D10120064946
:107A8000C87103204872054800F070FC01E000F066
:107A900043FC10BD8C1D0040C01D0040FC040000D4
:107AA00010B5041C201C0006000E00F037FF041C5B
:107AB000042846D00A281DD00B281FD00C2829D016
:107AC0000D2833D01A2825D01B2817D01D2838D0D0
:107AD00030282FD0342809D035280BD036280DD0A7
:107AE000372817D0382821D0092830D100F0ACFC35
:107AF00000202DE000F020FD002029E0154800685E
:107B00000079002802D100F09FFC01E000F094FD14
:107B100000201DE00F4800680079002802D100F025
:107B20000BFD01E000F0F4FD002011E000F080FE0C
:107B300000200DE00022101C111CFFF739FF00206F
:107B400006E000F02FFC201C0006000E00E00020E4
:107B500010BDC046B41D0040F0B5061C00257BE0FA
:107B6000281C0106090E0C2041434148405C0028B6
:107B70006FD1002760E0381C0106090E1420414334
:107B8000281C0206120E0C2042433A488058401826
:107B90000179042928D0052926D0072924D00829CD
:107BA00022D0092920D0022943D100F05BF9041C1E
:107BB000301C00283DD0201C0206120ED200381CBA
:107BC0000106090E14204143281C03061B0E0C203D
:107BD00043432848C058401881688C5C211C090622
:107BE000090E00F077F924E0381C0106090E142074
:107BF0004143281C0206120E0C2042431D488058A7
:107C0000401800F02FF9041C301C002811D0381C3B
:107C10000106090E14204143281C0206120E0C20F6
:107C20004243144880584018211C0906090E00F0F0
:107C300051F901373F063F0E281C0106090E0C20A2
:107C400041430D48405C011C381C0006000E884270
:107C500091D301352D062D0E281C0006000E11288B
:107C600000DA7DE72220FEF7A9F904490870F0BD8B
:107C70003D050000400500003E050000D621004003
:107C8000F0B5041C002561E0281C0106090E0C203B
:107C900041433E48405C002855D1002646E0301C58
:107CA0000106090E14204143281C0206120E0C2066
:107CB00042433748805840180179042909D00529E2
:107CC00007D0072905D0082903D0092901D00229A6
:107CD00029D100F011F9071C301C0106090E1420EF
:107CE0004143281C0206120E0C20424328488058AB
:107CF0004018391C0906090E00F0DCF8201C002889
:107D000011D0301C0106090E14204143281C020624
:107D1000120E0C2042431E4880584018391C090698
:107D2000090E00F0D7F801363606360E281C01067B
:107D3000090E0C2041431748405C011C301C000612
:107D4000000E8842ABD301352D062D0E281C0006EF
:107D5000000E112898DB002000F06CF803F02EFED6
:107D60000D480188090409140C48018000210C48C1
:107D70000170201C002808D0084800880004001466
:107D8000021C0120022105F055FAF0BD3D0500005E
:107D9000400500003E050000E4160000D42100402C
:107DA000D621004030B5041C201C00780A281AD0C7
:107DB000012822D1201C4578281C0006000EFEF761
:107DC00053FD281C0006000EFFF76AFE051C000686
:107DD000000E002805D0201C05F090F80006000ECB
:107DE0000CE001200AE0201C4078211C8978221C2C
:107DF000D27800F0A1FE012000E0002030BC08BCD9
:107E00001847C04610B50948FEF7D8F80406240EF6
:107E100024022404240C0648FEF7D0F80006000EC5
:107E20000443201C0004000C10BDC0461B010000D0
:107E30001A01000010B5041C201C0104090CFF20CD
:107E400001400648FEF7A4F8201C0104090C090AA9
:107E5000FF2001400248FEF79BF810BD1A01000008
:107E60001B01000030B5051C281C0369002B1FD026
:107E7000281C007B021C012000210DF09CF8040648
:107E8000240E281C4079011C201C0006000E88428C
:107E90000AD3281C007B021C032000212B1C1B6919
:107EA0000DF089F80406240E201C0006000E00E0E8
:107EB000002030BD10B5041C201C0369002B08D025
:107EC000201C007B021C081C0106090E02200DF07C
:107ED00072F810BD10B5041C201C0369002B09D0DA
:107EE000201C007B021C081C0106090E00200DF05E
:107EF00062F800E0002010BD10B5041C201C0369CE
:107F0000002B07D0201C007B021C032000210DF059
:107F100052F800E0002010BD30B5051C281C036994
:107F2000002B09D0281C007B021C042000210DF02E
:107F300042F80406240E00E00024201C0006000E77
:107F400030BDC04610B5011C081C0079012812D0B4
:107F500004280BD0052809D0062807D0072805D00B
:107F6000082803D0092801D0022806D1081CFFF7F1
:107F700079FF041C02E0002400E0FF24201C00061E
:107F8000000E10BD10B50C1C101C002805D0221CC2
:107F900014200321FEF75AF904E0221C14200021CA
:107FA000FEF754F910BDC04600B5011C081C02685C
:107FB000002A03D00021081CFEF748F900BDC04686
:107FC0000EB410B5021C85B007AB00A8111C1A1C1A
:107FD0000BF0AEFD00AC201C0CF0DCFE0106090E1F
:107FE000081C0106090E2820401A054A231C0321FB
:107FF000FEF72CF905B010BC08BC03B01847C0460A
:1080000035050000F0B50F1C061C83B0301C40790C
:10801000002800D05AE10021AD4801704EE1381C23
:108020000206120EAA480078011C914200D041E1DC
:10803000011C14224A43301C8068801800790228F1
:1080400020D0032814D0042869D0052841D0062860
:108050007ED0072800D1A0E0082800D1C2E009287E
:1080600000D1EEE00A2800D117E1012800D02DE16F
:1080700014204143301C8068415800200122FFF742
:1080800081FF23E192480078011C14204143301CF9
:10809000806841580022101CFFF774FF8C4800785C
:1080A000011C14204143301C80684018417900298C
:1080B00000DC0BE1051CFFF7D5FE041C0106090ED0
:1080C000C900281C8068401841688248FFF778FF83
:1080D000FCE07F480078011C14204143301C80687C
:1080E00041580022101CFFF74DFF79480078011C11
:1080F00014204143301C85686D18281CFFF7B2FE20
:10810000041C0BF051FF02907349029B181C0BF0EA
:1081100083FE021C7148191CFFF752FFD6E06C4821
:108120000078011C14204143301C80684158002213
:10813000101CFFF727FF66480078011C14204143FC
:10814000301C8068401881686548FFF739FFBDE042
:108150005F480078011C14204143301C806841585E
:1081600000200122FFF70EFF59480078011C14205F
:108170004143301C806840184179002900DCA5E0AB
:10818000051CFFF7C9FE041C0006000E002800D0E5
:108190009CE0281CFFF766FE98E04D480078011C23
:1081A00014204143301C806841580022101CFFF706
:1081B000E9FE47480078011C14204143301C8568C3
:1081C0006D18281CFFF74EFE041C002806D0201C4A
:1081D0000106090E4348FFF7F3FE77E04248FFF738
:1081E000EFFE73E03A480078011C14204143301C34
:1081F000806841580022101CFFF7C4FE3448007804
:10820000011C14204143301C85686D18281CFFF7A1
:1082100029FE041C2E480078011C14204143301C08
:108220008068401880680090201C0106090E4900F3
:108230000098405A00040014011C2C48FFF7C0FEAF
:1082400044E023480078011C14204143301C80681E
:1082500041580022101CFFF795FE1D480078011CB4
:1082600014204143301C85686D18281CFFF7FAFD67
:10827000041C17480078011C14204143301C8068FE
:10828000401880680190201C0106090E89000198A1
:1082900041581748FFF794FE18E00D480078011C7C
:1082A00014204143301C8068415800200122FFF710
:1082B00069FE0BE00648017801310170301C8079BD
:1082C000011C03480078884200D2A8E603B0F0BD44
:1082D000CD1D004035050000333353402605000016
:1082E000220500001C050000191B000016050000F7
:1082F0000E05000030B50D1C041C02200021FDF706
:10830000E9FF201CFFF750FE281C0106090E201C67
:10831000FFF778FE30BDC04610B50020114CE07468
:108320000020FFF777FB20602268002A01D100209F
:1083300016E00C4C906860600020A0750021101CB5
:10834000FFF7D8FF207C042805D03220FCF7C0FAC4
:108350002A20FCF7BDFA00210348C17701700120F3
:1083600010BDC046B41D0040A61D004030B5051C20
:1083700000200A4C20730020208002200021FDF7FD
:10838000A9FF2A1C0021081CFDF760FF207B143088
:10839000034A0321FDF75AFF30BDC046BC1D004013
:1083A0000C05000010B50021081C0122FEF796FD07
:1083B000134C1448008800040014FCF7F1FD2078E9
:1083C00002F0FEFE2078042805D03220FCF7A0FA47
:1083D0002A20FCF79DFA2120FCF79AFA2320FCF7CB
:1083E00097FA0021064841700078042807D1064812
:1083F0000078002803D00548007803F08FFA10BDFC
:10840000C41D0040D4210040A61D0040851F00402F
:1084100010B50A480068007906280ED1084804689B
:1084200020690849884204D1207B0121FFF7D4F953
:1084300003E0207B0021FFF7CFF910BDB41D004001
:10844000B81D00400D70000010B53548047835485F
:108450000078002812D0344800680179042955D1E9
:108460005D21FFF737FD3149087030480078282139
:10847000091A00205F2204F013FF47E02848017822
:10848000002903D026480139017008E02848006817
:108490008079011C01390906090E21480170204824
:1084A0000078021C211C0906090E91421ED0011CF5
:1084B000142041431E48026890684018017906293B
:1084C00005D1FFF729FD0006000E00280ED0144844
:1084D0000078011C14204143154802689068401838
:1084E00001790029CAD000790628C7D00C48007845
:1084F000142148430E490968896809180A4801602F
:1085000009480068FFF71EFD0A490870FFF780FF61
:1085100003480078011C06480068FFF7EBFE10BD19
:10852000CA1D0040C51D0040B81D0040C61D0040CA
:10853000B41D0040CB1D004010B5394804783948BF
:108540000078002812D038480068017904295DD1EC
:108550005E21FFF7BFFC35490870344800782821B8
:10856000091A00205F2204F09BFE4FE02C4801789E
:10857000013101702E4802689079011C284800786A
:10858000884202D300212648017025480078031C48
:10859000211C0906090E994228D0011C14204143D0
:1085A000906840180179062911D1007906280ED16A
:1085B0001B480078011C142041431D480068806856
:1085C0004018FFF7A9FC0006000E00280ED0144842
:1085D0000078011C14204143154802689068401837
:1085E00001790029C2D000790628BFD00C48007854
:1085F000142148430E490968896809180A4801602E
:1086000009480068FFF79EFC0A490870FFF700FF61
:1086100003480078011C06480068FFF76BFE10BD98
:10862000CA1D0040C51D0040B81D0040C61D0040C9
:10863000B41D0040CB1D004070B500242F480568D4
:10864000287904283ED0052824D0062807D00728FA
:1086500020D008281ED009281CD0022845D1274E3A
:10866000281CFFF7FFFBF074F17C002903D00124E4
:10867000234801390170214EF07C011C3068FFF75E
:1086800019FCF07C021CD20030688168895CFFF71D
:1086900021FC2AE0194E281CFFF7E4FBF074F17C62
:1086A000002903D00124164801390170134EF07CD3
:1086B000011C3068FFF7FEFBF07C011C3068FFF7FF
:1086C00009FC12E00F48007800280ED0281C5F211A
:1086D000FFF700FC0C4908700B4800782821091AA4
:1086E00000205F2204F0DCFD0124201C002804D0BF
:1086F0000648817D0068FFF7FDFD70BDB81D004094
:10870000CB1D0040C51D0040C61D0040B41D0040EB
:1087100010B5002440480068017904295CD005297F
:1087200032D0062907D007292ED008292CD00929B4
:108730002AD0022964D1FFF795FB384908703648E2
:1087400003685879011C013934480278101C8842AA
:1087500004DA012431480132027003E00906090EEF
:108760002E4801702D480078011C2B480068FFF747
:10877000A1FB2A480078021CD200274800688168C3
:10878000895CFFF7A7FB3BE023480068FFF76AFB23
:1087900022490870204803685879011C01391F4894
:1087A0000278101C884204DA01241C48013202704D
:1087B00003E00906090E1948017018480078011CE9
:1087C00015480068FFF776FB14480078011C124832
:1087D0000068FFF77FFB13E01148007800280FD0F6
:1087E0000D4800686021FFF775FB0E4908700D48C1
:1087F00000782821091A00205F2204F051FD01248D
:10880000201C002806D008480078011C0748006892
:10881000FFF770FD10BDC046B81D0040CB1D0040E5
:10882000C51D0040C61D0040CA1D0040B41D0040CB
:10883000F0B500252C1C33480768387903281BD075
:1088400004281FD00A2845D0012852D12E4800689C
:108850000079062803D0B8680078062804D10021E2
:10886000081C0122FEF73AFB264800688168097857
:10887000FFF730FB041C3CE0381C0021FFF72AFB0B
:10888000041C36E02148007800280DD020480570EF
:10889000381C0021FFF70EFB01242120FCF738F8DB
:1088A0002320FCF735F824E00120164E7073381CA5
:1088B0006121FFF70FFBB073B07B2821091A00205C
:1088C0005F2204F0EDFC2120FCF702F82320FBF7E7
:1088D000FFFF0EE00F480078002803D00D48057018
:1088E000012406E001210748C17345740A48FFF7D7
:1088F0003DFD201C002804D00348817D0068FFF75F
:10890000F9FCF0BDB81D0040B41D0040C51D00407D
:10891000C51D0040C71D0040E804000010B5011C43
:108920005B480078002803D1081C0006000EAEE06A
:10893000081C0D2800D1A4E0252815D0262813D026
:10894000272811D028280FD029280DD02A280BD06D
:108950002B2809D02C2807D02D2805D0302800D16D
:108960008FE0242800D091E04A4C2088000120802C
:10897000081C0106090E24390904090C2088084343
:108980002080207B1430444A0221FDF75FFC201C2C
:108990000C30017801310170207B042876D13F48EA
:1089A0000078012828D002282FD003284FD0002893
:1089B0006CD1384800883A49884203D0394909883F
:1089C000884206D13848FFF7D1FC012137480170B1
:1089D0005CE0374C374A14200221FDF737FC36485B
:1089E000FDF76EF8002020810020E074A07D011CBE
:1089F0002068FFF77FFC49E0022026494873088879
:108A000048802E48FFF7B2FC40E0224801884088A9
:108A100088420AD11F4C2A4A14200221FDF716FC75
:108A20002088A080FFF706FA04E0264A14200221DD
:108A3000FDF70CFC2048FDF743F800211C4801819C
:108A40000021C174817D0068FFF754FC1EE01148CD
:108A500000881349884203D012490988884202D10C
:108A6000FFF75AFC12E0134A14200221FDF7EEFB37
:108A70001548FDF725F80022101C111CFEF798FF81
:108A800004E00022101C111CFEF792FF002010BD14
:108A9000C71D0040BC1D0040E6040000C91D004089
:108AA00000110000C01D0040D2040000C91D00409C
:108AB000B41D0040C2040000E8030000B004000040
:108AC000A20400008F040000F401000000C09FE534
:108AD0001CFF2FE1D98A000000B513480078002858
:108AE0001FD01248018809040914081C002818DD49
:108AF0000E48013901800D48008800040014002848
:108B00000FD101200022111C04F0CAFB0848007894
:108B1000002803D007490548018002E0C821034826
:108B2000018008BC1847C046C51D0040C21D00405A
:108B3000CC1D00409001000010B5031C1B480078BC
:108B4000002832D0181C012816D000282DD1184832
:108B5000184CE08100202076081C2077101CE0765D
:108B6000A07D011C2068FFF7C5FB207FFDF758FCA6
:108B7000A0760F48E08118E00F48007800280AD05E
:108B800000200A49C871C87A497A0B1C0B4A022195
:108B9000FDF75CFB09E001200449C871C87A897AB5
:108BA0000B1C064A0221FDF751FB10BDC51D0040FC
:108BB00090010000B41D0040CC1D00408C0400005A
:108BC00010B581B02A480068FDF738FA00284AD16C
:108BD0002748006800A9FDF78FFA00A80078FBF786
:108BE0009FFA00A80178402902D1002221490A7089
:108BF0002049097801290AD0002934D10178402977
:108C000031D101211B4A1170002151702BE00178F4
:108C1000202910DB01787F290DDC01781548031C21
:108C200001331A78141C01341C70131C124AD154DD
:108C30004078142817DB00A800780D280DD10F48C4
:108C40000078011C0C4802F091F90006000E012882
:108C500003D100210748017005E0064C0848FDF7E4
:108C6000C3F90020207001B010BC08BC1847C046F2
:108C7000D41D0040311F00401C1F0040321F004027
:108C8000801F000010B5021C074C101C211C0CF0AA
:108C900079F907D3054C101C211C0CF073F901D88D
:108CA000012000E0002010BD000070C100007041F4
:108CB000F0B50B1C061C002400252A1C301C017872
:108CC0002D2902D10122013609E02B2901D10136DB
:108CD00005E0302901DB392901DD00204BE03BE0D4
:108CE000301C0778302F27DB392F25DC281C0006A5
:108CF000000E012804D0281C0006000E002819D1FF
:108D0000201C1D490AF0D4FF041C381C30380BF01D
:108D1000F5FE011C201C0AF021FF041C281C000683
:108D2000000E012817D1201C13490BF075F8041C04
:108D3000022510E000201EE0301C00782E2808D10B
:108D4000281C0006000E002801D1012503E00020A8
:108D500011E000200FE00136301C00780028BFD160
:108D6000101C002803D0201C0CF0FEF8041C221C50
:108D7000181C02600120F0BD00002041031C0022ED
:108D80000CE0181C0078202806DB7F2804DC013268
:108D90001206120E013301E000200EE0181C0078CC
:108DA0000028EED1081C0106090E101C0006000E5A
:108DB000884201D9002000E001207047081C00060D
:108DC000000E032801D1012000E000207047C046BA
:108DD00000B502F005FA0006000E042807D1164877
:108DE0000078012801D1092024E00A2022E013485C
:108DF0000078012811D002280FD003280DD00428B4
:108E00000BD0052809D0062807D0072805D0082848
:108E100005D0092805D000280BD101300AE0002038
:108E200008E005480078012801D1092002E00A2065
:108E300000E0002000BDC046851F0040D621004054
:108E400070B50D1C041C281C0006000E042848D117
:108E5000201CC678312E1AD0322E18D0332E16D0C0
:108E6000342E14D0352E12D0362E10D0372E0ED0F0
:108E7000382E0CD0392E18D03F2E1AD0532E20D099
:108E8000302E2AD10120082104F052FA27E002F006
:108E9000A7F90006000E042801D102F01FFE311CC4
:108EA0003139012004F044FA19E0012002F036FDC6
:108EB00015E0FFF78DFF0106090E1548FDF794F840
:108EC0000DE002F08DF90006000E012807D1012106
:108ED000081C402204F058F901E0002014E00120B1
:108EE00012E0281C0006000E05280CD1201CC078BA
:108EF000312808D1201C0079302804D1022002F04A
:108F00000DFD012000E0002070BC08BC1847C046E1
:108F10009521000000B5021C081C0006000E042864
:108F20001FD1101CC078312803D03F2807D030282B
:108F300013D1011C3039012004F0DAF90FE004F0FC
:108F400011FB0006000E012803D10748FDF74CF87D
:108F500005E00648FDF748F801E0002002E00120A6
:108F600000E0002008BC18478E2100008721000087
:108F700000B5021C081C0006000E04280DD1101CB0
:108F8000C078312801D0302807D1021C303A0120A6
:108F9000022104F0EDF9012000E0002008BC184790
:108FA00001207047081C0006000E052801D1012091
:108FB00000E000207047C04600B5021C081C0006F7
:108FC000000E052813D1101C0079312806D0302856
:108FD00009D105200121FCF7DBFF06E00520002177
:108FE000FCF7D6FF01E0002002E0012000E00020B5
:108FF00008BC184700B50022081C0006000E042813
:1090000012D10B480078032806D10A4800780028BE
:1090100001D1012200E00222101C0106090E0648BF
:10902000FCF7E2FF012000E0002008BC1847C04622
:10903000E0210040E52100407F21000000B5021C36
:10904000081C0006000E04281FD1101CC07831280F
:1090500005D0322803D03F280CD0302811D1011C74
:1090600030390906090E0A4801700948007808F0ED
:1090700069F808E006480078011C0648FCF7B4FFD0
:1090800001E0002002E0012000E0002008BC1847B9
:10909000E52300407721000010B5041C00231A1CB2
:1090A000081C0006000E042826D1201CC0783F288A
:1090B00022D113480078082801D1042216E0114873
:1090C0000078022801D11A1C10E00F48007801280E
:1090D00007D0032807D0042807D0002806D106228D
:1090E00004E0032202E0012200E00222101C01063B
:1090F000090E0648FCF778FF012010BC08BC184791
:10910000D6210040E2210040E02100406F21000014
:1091100000B5021C081C0006000E052830D1101CEA
:109120000079312803D03F281DD0302828D1164897
:109130000078042815D115480078032811D0144868
:109140000078012803D001211148017002E00021BC
:109150000F48017001210F4801700D48007807F099
:1091600069FE01200DE00A480078012803D10A4871
:10917000FCF73AFF02E00948FCF736FF012000E067
:10918000002008BC1847C046E0210040E92100400B
:10919000EA2100409C240040672100005F2100007C
:1091A000002111480078002819D002280AD006288A
:1091B0000FD0012813D101210C48007800280ED0CF
:1091C00002210CE0032109480078002807D004217F
:1091D00005E0052105480078002800D00621081C7C
:1091E0000006000E7047C046E6210040E72100401F
:1091F00000B5021C081C0006000E052858D1101CE2
:109200000079312811D0322815D0332818D03428CD
:109210001CD0352820D0362824D03F2828D030280C
:109220002FD10021244801702DE001202349087529
:109230000020487527E0012020490875487522E084
:1092400002201E490875002048751CE002201B49B9
:1092500008750120487516E0062018490875002099
:10926000487510E0062015490875012048750AE088
:10927000FFF796FF0106090E1148FCF7B5FE012025
:1092800017E0002015E00F48007803280ED10E48A3
:10929000007800280AD101210C48017006480078A6
:1092A00007F0EEFD0120002103F0A4FF012000E003
:1092B000002008BC1847C046E6210040D2210040EB
:1092C00056210000E0210040E52100409C240040A0
:1092D000002108480078002807D0022805D1012184
:1092E00005480078002800D00221081C0006000E66
:1092F0007047C046E6210040E421004000B5021C52
:10930000081C0006000E052839D1101C00793128F0
:1093100009D032280DD03F2811D0302818D1002193
:109320001848017016E0022017490875002088745B
:1093300010E0022014490875012088740AE0FFF744
:10934000C7FF0106090E1148FCF74EFE012017E089
:10935000002015E00E48007803280ED10D48007853
:1093600000280AD001210C4801700648007807F057
:1093700087FD0120002103F03DFF012000E00020D7
:1093800008BC1847E6210040D22100404D210000D2
:10939000E0210040E52100409C2400400020011C09
:1093A000164A1278012A09D0022A0ED0032A13D0B5
:1093B000042A18D0002A1CD1011C1AE001211048EF
:1093C0000078002815D0022113E003210C48007812
:1093D00000280ED004210CE005210948007800285F
:1093E00007D0062105E0072105480078002800D0B5
:1093F0000821081C0006000E7047C046E32100400B
:10940000E421004000B5021C081C0006000E0428E0
:1094100064D1101CC078312815D0322819D03328D7
:109420001CD0342820D0352824D0362828D03728FE
:109430002CD0382830D03F2834D030283BD10021E0
:109440002848017039E001202749487400208874B9
:1094500033E001202449487488742EE00220224918
:1094600048740020887428E002201F4948740120B5
:10947000887422E003201C494874002088741CE092
:109480000320194948740120887416E00420164905
:1094900048740020887410E00420134948740120A7
:1094A00088740AE0FFF77AFF0106090E0F48FCF7FF
:1094B0009BFD012013E0002011E00D4800780128F9
:1094C0000AD101210B4801700648007807F02CFDF5
:1094D0000120002103F08EFE012000E0002008BCE6
:1094E0001847C046E3210040D2210040452100003A
:1094F000E02100409C2400400120704710B5041C6E
:1095000081B000200090081C0006000E052820D124
:10951000201C00793F280FD0442807D0552814D1AB
:1095200001200021002203F085FE10E00121081C2B
:10953000002203F07FFE0AE01A48008800040014AD
:10954000011C1948FCF750FD01E0002025E0012036
:1095500023E0201C007973281ED1201C053000A9AF
:10956000FFF7A6FB0006000E012815D100980AF0AF
:1095700045FD0004001403F0E5FF0006000E01287D
:109580000AD100980AF03AFD0204121401200221C7
:1095900003F050FE012000E0002001B010BC08BC28
:1095A0001847C046D42100403B21000070B5161C6E
:1095B0000C1C051C321C201C03061B0E9B00281CC7
:1095C0000106090E1C204143C9180D484250281CB1
:1095D0000006000E07F0D8FD301C05F069FF0106FB
:1095E000090E281C0006000E05225043054A80186B
:1095F000221C1206120E8018FCF7CAFC70BDC04671
:10960000B42200403B010000021C081C31280BD092
:10961000322809D0332807D0342805D0352803D084
:10962000362801D0302809D1081C0106090E30392E
:109630000906090E101C0170012000E0002070478F
:1096400000B5031C82B0002200A802700020019027
:10965000081C0006000E082826DD181C4079732817
:1096600022D1181C8079011C00A8FFF7CDFF00064D
:10967000000E012818D1181C073001A9FFF718FBAC
:109680000006000E01280FD10198FFF7FBFA000633
:10969000000E012808D100A80078011C019A0020C2
:1096A000FFF784FF012000E0002002B008BC18474B
:1096B00000B5031C82B0002200A8027000200190B7
:1096C000081C0006000E082826DD181C40797328A7
:1096D00022D1181C8079011C00A8FFF795FF000615
:1096E000000E012818D1181C073001A9FFF7E0FA75
:1096F0000006000E01280FD10198FFF7C3FA0006FB
:10970000000E012808D100A80078011C019A012050
:10971000FFF74CFF012000E0002002B008BC184712
:1097200000B5031C82B0002200A802700020019046
:10973000081C0006000E082826DD181C4079732836
:1097400022D1181C8079011C00A8FFF75DFF0006DC
:10975000000E012818D1181C073001A9FFF7A8FA3C
:109760000006000E01280FD10198FFF78BFA0006C2
:10977000000E012808D100A80078011C019A0220DF
:10978000FFF714FF012000E0002002B008BC1847DA
:1097900000B5031C82B0002200A8027000200190D6
:1097A000081C0006000E092826DD181C8079732885
:1097B00022D1181CC079011C00A8FFF725FF000664
:1097C000000E012818D1181C083001A9FFF770FA03
:1097D0000006000E01280FD10198FFF753FA00068A
:1097E000000E012808D100A80078011C019A04206D
:1097F000FFF7DCFE012000E0002002B008BC1847A3
:1098000010B5041C82B0002200A802700020019054
:10981000081C0006000E0A2826DD201CC0797328CB
:1098200022D1201C007A011C00A8FFF7EDFE0006E3
:10983000000E012818D1201C093001A9FFF738FAC1
:109840000006000E01280FD10198FFF71BFA000651
:10985000000E012808D100A80078011C019A0720F9
:10986000FFF7A4FE012000E0002002B010BC08BCFD
:109870001847C04610B5041C82B0002200A8027030
:1098800000200190081C0006000E0A2826DD201C7E
:10989000C079732822D1201C007A011C00A8FFF790
:1098A000B3FE0006000E012818D1201C093001A9C2
:1098B000FFF7FEF90006000E01280FD10198FFF70F
:1098C000E1F90006000E012808D100A80078011C6B
:1098D000019A0620FFF76AFE012000E0002002B096
:1098E00010BC08BC1847C04610B5041C82B000224A
:1098F00000A8027000200190081C0006000E092834
:1099000026DD201C8079732822D1201CC079011CFF
:1099100000A8FFF779FE0006000E012818D1201CD0
:10992000083001A9FFF7C4F90006000E01280FD185
:109930000198FFF7A7F90006000E012808D100A83A
:109940000078011C019A0320FFF730FE012000E09F
:10995000002002B010BC08BC1847C04610B5041C5B
:1099600082B0002200A8027000200190081C0006AE
:10997000000E092826DD201C8079732822D1201CA6
:10998000C079011C00A8FFF73FFE0006000E012869
:1099900018D1201C083001A9FFF78AF90006000E33
:1099A00001280FD10198FFF76DF90006000E01287C
:1099B00008D100A80078011C019A0520FFF7F6FDE8
:1099C000012000E0002002B010BC08BC1847C046CF
:1099D00000B5021C081C0006000E052815D1101C3D
:1099E0000079312809D030280FD1002108480170B2
:1099F000002007F0DDFB012008E001210448017090
:109A0000012007F0D5FB012000E0002008BC18472A
:109A1000E623004000B5021C081C0006000E0428C6
:109A20001FD1101CC078312803D03F2807D0302820
:109A300013D1011C3039022003F05AFC0FE002F070
:109A400019FE0006000E012803D10748FCF7CCFAE6
:109A500005E00648FCF7C8FA01E0002002E001201A
:109A600000E0002008BC1847342100002D21000030
:109A700011480078012811D002280FD003280DD0FA
:109A800004280BD0052809D0062807D0072805D0C0
:109A9000082805D0092805D000280BD101300AE09C
:109AA000002008E005480078012801D1092002E0E3
:109AB0000A2000E000207047DA210040851F0040A6
:109AC00070B50D1C041C281C0006000E04283BD198
:109AD000201CC678312E18D0322E16D0332E14D03A
:109AE000342E12D0352E10D0362E0ED0372E0CD06C
:109AF000382E0AD0392E0ED03F2E14D0302E1BD146
:109B00000220082103F014FC18E0311C3139022036
:109B100003F00EFC12E0012002F0B6FD0220092144
:109B200003F006FC0AE0FFF7A3FF0106090E154843
:109B3000FCF75AFA012022E0002020E00220002158
:109B400003F058FB01201AE0281C0006000E05282F
:109B500014D1201CC078312810D1201C0079302865
:109B60000CD1022002F090FD0220092103F0E0FB5D
:109B70000220002103F03EFB012000E0002070BC29
:109B800008BC18472521000010B5041C81B0081C32
:109B90000006000E042820D1201CC0783F280FD0DA
:109BA000442807D0552814D102200021002203F0B8
:109BB00041FB10E002200121002203F03BFB0AE000
:109BC0001A48008800040014011C1948FCF70CFA1C
:109BD00001E0002025E0012023E0201CC07873284C
:109BE0001ED1201C043000A9FFF762F80006000E09
:109BF000012815D100980AF001FA0004001403F0BE
:109C0000A1FC0006000E01280AD100980AF0F6F91E
:109C1000020412140221081C03F00CFB012000E0D6
:109C2000002001B010BC08BC1847C046DC21004031
:109C30001C21000000B5021C081C0006000E0428B0
:109C400016D1101CC07833280DD034280BD03528FD
:109C500009D0362807D0372805D0382803D03F2828
:109C600006D0322804D13138F9F7CAFE012000E0CD
:109C7000002008BC1847C04670B50D1C041C281CE9
:109C80000006000E042832D1201CC678312E17D0D1
:109C9000322E15D0332E13D0342E11D0352E0FD0B6
:109CA000362E0DD0372E0BD0382E09D0392E0ED0AF
:109CB000302E1CD10220082103F03AFB012034E0B1
:109CC000311C3139022003F033FB01202DE0042048
:109CD00001F068FA0006000E002802D1022002F00E
:109CE000D3FC0220092103F023FB01201DE0281CE6
:109CF0000006000E052817D1201CC078312813D18A
:109D0000201C007930280FD1042001F04BFA000606
:109D1000000E002802D1012002F0B6FC0220092129
:109D200003F006FB012000E0002070BC08BC1847CF
:109D300000B5021C081C0006000E04280DD1101CE2
:109D4000C078312801D0302807D1021C303A0221D6
:109D5000081C03F00DFB012000E0002008BC1847A0
:109D60000120704710B5041C81B000200090081C31
:109D70000006000E032817D1201C80783F2811D040
:109D8000442807D055280BD101200021002203F0E0
:109D900051FA07E00121081C002203F04BFA01E010
:109DA000002025E0012023E0201C807873281ED1AC
:109DB000201C033000A9FEF77BFF0006000E0128DF
:109DC00015D100980AF01AF90004001403F0BAFB48
:109DD0000006000E01280AD100980AF00FF90204CB
:109DE00012140120022103F025FA012000E00020D6
:109DF00001B010BC08BC184700B5021C081C0006C6
:109E0000000E03280FD1101C8078312805D030288F
:109E100007D10020F9F734FF05E00120F9F730FF02
:109E200001E0002000E0002008BC184730B5051C08
:109E3000081C0006000E022812D1281C4078041CC1
:109E40002B2C05D10020012101F0C6FC012008E0E7
:109E50002D2C05D10121081C01F0BEFC012000E0E1
:109E6000002030BC08BC184710B5021C81B0081C8B
:109E70000006000E042824DB101C033000A9FEF7A6
:109E800017FF0006000E01281BD100980AF0B6F853
:109E9000041C201C0006000E1E2801DD002011E01D
:109EA00001F09EF90006000E042808D1201C0006CF
:109EB000000E01F023FE0420002103F09BF9012095
:109EC00000E0002001B010BC08BC1847012070471A
:109ED00030B50D1C041C81B0281C0006000E04289F
:109EE00013D1201CC078442806D0552809D102205F
:109EF000002101F071FC06E00320002101F06CFC60
:109F000001E0002022E0012020E0281C0006000ED5
:109F100004281ADD201C033000A9FEF7C9FE000644
:109F2000000E012811D100980AF068F8031C181CD3
:109F3000022101F0CBFC0006000E012805D1191CFE
:109F4000022001F009FC012000E0002001B030BC3B
:109F500008BC184710B5021C81B0081C0006000E92
:109F6000042824DB101C033000A9FEF7A1FE000624
:109F7000000E01281BD100980AF040F8041C201C98
:109F80000006000E1E2801DD002011E001F028F976
:109F90000006000E042808D1201C0006000E01F067
:109FA000ADFD0420002103F025F9012000E0002090
:109FB00001B010BC08BC18470120704730B50D1C1B
:109FC000041C81B0281C0006000E042813D1201C9C
:109FD000C078442806D0552809D10220002101F07C
:109FE000FBFB06E00320002101F0F6FB01E000206E
:109FF00025E0012023E0281C0006000E04281DDDBA
:10A00000201C033000A9FEF753FE0006000E0128B5
:10A0100014D10D49009809F04BFE09F0EFFF031C25
:10A02000181C012101F052FC0006000E012805D188
:10A03000191C012001F090FB012000E0002001B07C
:10A0400030BC08BC1847C04600007A4400B5021C6A
:10A05000081C0006000E03282CD1101C8078312823
:10A0600010D03F281BD0302820D101F0B9F80006CD
:10A07000000E04281CD10021104801700020FAF7BE
:10A080000DF815E001F0ACF80006000E04280FD121
:10A0900001210A4801700120FAF700F808E007489A
:10A0A0000078011C0648FBF79FFF01E0002002E05A
:10A0B000012000E0002008BC1847C046881F00406F
:10A0C0001521000010B5081C0006000E032820D141
:10A0D00012480078012813D1114C2068114B191C2B
:10A0E0000AF06EFF64210AF06BFF081C021C206856
:10A0F000191C0AF065FF081C0B48FBF775FF08E008
:10A100000748006807490AF05BFF081C0748FBF78F
:10A110006BFF012010BC08BC1847C046851F0040DB
:10A12000741F0040E8030000092100000121000025
:10A1300000B5021C081C0006000E03280FD1101CDD
:10A140008078312805D0322803D0332801D0302838
:10A1500005D13038022102F0F5FF012000E0002097
:10A1600008BC184770B5061C301CC078312813D0C5
:10A17000322811D033280FD034280DD035280BD0F9
:10A18000362809D0372807D0382805D030280ED1F6
:10A19000184A156883240CE0041CA2001648855850
:10A1A0000C204443154824182406240E01E0002006
:10A1B0001DE0081C0006000E042817DD301C0430CA
:10A1C0000C21FEF7DBFD0006000E01280CD1281C37
:10A1D000311C04310C220AF0EDFD201C0006000E9B
:10A1E0002A1C0C21FDF702F9012000E0002070BCC0
:10A1F00008BC1847002000401C1F0040D7FDFFFF8F
:10A2000000B5011C81B0081CC07873281DD1081C42
:10A21000043000A9FEF74CFD0006000E012814D101
:10A220000098FEF72FFD0006000E01280DD10099C1
:10A230000020FAF7DFFE009805F03AF90106090E52
:10A240001920FBF7A5FE012000E0002001B008BCAA
:10A250001847C04600B5011C81B0081CC07873289F
:10A260001DD1081C043000A9FEF722FD0006000ED7
:10A27000012814D10098FEF705FD0006000E012804
:10A280000DD100990120FAF7B5FE009805F010F9FC
:10A290000106090E1A20FBF77BFE012000E00020DA
:10A2A00001B008BC1847C04600B5011C81B0081CAD
:10A2B000C07873281DD1081C043000A9FEF7F8FCF3
:10A2C0000006000E012814D10098FEF7DBFC000602
:10A2D000000E01280DD100990220FAF78BFE00989C
:10A2E00005F0E6F80106090E1B20FBF751FE0120E0
:10A2F00000E0002001B008BC1847C04600B5011CB2
:10A3000081B0081C007973281DD1081C053000A9F4
:10A31000FEF7CEFC0006000E012814D10098FEF7CF
:10A32000B1FC0006000E01280DD100990420FAF7B7
:10A3300061FE009805F0BCF80106090E1D20FBF730
:10A3400027FE012000E0002001B008BC1847C046ED
:10A3500000B5011C81B0081C007973281DD1081CB0
:10A36000053000A9FEF7A4FC0006000E012814D158
:10A370000098FEF787FC0006000E01280DD1009919
:10A380000320FAF737FE009805F092F80106090E4F
:10A390001C20FBF7FDFD012000E0002001B008BCFF
:10A3A0001847C04600B5011C81B0081C007973280D
:10A3B0001DD1081C053000A9FEF77AFC0006000E2E
:10A3C000012814D10098FEF75DFC0006000E01285C
:10A3D0000DD100990720FAF70DFE009805F068F8F6
:10A3E0000106090E2020FBF7D3FD012000E000202C
:10A3F00001B008BC1847C04600B5011C81B0081C5C
:10A40000007973281DD1081C053000A9FEF750FC07
:10A410000006000E012814D10098FEF733FC000658
:10A42000000E01280DD100990620FAF7E3FD0098EF
:10A4300005F03EF80106090E1F20FBF7A9FD0120DB
:10A4400000E0002001B008BC1847C04600B5011C60
:10A4500081B0081C007973281DD1081C053000A9A3
:10A46000FEF726FC0006000E012814D10098FEF726
:10A4700009FC0006000E01280DD100990520FAF70D
:10A48000B9FD009805F014F80106090E1E20FBF72F
:10A490007FFD012000E0002001B008BC1847C04645
:10A4A00010B5021C081C00280DD00024101C211C13
:10A4B0000AF068FD15D30C4C101C211C0AF062FD3B
:10A4C0000FD801200EE00024101C211C0AF05AFDB8
:10A4D00007D3064C101C211C0AF054FD01D80120A2
:10A4E00000E0002010BDC0460000C8429B6CF24155
:10A4F000021C081C0006000E042811D1101CC07894
:10A50000312805D0302807D100210648017005E028
:10A5100001210448017001E0002002E0012000E078
:10A5200000207047301F004000B5021C81B0081C9D
:10A530000006000E032826DD101C033000A9FEF7DC
:10A54000B7FB0006000E01281DD111480078011C40
:10A550000098FFF7A5FF0006000E012813D1009810
:10A5600009F04CFD0106090E0022101CFCF786FCC8
:10A57000009809F043FD0106090E02200022FCF7B5
:10A580007DFC012000E0002001B008BC1847C04657
:10A59000301F004000B5021C81B0081C0006000EF0
:10A5A000032826DD101C033000A9FEF781FB0006FE
:10A5B000000E01281DD111480078011C0098FFF7FA
:10A5C0006FFF0006000E012813D1009809F016FD58
:10A5D0000106090E00200122FCF750FC009809F04A
:10A5E0000DFD0106090E02200122FCF747FC0120A7
:10A5F00000E0002001B008BC1847C046301F0040F2
:10A6000000B5021C81B0081C0006000E032826DDE0
:10A61000101C033000A9FEF74BFB0006000E0128BA
:10A620001DD111480078011C0098FFF739FF000682
:10A63000000E012813D1009809F0E0FC0106090E74
:10A6400000200222FCF71AFC009809F0D7FC010652
:10A65000090E0222101CFCF711FC012000E0002072
:10A6600001B008BC1847C046301F004000B5021CAE
:10A6700081B0081C0006000E042826DD101C0430E2
:10A6800000A9FEF715FB0006000E01281DD1114898
:10A690000078011C0098FFF703FF0006000E012858
:10A6A00013D1009809F0AAFC0106090E002004222B
:10A6B000FCF7E4FB009809F0A1FC0106090E02205A
:10A6C0000422FCF7DBFB012000E0002001B008BC05
:10A6D0001847C046301F004000B5021C81B0081C5E
:10A6E0000006000E042826DD101C043000A9FEF729
:10A6F000DFFA0006000E01281DD111480078011C68
:10A700000098FFF7CDFE0006000E012813D1009837
:10A7100009F074FC0106090E00200322FCF7AEFBD1
:10A72000009809F06BFC0106090E02200322FCF7D9
:10A73000A5FB012000E0002001B008BC1847C0467E
:10A74000301F004000B5021C81B0081C0006000E3E
:10A75000042826DD101C043000A9FEF7A9FA000623
:10A76000000E01281DD111480078011C0098FFF748
:10A7700097FE0006000E012813D1009809F03EFC58
:10A780000106090E00200722FCF778FB009809F06B
:10A7900035FC0106090E02200722FCF76FFB0120A1
:10A7A00000E0002001B008BC1847C046301F004040
:10A7B00000B5021C81B0081C0006000E042826DD2E
:10A7C000101C043000A9FEF773FA0006000E0128E1
:10A7D0001DD111480078011C0098FFF761FE0006AA
:10A7E000000E012813D1009809F008FC0106090E9B
:10A7F00000200622FCF742FB009809F0FFFB01064F
:10A80000090E02200622FCF739FB012000E000209F
:10A8100001B008BC1847C046301F004000B5021CFC
:10A8200081B0081C0006000E032826DD101C033032
:10A8300000A9FEF73DFA0006000E01281DD11148BF
:10A840000078011C0098FFF72BFE0006000E01287F
:10A8500013D1009809F0D2FB0106090E0020052251
:10A86000FCF70CFB009809F0C9FB0106090E022059
:10A870000522FCF703FB012000E0002001B008BC2A
:10A880001847C046301F004000B5021C81B0081CAC
:10A890000006000E032826DD101C033000A9FEF779
:10A8A00007FA0006000E01281DD111480078011C8E
:10A8B0000098FFF7F5FD0006000E012813D100985F
:10A8C00009F09CFB0106090E0022101CFCF764F83D
:10A8D000009809F093FB0106090E02200022FCF704
:10A8E0005BF8012000E0002001B008BC1847C0461A
:10A8F000301F004010B5041C081C0006000E05287F
:10A9000014D1201C0079312801D030280ED1011C2F
:10A910003039002000F084FB201C0079011C303904
:10A9200002200022FCF76EFA012000E0002010BC9B
:10A9300008BC184710B5041C081C0006000E0528AA
:10A9400014D1201C0079312801D030280ED1011CEF
:10A950003039022000F064FB201C0079011C3039E2
:10A960000222101CFCF74EFA012000E0002010BC6F
:10A9700008BC184710B5041C081C0006000E05286A
:10A9800014D1201C0079312801D030280ED1011CAF
:10A990003039032000F044FB201C0079011C3039C1
:10A9A00002200322FCF72EFA012000E0002010BC58
:10A9B00008BC184710B5041C081C0006000E05282A
:10A9C00014D1201C0079312801D030280ED1011C6F
:10A9D0003039042000F024FB201C0079011C3039A0
:10A9E00002200422FCF70EFA012000E0002010BC37
:10A9F00008BC184710B5041C081C0006000E0528EA
:10AA000014D1201C0079312801D030280ED1011C2E
:10AA10003039062000F004FB201C0079011C30397D
:10AA200002200622FCF7EEF9012000E0002010BC15
:10AA300008BC184710B5041C081C0006000E0528A9
:10AA400014D1201C0079312801D030280ED1011CEE
:10AA50003039072000F0E4FA201C0079011C30395D
:10AA600002200722FCF7CEF9012000E0002010BCF4
:10AA700008BC184710B5041C081C0006000E04286A
:10AA800014D1201CC078312801D030280ED1011CEF
:10AA90003039012000F0C4FA201CC078011C303984
:10AAA00002200122FCF7AEF9012000E0002010BCDA
:10AAB00008BC184710B5041C081C0006000E052829
:10AAC00014D1201C0079312801D030280ED1011C6E
:10AAD0003039052000F0A4FA201C0079011C30391F
:10AAE00002200522FCF78EF9012000E0002010BCB6
:10AAF00008BC184700B5011C081C09F07FFA011CAE
:10AB0000081C282815D0322813D03C2811D04628FC
:10AB10000FD050280DD05A280BD0642809D06E28A9
:10AB200007D0782805D0822803D0962801D00028A5
:10AB300001D1012000E0002000BDC046011C081C1E
:10AB4000282817D0322817D03C2817D0462817D0ED
:10AB5000502817D05A2817D0642817D06E2817D03D
:10AB6000782817D0822817D0962817D0002817D118
:10AB7000002016E0012014E0022012E0032010E083
:10AB800004200EE005200CE006200AE0072008E083
:10AB9000082006E0092004E00A2002E00B2000E083
:10ABA0000020704700B5021C81B0081C0006000E92
:10ABB00003282DDD101C033000A9FEF779F80006EC
:10ABC000000E012824D10098FFF794FF0006000E24
:10ABD00001281DD1009809F011FA0006000EFFF7B8
:10ABE000ADFF09F0E1F90090009809F007FA0106BD
:10ABF000090E00200522FCF73FFA009809F0FEF943
:10AC00000106090E02200522FCF736FA012000E0B9
:10AC1000002001B008BC184700B5021C81B0081C18
:10AC20000006000E05282DDD101C053000A9FEF7DA
:10AC30003FF80006000E012824D10098FFF75AFFC4
:10AC40000006000E01281DD1009809F0D7F9000672
:10AC5000000EFFF773FF09F0A7F90090009809F0C4
:10AC6000CDF90106090E0022101CFCF705FA009828
:10AC700009F0C4F90106090E02200022FCF7FCF9D4
:10AC8000012000E0002001B008BC184700B5021CFC
:10AC900081B0081C0006000E05282DDD101C0530B3
:10ACA00000A9FEF705F80006000E012824D100983F
:10ACB000FFF720FF0006000E01281DD1009809F0C3
:10ACC0009DF90006000EFFF739FF09F06DF90090BD
:10ACD000009809F093F90106090E00200122FCF703
:10ACE000CBF9009809F08AF90106090E0220012229
:10ACF000FCF7C2F9012000E0002001B008BC1847B1
:10AD000000B5021C81B0081C0006000E05282DDDD0
:10AD1000101C053000A9FDF7CBFF0006000E01282E
:10AD200024D10098FFF7E6FE0006000E01281DD191
:10AD3000009809F063F90006000EFFF7FFFE09F026
:10AD400033F90090009809F059F90106090E002026
:10AD50000222FCF791F9009809F050F90106090E5A
:10AD60000222101CFCF788F9012000E0002001B04D
:10AD700008BC184700B5021C81B0081C0006000E74
:10AD800005282DDD101C053000A9FDF791FF0006F8
:10AD9000000E012824D10098FFF7ACFE0006000E3B
:10ADA00001281DD1009809F029F90006000EFFF7CF
:10ADB000C5FE09F0F9F80090009809F01FF90106A6
:10ADC000090E00200422FCF757F9009809F016F943
:10ADD0000106090E02200422FCF74EF9012000E0D2
:10ADE000002001B008BC184700B5021C81B0081C47
:10ADF0000006000E05282DDD101C053000A9FDF70A
:10AE000057FF0006000E012824D10098FFF772FEBC
:10AE10000006000E01281DD1009809F0EFF8000689
:10AE2000000EFFF78BFE09F0BFF80090009809F0C4
:10AE3000E5F80106090E00200322FCF71DF9009831
:10AE400009F0DCF80106090E02200322FCF714F9D0
:10AE5000012000E0002001B008BC184700B5021C2A
:10AE600081B0081C0006000E06282DDD101C0630DF
:10AE700000A9FDF71DFF0006000E012824D100984F
:10AE8000FFF738FE0006000E01281DD1009809F0DA
:10AE9000B5F80006000EFFF751FE09F085F80090A6
:10AEA000009809F0ABF80106090E00200722FCF714
:10AEB000E3F8009809F0A2F80106090E0220072223
:10AEC000FCF7DAF8012000E0002001B008BC1847C8
:10AED00000B5021C81B0081C0006000E06282DDDFE
:10AEE000101C063000A9FDF7E3FE0006000E012845
:10AEF00024D10098FFF7FEFD0006000E01281DD1A9
:10AF0000009809F07BF80006000EFFF717FE09F025
:10AF10004BF80090009809F071F80106090E002026
:10AF20000622FCF7A9F8009809F068F80106090E56
:10AF300002200622FCF7A0F8012000E0002001B06A
:10AF400008BC184701207047021C081C0378101C1D
:10AF50000078984201D0002006E001320131101C37
:10AF600000780028F1D101207047C04670B50E1C52
:10AF7000051C0024301C0106090E281C44541EE048
:10AF8000201C0106090E8900124840580068291C3F
:10AF9000FFF7DAFF0006000E01280DD1301C010674
:10AFA000090E281C221C13061B0E9B00094AD258AE
:10AFB000526809F0FFFF0BE001342406240E201C28
:10AFC0000106090E8900034840580028D8D1002006
:10AFD00070BDC046D81D004000B5011C081C00060D
:10AFE000000E06F0A9FA012000BDC04600B5021C03
:10AFF000081C0104090C101C0006000E06F0E2FA01
:10B00000012000BD00B50A1C011C081C0006000E32
:10B01000111C0906090E06F067FB012000BDC046A1
:10B0200000B50A1C011C081C0006000E111C0906B4
:10B03000090E06F0B1FB012000BDC04600B50A1C98
:10B04000011C081C0006000E111C0906090E06F062
:10B0500011FC012000BDC04600B5131C0A1C011CD8
:10B06000081C0006000E111C0906090E1A1C120607
:10B07000120E06F09FFB012000BDC04600B50A4835
:10B08000006800280AD1094809F0C0FE0649086096
:10B0900005480068002801D1002004E00020024992
:10B0A000C8808880012000BD341F0040980800003F
:10B0B00030B50B1C051C00F05FF8002801D0002003
:10B0C00022E0124CA088000400140130C82109F0CD
:10B0D0009BFF011C0804000CA080A0880004001441
:10B0E000011C0B204143206840180130191C082224
:10B0F00009F060FE281CA188090409140A1C0B2110
:10B100004A4321688854012030BDC046341F0040A6
:10B1100000B5021C00F020F8002801D0002017E044
:10B120000C4BD888000400140130C82109F06CFFD2
:10B13000011C0804000CD880D888000400140B21DE
:10B14000484319680918101C0B2209F033FE01202E
:10B1500000BDC046341F0040064841880904091458
:10B16000008800040014884201D1012000E0002082
:10B170007047C046381F004000B5094A10880004D7
:10B1800000140130C82109F03FFF011C5088000461
:10B190000014814201D1012000E0002000BDC04622
:10B1A000381F0040011C081C0106090E03480078E6
:10B1B000884201D1012000E000207047581F004064
:10B1C000021C101C0006000E002801D1002003E024
:10B1D000111C0248017001207047C046581F0040F2
:10B1E000014800787047C046581F004070B5061CE3
:10B1F000301C0578281C0006000E002802D1FFF73D
:10B20000EFFF051C002414E0201C03061B0E9B000E
:10B210000D48C15808782A1C1206120E904205D11A
:10B22000301C0130496809F0C4FE0BE001342406EB
:10B23000240E201C0106090E8900034840580028EE
:10B24000E2D1002070BDC0463C1F004070B5041C18
:10B2500081B0201C007809283AD00C2865D00D2830
:10B2600000D1C1E10E2800D110E2012800D066E231
:10B27000201C4078FBF7F8FA0120FAF7D1FF00F024
:10B2800067FC0006000E012805D000F061FC0006F6
:10B29000000E022808D1002000F052FC05200021F9
:10B2A00000F09AFA01204BE2201C4578281C000689
:10B2B000000E00F065FF051C0006000E002805D0FA
:10B2C000201C01F01BFE0006000E39E2012037E2CF
:10B2D000FFF786FF0006000E042801D000202FE2B1
:10B2E000DE48417C827D006800F02EFD01200021B7
:10B2F000FAF7F0FFDA480078012805D1D94A14207E
:10B300000221FAF7A3FF0EE0D7480078002805D005
:10B31000D64A14200221FAF799FF04E0D44A1420F7
:10B320000221FAF793FF01200AE2FFF759FF000616
:10B33000000E042801D0002002E2201C40780128E1
:10B3400053D0022800D195E0032800D1A5E00428BD
:10B3500000D1B5E0052800D13FE1002800D0EEE1A2
:10B36000201C807801280DD100F0F2FB0006000EB1
:10B37000012801D10020E3E10220F8F733FE01208B
:10B3800000F0DEFB00F0E4FB0006000E012801D017
:10B390000020D5E1B14D687C011C2868012200F035
:10B3A000CDFD2860687C021C28680021F8F766FD46
:10B3B0001E20FAF785FB0420002101F01BFF687CAA
:10B3C000011C286800F080FC0006000E012804D152
:10B3D0000520002100F000FAB1E17820FAF770FBB7
:10B3E0000021081C00F0F8F9A9E1201C8078012850
:10B3F0000DD100F0ADFB0006000E012801D10020A8
:10B400009EE10220F8F7EEFD012000F099FB00F02C
:10B410009FFB0006000E012801D0002090E18F4D17
:10B42000687C011C2868002200F088FD2860687C88
:10B43000021C28680021F8F721FD1E20FAF740FBC6
:10B440000420002101F0D6FE687C011C286800F071
:10B450003BFC0006000E012804D10520002100F06D
:10B46000BBF96CE17820FAF72BFB0120002100F0FA
:10B47000B3F964E1794D687C011C2868012200F071
:10B480005DFD2860687C021C28680021F8F7F6FC46
:10B490000420002101F0AEFE51E1704D687C011CDA
:10B4A0002868002200F04AFD2860687C021C286899
:10B4B0000021F8F7E3FC0420002101F09BFE3EE1AF
:10B4C000201C807801281BD100F042FB0006000EF2
:10B4D000022801D1002033E10220F8F783FD022089
:10B4E00000F02EFB63480078012803D16249086808
:10B4F000486002E061490868086100216048017005
:10B5000000F026FB0006000E022801D0002017E103
:10B51000524D687C021C28680021F8F7AFFC1E2001
:10B52000FAF7CEFA687C011CA87D021C286800F09E
:10B530000BFC2868012100F0C7FB0006000E012863
:10B5400012D10320F8F74EFD444DA87D697C0A1CFA
:10B55000296800F059FB4B48FAF7B2FA0220F8F7D5
:10B5600041FDA87D0130A87542480678301C0128AD
:10B5700004D142498A680969914206D3022813D14D
:10B5800041480168406988420ED2344D311C286818
:10B59000012200F0D3FC28600420002100F01CF9F7
:10B5A0007820FAF78DFACAE000202C4DA87500200B
:10B5B000321C2A4900F032F9687C021C28680021FC
:10B5C000F8F75CFC002000F0BBFA0320F8F70AFD56
:10B5D0000420002101F00EFEB1E0002000F0B0FADE
:10B5E0000320F8F7FFFCAAE0201C4078012821D0B6
:10B5F000002800D0A3E0201C80781E4D29780A1C6A
:10B6000000A900F00BF9201C8078687128780128C7
:10B6100003D118494879887002E016494879487082
:10B6200000990E480160417C0A1C00680021F8F76F
:10B6300025FC84E0201C033000F090FA0090201CD0
:10B6400080780C4D2978022200F032FC687168790C
:10B6500029780A1C009900F0D7FA70E0741F0040A6
:10B66000D8210040DC210000891F0040D7210000C4
:10B67000D0210000851F0040701F0040641F004063
:10B680008A1F0040E8030000601F0040FFF7A8FD8C
:10B690000006000E042801D0002051E0201C407854
:10B6A000012827D002284AD1201C023000F056FA87
:10B6B00000900098022100F009F90006000E012810
:10B6C0003DD121480078022806D000991F4801602A
:10B6D000022000F0C9FB08E000991D480160417C90
:10B6E0000A1C00680021F8F7C9FB0420002101F0C2
:10B6F00081FD24E0201C023000F030FA0090009818
:10B70000012100F0E3F80006000E012817D10E48D1
:10B710000078012806D000990E480160012000F051
:10B72000A3FB08E000990A480160417C0A1C0068FC
:10B730000021F8F7A3FB0420002101F05BFD0020AD
:10B7400001B070BC08BC1847851F00407C1F00403A
:10B75000741F0040781F004030B50C1C051C82B0DF
:10B760001C4900A808220B780370491C401C521E7B
:10B77000F9D10E2100A80170291C01206844017034
:10B78000211C090EFF2001400906090E0220684411
:10B790000170211C090CFF2001400906090E03203D
:10B7A00068440170211C090AFF2001400906090EA6
:10B7B00001A80170211CFF2001400906090E052087
:10B7C0006844017000A90420FFF772FC0006000E17
:10B7D00002B030BD8822000030B50C1C051C82B0C0
:10B7E0000D4900A808220B780370491C401C521E0A
:10B7F000F9D10C2100A80170291C012068440170B6
:10B80000211C02206844017000A90420FFF750FCAD
:10B810000006000E02B030BD90220000F0B50D1CF5
:10B82000061C101C0006000E01281FD1301C01064A
:10B83000090E204FF87C4018FAF7C0FB0406240ECE
:10B840006420444339686418201C884209D31A488C
:10B850000168201C884204D8221C281C0260012098
:10B8600026E016480268281C026020E0301C010611
:10B87000090E134E301C203000784018FAF79EFB5A
:10B880000406240EB07F444331686418201C8842AB
:10B8900009D30C480168201C884204D8221C281CAB
:10B8A0000260012004E008480268281C02600020B1
:10B8B000F0BDC046701F00406C1F0040681F004074
:10B8C000641F0040601F00405C1F0040021C081CF9
:10B8D0000006000E01280BD10C480168101C88429C
:10B8E00012D30B480168101C88420DD801200CE0CF
:10B8F00008480168101C884206D307480168101CDC
:10B90000884201D8012000E000207047701F0040ED
:10B910006C1F0040641F0040601F004010B5031CF6
:10B920000420FFF74DFC181C0006000E012807D16B
:10B9300001202049487448680860C87C887506E082
:10B9400002201C49487488680860887C8875194CF6
:10B95000A07D00F0D3F8607CF8F790FB607C021CBF
:10B9600020680021F8F78AFA0320F8F73BFB04204F
:10B97000002101F03FFC0820F7F75EFF0E48007839
:10B98000002809D00220FFF727FB012005F018FA54
:10B990000220F7F7B7FF02E00020F7F7B3FF3220ED
:10B9A000F8F796FF2A20F8F793FF0020F9F7F2FA4C
:10B9B000012010BD741F0040A01D004010B50024E0
:10B9C00010E0201C0006000EA1300021FAF7E0FA7A
:10B9D000201C0006000EBF300021FAF7D9FA01340E
:10B9E0002406240E201C0006000E1E28E9DB00247D
:10B9F00010E0201C0006000EDD300021FAF7C8FA26
:10BA0000201C0006000EFB300021FAF7C1FA0134B9
:10BA10002406240E201C0006000E1E28E9DB10BDA3
:10BA200000B5FFF7DDFB0006000E042849D12548CC
:10BA30000078002845D00021224801702248018862
:10BA400009040914002914D01F48013901801E4837
:10BA5000008800040014002833D11C48F9F728FBA3
:10BA60000106090E1A4801700420002101F0C2FBF2
:10BA700027E01648F9F71CFB0206120E101C0106FF
:10BA8000090E14480078884218D013480178013113
:10BA90000170114800780A2808D1101C0A49C8739F
:10BAA000101C48720420002101F0A4FB0A48007811
:10BAB0000A2806DD0B210848017002E00021064833
:10BAC000017000BD10050040801F00400000001004
:10BAD000891F00408F1F0040901F004000B50120CB
:10BAE000FFF76EFB02200021FAF7F4FB3220F8F793
:10BAF0000FFF2A20F8F70CFF00BDC04610B5041C4C
:10BB000082B00E4900A808220B780370491C401C23
:10BB1000521EF9D10D2100A80170002101206844B6
:10BB20000170211C02206844017000A90420FFF765
:10BB3000BFFA0006000E02B010BDC04698220000F9
:10BB4000021C111C014801707047C0468B1F004049
:10BB5000014800787047C0468B1F0040021C101C33
:10BB60004078031C1B04101C017809061943101CA3
:10BB7000807800020143101CC0780143081C704704
:10BB800030B50C1C051C82B01E4900A808220B7899
:10BB90000370491C401C521EF9D10D2100A80170F0
:10BBA0000121012068440170291C022068440170B1
:10BBB000211C090EFF2001400906090E03206844DC
:10BBC0000170211C090CFF2001400906090E01A883
:10BBD0000170211C090AFF2001400906090E0520F9
:10BBE00068440170211CFF2001400906090E06204F
:10BBF0006844017000A90420FFF75AFA0006000EFD
:10BC000002B030BDA022000030B50C1C051C101C79
:10BC10000006000E012824D1281C0006000E1E2854
:10BC200045DA24480068211C814240D322490A6831
:10BC3000211C91423BD8241A201C642109F0C0F930
:10BC4000081C041C281C0106090E1C48007840181A
:10BC5000211C0906090E0906090EFAF799F90120B7
:10BC600026E0281C0006000E1E2820DA1448006872
:10BC7000211C81421BD313490A68211C914216D80A
:10BC8000241A0C4A907C011C201C09F099F9081C0C
:10BC9000041C281C0106090E107D4018211C0906F1
:10BCA000090E0906090EFAF773F9012000E00020D9
:10BCB00030BDC046701F00406C1F0040831F004015
:10BCC000641F0040601F004070B50D1C061C022060
:10BCD000F8F788F9281C0206120E301C0121F8F72B
:10BCE000CDF86420F9F7ECFEF8F748F9114C044060
:10BCF000281C0206120E301C0021F8F7BFF8281C81
:10BD00000006000E012809D1201C0B4988420FD3E0
:10BD1000201C0A4988420BD801200AE0201C08494F
:10BD2000884205D3201C0749884201D8012000E041
:10BD3000002070BDFFFF0F003A390500C63905002D
:10BD4000363800004A38000070B5151C0E1C041C63
:10BD500083B03B4900A809220B780370491C401CA2
:10BD6000521EF9D1301C0006000E01283AD1201CC9
:10BD7000344A111C09F024F9642109F021F9081C46
:10BD8000031C201C111C09F01BF9081C021C00A834
:10BD90002D4907F09FFE281C0006000E8021084256
:10BDA00011D0281C0006000E7F2108400A2109F04E
:10BDB0002BF9081C01B4254A01AB00200121FAF738
:10BDC00045FA01B00AE0281C0006000E01B4204A22
:10BDD00001AB00200121FAF739FA01B0211C1D48FE
:10BDE00001602AE000A81C49221C07F073FE281CF1
:10BDF0000006000E8021084211D0281C0006000E0B
:10BE00007F2108400A2109F0FFF8081C01B4134AF9
:10BE100001AB00200121FAF719FA01B00AE0281C51
:10BE20000006000E01B40E4A01AB00200121FAF712
:10BE30000DFA01B0211C0B48016003B070BDC04673
:10BE4000A8220000E80300007C2200006C22000011
:10BE50005B220000781F00405322000043220000B4
:10BE6000322200007C1F004010B5011C081C000697
:10BE7000000E012807D101200C4948744868086069
:10BE8000C87C887506E00220084948748868086004
:10BE9000887C8875054C607CF8F7F0F8607C021CA3
:10BEA00020680021F7F7EAFF012010BD741F004051
:10BEB000031C081C0006000E01281DD1101C0028C0
:10BEC0000AD0022811D0012833D1181C002830D004
:10BED000013B1B061B0E2CE0181C0006000E1E2842
:10BEE00027DA01331B061B0E23E0181C0006000E88
:10BEF0001E281EDD01231CE0101C00280AD0022889
:10BF000011D0012815D1181C002812D0013B1B06A6
:10BF10001B0E0EE0181C0006000E1E2809DA013365
:10BF20001B061B0E05E0181C0006000E1E2800DD77
:10BF30000123181C0006000E7047C046031C081C95
:10BF40000006000E012814D1101C002808D064330C
:10BF500016480168181C884225D91548036822E054
:10BF6000643B13480168181C88421CD20F480368C0
:10BF700019E0101C00280CD00E49081C2230007853
:10BF8000021C9B180968181C88420CD90A480368CF
:10BF900009E00949887F021C9B1A0968181C88421D
:10BFA00001D204480368181C7047C0466C1F00404B
:10BFB000701F0040601F0040641F0040011C081CEF
:10BFC000242824D0252822D0262820D027281ED077
:10BFD00028281CD029281AD02A2818D02B2816D077
:10BFE0002C2814D02D2812D02E2822D114480278C3
:10BFF0000A3213480270124800785A2802DD0021E4
:10C000000F4801700F4841780170032114E0081CAB
:10C010000106090E24390B48427889180906090ED1
:10C0200001700021417001788022114301700321C9
:10C0300002E0002202480270081C0006000E704751
:10C040008E1F00408D1F004000B50020FFF778FDD7
:10C050000420002101F0CEF800BDC04610B5041C3C
:10C06000201C0006000E802108420ED0201C000675
:10C07000000E7F2108400A2108F0C6FF081C031C9F
:10C08000064A14200221FAF7E1F8201C03061B0ED1
:10C09000034A14200221FAF7D9F810BD1C2200002F
:10C0A0000522000000B50320FFF74AFD0348017890
:10C0B00081708078FFF7D2FF00BDC0468A1F004024
:10C0C00070B5011C081C032816D0072832D0082898
:10C0D0003FD034282ED035283BD0382804D0212812
:10C0E00045D1FFF7B1FF42E02249087E0968FFF71A
:10C0F00047FDFFF7A9FF3AE01F480578281C802478
:10C10000204210D07F2028401A4E7076707E717CBD
:10C110000222FFF7CDFE3076307E3168FFF730FD2A
:10C12000FFF792FF23E01548057000782043FFF7E2
:10C1300095FF1CE00F4C207E7F2108402076207E5A
:10C14000617C0022FFF7B4FE2076207EFFF786FF99
:10C150000DE0084C207E7F2108402076207E617C07
:10C160000122FFF7A5FE2076207EFFF777FF002053
:10C1700070BDC046741F00408D1F00408C1F0040E2
:10C1800070B5041C201C0006000EFFF717FF041CEE
:10C19000FFF7DEFC0006000E032805D1201C000678
:10C1A000000EFFF78DFF041C201C032800D104E1C2
:10C1B000042800D134E1052800D1C0E0062800D1D0
:10C1C000C5E0072800D1D4E0082800D1E3E00B281F
:10C1D00000D1C4E00C2800D1C6E00D2800D125E133
:10C1E0000E2800D11CE10F2800D119E1102800D140
:10C1F00016E1112800D113E1122800D110E1132813
:10C2000000D10DE1142800D10AE1152800D107E181
:10C210001A2800D10AE11B2800D107E11D2800D10E
:10C22000FEE01E2800D192E01F2800D187E02028E0
:10C2300076D0212800D1E6E0222876D0232879D0B4
:10C24000302800D1F2E0312800D1EFE0342800D1CD
:10C250008FE0352800D19EE0362800D17FE03728D6
:10C2600000D181E0392800D1D0E03A2800D1DDE0CA
:10C270003B2800D1DAE0412800D1D1E0422800D1AA
:10C28000CEE0432800D1CBE0442800D1C8E04528C7
:10C2900000D1C5E0462800D1C2E0472800D1BFE068
:10C2A000482800D1BCE02F2800D0C3E062480088B5
:10C2B0000004001400281CD060480078002806D034
:10C2C00000215E4801700020F7F7E8FE05E001213B
:10C2D0005A4801700120F7F7E1FE59480078F7F756
:10C2E000CDFE57480078021C564800680021F7F739
:10C2F000C5FD64215048018001200021F9F7EAFFC3
:10C300004E480078002805D04F4A14200221F9F742
:10C310009DFF8FE04D4A14200221F9F797FF89E035
:10C3200004200121FFF758FA84E000200121FFF7E3
:10C3300053FA7FE00121081CFFF74EFA7AE04048EB
:10C340000078012876D00120FFF7E8FA72E03C4837
:10C35000007802286ED00220FFF7E0FA6AE003209E
:10C360000021FFF739FA65E002200021FFF734FAD7
:10C3700060E037480078324909780022FFF798FDDD
:10C380003349087032480078FFF7B8FB04200021D9
:10C3900000F030FF4EE02E4800782949097801224C
:10C3A000FFF786FD2A49087029480078FFF7A6FBA9
:10C3B0000420002100F01EFF3CE0264801780D1CFF
:10C3C0008026354215D07F20014022480170214847
:10C3D00000781B4909780222FFF76AFD1C490870A2
:10C3E0001B480078FFF78AFB0420002100F002FFC1
:10C3F00020E02A1C324312480078011C11480068D2
:10C40000FFF7A2FC16E0FFF74DFE13E00120032129
:10C41000002200F0ADFF0420002100F0EBFE09E057
:10C42000FFF75CFB201C0006000E04E0201C000649
:10C43000000E00E0002070BD801F0040881F0040FB
:10C44000851F0040741F0040F3210000E12100001F
:10C450008A1F00408D1F004030B5041C201C00784E
:10C46000092818D00F2800D1A1E0102869D0112880
:10C4700071D0122878D0012800D0DDE0201C45784A
:10C48000281C0006000EFAF7EFF9281C0006000E23
:10C4900000F0D6F9D2E000F0EDF8002800D1CDE0B0
:10C4A00002200021F9F78AFF66480078092827D181
:10C4B00065480078012818D1644B1868644A111C3B
:10C4C00008F07EFD642108F07BFD081C01B41868AB
:10C4D000111C08F075FD081C01B45E4B0021081CFE
:10C4E0001E22F9F72FFF02B014E05848006801B48B
:10C4F000594B0021081C1E22F9F724FF01B009E066
:10C500005648006801B4564B0021081C1E22F9F75A
:10C5100019FF01B053480078012805D1524B14206F
:10C5200000211E22F9F70EFF504800880004001475
:10C5300001B44F4B112003211E22F9F703FF01B074
:10C540007CE0201C4078002802D000F0D5F875E08F
:10C5500000F020F972E000F08DF800286ED0201C69
:10C56000407800F049F969E000F084F8002865D0CF
:10C57000201C407802280DD003280FD139480078BC
:10C58000012803D100213748017007E00121354817
:10C59000017003E0201C8178324801703148007836
:10C5A000F7F72EFB0220002100F024FE46E000F009
:10C5B00061F8002842D0201C407801280ED00228C3
:10C5C00018D000282BD12948018809040914081C17
:10C5D0000F2824DA01312548018020E02348018812
:10C5E00009040914081C5A22D04218DD01391F48D9
:10C5F000018014E0201C8078021C1202201CC078EC
:10C6000002431204120C101C0004001400F064F821
:10C610000006000E012802D1111C144801801348A5
:10C6200000880004001408F069FAF8F7ADFC022055
:10C63000002100F0DFFD01E0012000E0012030BC1E
:10C6400008BC1847DA210040851F0040741F0040D5
:10C65000E8030000D5220000C4220000941F00401F
:10C66000BD220000DE210040B8220000DC21004095
:10C67000B422000003480078012801D1012000E025
:10C6800000207047D921004010B5011C081C00068D
:10C69000000E022805D102200D4908704878487123
:10C6A00004E001200A49087088784871094C607CD0
:10C6B000F7F7E4FCA07D617C0A1C0649FFF7AEF8A1
:10C6C000607C021C20680021F7F7D8FB012010BD18
:10C6D000851F0040741F0040011C081C000400144A
:10C6E0000F2807DC081C000400145A21C84201DB93
:10C6F000012000E00020704710B51F480078002896
:10C7000001D100F05BFE1D480078012830D01C48A4
:10C71000194C60811B480078F7F7B0FC1948007885
:10C72000021C194800680021F7F7A8FB207AF7F7E8
:10C73000BFF8207A00F0AAFE144908600220002108
:10C7400000F058FD608900040014021C0221081C3E
:10C7500000F070FD0221081C002200F009FE0C48C8
:10C760000078012801D0022802D10120F7F754F9FE
:10C7700001210248017010BDD2210040D9210040A2
:10C78000E2FF0000851F0040741F0040941F00401E
:10C79000A11D004000B51448007800280BD00120EE
:10C7A000F7F72EFA11480078012801D0022802D1AB
:10C7B0000020F7F731F90E480078012805D0012054
:10C7C000F9F72EFD00F030FE09E002200021F9F714
:10C7D000F5FD084B002003210A22F9F7B3FD0021E3
:10C7E0000148017000BDC046D9210040A11D004094
:10C7F000D3210040EA22000000B5021C0023101CD7
:10C800000106090E0C480078884203D0111C0A4822
:10C81000017001230848007800F038FE07490860DD
:10C82000181C002803D004480078F7F741F80220CC
:10C83000002100F0DFFC00BDDA210040941F004021
:10C8400030B5041C55480078002808D1201C4B281E
:10C8500000D0A2E00220012100F04AFD9DE0201C52
:10C860004D2827D04E2838D04F2849D0502861D0A5
:10C87000512879D052287DD0532800D180E0542807
:10C8800000D183E0552800D180E056287ED057287B
:10C890007CD058287AD0592878D05A2876D05B286E
:10C8A00074D05C2872D04C2877D10220002100F08F
:10C8B0001FFD72E00420FEF775FC0006000E002844
:10C8C00002D10220FFF7E0FE0220092100F030FD36
:10C8D0000220002100F08EFC5FE00420FEF762FCE5
:10C8E0000006000E002802D10120FFF7CDFE022035
:10C8F000092100F01DFD0220002100F07BFC4CE02E
:10C900000420FEF74FFC0006000E002845D1244805
:10C910000078092809D1234D687929780022FFF78A
:10C92000C7FA68716879FFF7E9F80220002100F082
:10C9300061FC32E00420FEF735FC0006000E002802
:10C940002BD117480078092809D1164D6879297824
:10C950000122FFF7ADFA68716879FFF7CFF802207E
:10C96000002100F047FC18E002200321002200F023
:10C97000FFFC12E002200021002200F05BFC0CE032
:10C9800002200121002200F055FC06E0201C0106D7
:10C99000090E5439022000F0CBFC30BDD9210040F3
:10C9A000DA210040851F004000B5021C0120FEF77F
:10C9B000F9FB002804D10420FEF7F4FB002807D07F
:10C9C000101C03041B14074A11200121F9F73EFC37
:10C9D0000420FEF7E7FB002803D00420322100F0FA
:10C9E000E5FE00BDE028000070B50D1C061C01200E
:10C9F0000021F9F76FFCDA480078012805D1D94AFF
:10CA000014200221F9F722FC51E2D74800780228CD
:10CA10000FD1D6480078082805D1D54A1420022124
:10CA2000F9F714FC43E2D34A14200221F9F70EFC73
:10CA30003DE2CE480078082805D1CF4A14200221D3
:10CA4000F9F704FC33E2301C01280ED0032800D192
:10CA5000B5E0042800D1D9E1002800D027E2C74A78
:10CA600014200221F9F7F2FB21E2C548047804F012
:10CA7000DBFA0006000E0C2800D1002404F0D4FAE2
:10CA80000006000E042805D1201C0006000E032815
:10CA900000D10024201C01283AD002284DD00328C0
:10CAA00060D0042873D0002800D000E2B54A1420DA
:10CAB0000021F9F7CBFBAC480078012805D1B24A38
:10CAC0001E200221F9F7C2FBF1E104F0ADFA0028C3
:10CAD0000CD0042810D00C2814D0012800D0E6E196
:10CAE000AA4A1E200221F9F7B1FBE0E1A64A1E2066
:10CAF0000221F9F7ABFBDAE1A54A1E200221F9F782
:10CB0000A5FBD4E1A34A1E200221F9F79FFBCEE149
:10CB1000A14A14200021F9F799FBA04800780028C9
:10CB200005D09F4A22200221F9F790FBBFE19D4AE0
:10CB300022200221F9F78AFBB9E19B4A1420002147
:10CB4000F9F784FB95480078002805D0944A222004
:10CB50000221F9F77BFBAAE1924A22200221F9F790
:10CB600075FBA4E1914A14200021F9F76FFB8B4873
:10CB70000078002805D08E4A22200221F9F766FBB2
:10CB800095E1884A22200221F9F760FB8FE1894A6A
:10CB900014200021F9F75AFB80480078002808D0BB
:10CBA000012800D083E1844A1E200221F9F74EFBC0
:10CBB0007DE1824A1E200221F9F748FB77E1804897
:10CBC000047D007F00281ED07E4A14200021F9F742
:10CBD0003DFB7D480078012809D002280DD00028AF
:10CBE000FFD17A4A24200221F9F730FB5FE1784A2D
:10CBF00024200221F9F72AFB59E1764A2420022158
:10CC0000F9F724FB53E174480078012853D0022837
:10CC100000D195E0002800D049E1201C002844D034
:10CC2000012818D002282BD006283ED16B4A1420A8
:10CC30000021F9F70BFB6A480078002805D05E4A0E
:10CC40001E200221F9F702FB31E15C4A1E2002217D
:10CC5000F9F7FCFA2BE1634A14200021F9F7F6FA00
:10CC60005F480078002805D04D4A21200221F9F7BD
:10CC7000EDFA1CE14B4A21200221F9F7E7FA16E10F
:10CC8000594A14200021F9F7E1FA554800780028A4
:10CC900005D0434A21200221F9F7D8FA07E1414A99
:10CCA00021200221F9F7D2FA01E1504A1420022191
:10CCB000F9F7CCFAFBE0201C00283BD002280BD06F
:10CCC00003281ED0052822D0062833D1484A142034
:10CCD0000221F9F7BBFAEAE0434A14200021F9F7F0
:10CCE000B5FA3F480078002805D02D4A21200221BE
:10CCF000F9F7ACFADBE02B4A21200221F9F7A6FA7A
:10CD0000D5E03C4A14200221F9F7A0FACFE0012037
:10CD10000021F9F753FB384A14200021F9F796FA5D
:10CD2000364B142002213222F9F70CFB0021344843
:10CD30000170BCE0304A14200221F9F787FAB6E00E
:10CD4000201C062805D12F4A14200221F9F77EFA6B
:10CD5000ADE02D4A14200221F9F778FAA7E0C04689
:10CD6000D8210040DB280000E2210040D62100400D
:10CD7000D4280000CD280000BC280000B228000004
:10CD8000E3210040AE280000A72800009E280000F4
:10CD9000972800009028000084280000E42100402B
:10CDA0007E280000782800006B2800006128000021
:10CDB0005A28000052280000492800003E280000A0
:10CDC000D22100402D280000E82100402B2800003F
:10CDD0002628000021280000E52100401728000037
:10CDE000E721004009280000FB270000E927000098
:10CDF000D4270000C0270000AE27000099270000BC
:10CE0000E621004085270000742700002848047EA2
:10CE1000007F002800D00024281C012816D00228FA
:10CE20002AD003283ED0002841D1201C0006000E45
:10CE3000012805D11F4A14200221F9F707FA36E02C
:10CE40001D4A14200221F9F701FA30E01B4A142090
:10CE50000021F9F7FBF9201C0006000E012805D17E
:10CE6000174A1B200221F9F7F1F920E0154A1B208F
:10CE70000221F9F7EBF91AE0104A14200021F9F722
:10CE8000E5F9201C0006000E012805D10C4A1B20E4
:10CE90000221F9F7DBF90AE00B4A1B200221F9F71E
:10CEA000D5F904E0094A14200221F9F7CFF970BD41
:10CEB000D221004065270000612700005A270000AA
:10CEC0004F270000462700003F27000035270000BD
:10CED00000B53220F8F7F4FD07480021F8F7D8F83C
:10CEE0003220F8F7EDFD04480121F8F7D1F896203B
:10CEF000F8F7E6FD00BDC0460008000030B5051C8F
:10CF0000281C0078042831D0092847D00B2853D09A
:10CF10000F2800D19AE0102814D011281CD0122814
:10CF200071D0012800D0D5E0281C4478201C0006D0
:10CF3000000EF9F799FC201C0006000E03F050F8D3
:10CF40000120C8E0281C4078002802D000F0A6FD8F
:10CF5000C0E000F001FEBDE000F004FB002800D1BD
:10CF6000B8E0281C407800F01BFDB3E000F0FAFAAE
:10CF7000002800D1AEE0281C407858498873281C4E
:10CF80008078C8730120FEF70DF9002800D1A1E0D8
:10CF90005249887BC97BFFF727FD9BE000F0E2FA4E
:10CFA000002800D196E00120FEF7FCF8002800D10F
:10CFB00090E000F05FFC8DE000F0D4FA002800D192
:10CFC00088E0281C4078002806D002280FD1281CB1
:10CFD0008178434801700AE04148017801310170CD
:10CFE0003F480078032802DD00213D4801703C489D
:10CFF0000078F8F78DFF3A480078011C02200022E3
:10D00000F9F718FD66E000F0ADFA002862D0281CA0
:10D01000407802280DD003280FD13248007801282B
:10D0200003D100212F48017007E001212D48017034
:10D0300003E0281C81782B4801702A48007800F012
:10D04000FDFC0120002100F0D5F843E000F08AFA51
:10D0500000283FD0281C407801280ED0022818D084
:10D0600000282BD12048018809040914081C0F2826
:10D0700024DA01311C48018020E01B4801880904A2
:10D080000914081C5A22D04218DD013916480180C3
:10D0900014E0281C8078041C2402281CC078044357
:10D0A0002404240C201C0004001400F04BFA000699
:10D0B000000E012802D1211C0B4801800A4800887B
:10D0C00000040014F7F76CFF074800880004001400
:10D0D000FFF76AFC002030BC08BC1847D221004092
:10D0E000DF210040D8210040D421004000B5021CBF
:10D0F0000520FEF757F80006000E002801D1002099
:10D1000009E0101C054909780A1C92000449895855
:10D11000496807F04EFF08BC1847C0469F220040F0
:10D120008821004000B5011C081C0078012805D1A9
:10D13000081C4078622801D102F098FA002008BC4F
:10D140001847C04630B50D1C041C82B00D4900A81C
:10D1500008220B780370491C401C521EF9D10B2188
:10D1600000A80170291C012068440170211C0220C4
:10D170006844017000A90120FDF79AFF0006000E27
:10D1800002B030BD94290000F0B5141C0E1C051C23
:10D1900082B0154F154900A808220B780370491C6E
:10D1A000401C521EF9D13878002816D000211048B2
:10D1B0000170012100A80170211C01206844017048
:10D1C000311C022068440170281C0006000E00A9D2
:10D1D000FDF76EFF0006000E03E0211C04480170FD
:10D1E000002002B0F0BDC0467C0500409C29000034
:10D1F0008522004030B50D1C041C82B00C4900A8EB
:10D2000008220B780370491C401C521EF9D10921D9
:10D2100000A80170291C012068440170201C000630
:10D22000000E00A9FDF744FF0006000E02B030BD5D
:10D230008C29000070B5151C0E1C041C82B0174907
:10D2400000A808220B780370491C401C521EF9D11B
:10D250000F2100A80170311C012068440170281CB6
:10D26000010409140912FF2001400906090E0220D9
:10D2700068440170281C01040914FF2001400906BC
:10D28000090E032068440170201C0006000E00A94E
:10D29000FDF70EFF0006000E02B070BDA4290000CD
:10D2A00070B5141C0D1C061C82B0104900A8082281
:10D2B0000B780370491C401C521EF9D10A2100A8AA
:10D2C0000170311C012068440170291C022068444F
:10D2D0000170211C03206844017000A90320FDF7A0
:10D2E000E7FE0006000E02B070BDC046AC2900008B
:10D2F00030B50D1C041C82B00C4900A808220B7824
:10D300000370491C401C521EF9D1102100A8017065
:10D31000291C012068440170201C0006000E00A991
:10D32000FDF7C6FE0006000E02B030BD84290000E5
:10D3300030B50D1C041C82B00C4900A808220B78E3
:10D340000370491C401C521EF9D1112100A8017024
:10D35000291C012068440170201C0006000E00A951
:10D36000FDF7A6FE0006000E02B030BD7C290000CD
:10D3700070B5151C0E1C041C82B00F4900A80822B1
:10D380000B780370491C401C521EF9D1122100A8D1
:10D390000170311C012068440170291C022068447E
:10D3A0000170201C0006000E00A9FDF781FE00069A
:10D3B000000E02B070BDC0467429000010B50120F7
:10D3C000F6F72EFC0020F6F73BFC1248F8F778FB46
:10D3D000F8F76EF8FFF77CFD0F480078002802D1BF
:10D3E00001210D48017001200C4C2070F6F762F904
:10D3F000F6F72EF800F00EFB607BF8F789FD0021B0
:10D40000074801700748F8F75BFB012104480170E9
:10D4100010BDC046F4010000DF210040D2210040D1
:10D420007C0500408813000030B502200021F8F789
:10D4300051FF104C104A08200321F8F707FF0F484E
:10D44000F8F73EFB0E4A08200321F8F7FFFE002004
:10D45000F6F7E6FB0120F6F7F3FB00250948057017
:10D46000F8F71EF825700848F8F72AFB012020700D
:10D4700030BDC0467C05004028270000F4010000B4
:10D4800022270000D221004088130000021C101C3B
:10D49000012811D0022811D0032811D0042811D05E
:10D4A000052811D0062811D0072811D0082811D03E
:10D4B000002810D109490EE009490CE009490AE0A9
:10D4C000094908E0094906E0094904E0094902E080
:10D4D000094900E00949081C7047C046092200407C
:10D4E0001622004023220040302200403D2200400E
:10D4F0004A2200405722004064220040FC210040A4
:10D5000000B500200E49487001224A7188734874A2
:10D510008874087608750020F8F750FD011C081C77
:10D520000006000E542807D000205421F8F730FDE3
:10D530000020FAF7A5FB02E00120FAF70DFB00BD81
:10D54000D2210040011C081C000400140F2807DC35
:10D55000081C000400145A21C84201DB012000E02D
:10D560000020704703480078012801D1012000E025
:10D5700000207047D3210040F0B5171C0E1C051C7D
:10D5800082B0002174480170281C00A90870311C69
:10D590000C06240E01342406240E0006000E082872
:10D5A00003D1002100A80170022402200021F8F715
:10D5B00091FE6A48008800040014031C684A002099
:10D5C0000121F8F743FE002101A801705FE000AAE5
:10D5D0001078092107F0F4FC011C11701078002864
:10D5E00002D0082806D10324201C0006000E0128C2
:10D5F00000D102243DE001200021F8F76BFE201C41
:10D600000106090E89005748405801B401A8007866
:10D61000011C890054484358544A14200221F8F749
:10D6200015FE01B000A80078211C0906090EF6F7C6
:10D63000D1F900280BD000A80078211C0906090E9A
:10D6400002F05CFA012144480170012082E0484860
:10D6500000781D2801D0042805D101200021FFF702
:10D6600047FE002076E06420F8F72AFA0134240609
:10D67000240E201C0006000E0328BCDD012401A896
:10D6800001780131017000A801780131017001A811
:10D69000007809289BDB281C08284FD0002805D1DA
:10D6A000201C0006000E012800D1022401243DE0C8
:10D6B00001200021F8F70EFE201C0106090E89004A
:10D6C0002848405801B401A80078011C8900264868
:10D6D0004358264A14200221F8F7B8FD01B000A8EB
:10D6E0000078211C0906090EF6F774F900280BD002
:10D6F00000A80078211C0906090E02F0FFF901219B
:10D7000015480170012025E0194800781D2801D036
:10D71000042805D101200021FFF7EAFD002019E0CF
:10D720006420F8F7CDF901342406240E301C0106DC
:10D73000090E201C0006000E8842B9D9381C0028AA
:10D7400000D040E701210448017001200021FFF7CB
:10D7500051FD002002B0F0BD7C050040D421004006
:10D76000BA250000C0210040E01F0040B4250000A1
:10D770008522004000B5011C081C002804D00121AE
:10D78000081CF8F705FC03E001200021F8F700FC75
:10D7900000BDC04600B50120F8F710FC0006000EE1
:10D7A000012801D1012000E0002000BD10B40A1CB6
:10D7B000041C231C0348011C94310B70111C0180B4
:10D7C00010BC7047F221004000C09FE51CFF2FE114
:10D7D000D5D7000000B50B480188090409140029B9
:10D7E0000DD0084801390180064800880004001463
:10D7F000002804D1044800780021FFF7FBFC08BC96
:10D800001847C046F22100408622004010B532245D
:10D8100000211248017002200021F8F75BFD104A38
:10D8200001200021F8F712FD0E4801B40E4A0F4BFB
:10D8300014200321F8F70AFD01B06420F8F740F93D
:10D840000B480078002805D1201C013C2404241436
:10D850000028F2D101210148017010BD7C05004073
:10D8600077040000E4280000F7280000F0280000FA
:10D870008522004010B50021081CF8F72BFD094C4B
:10D88000094A0A4803680021081CF8F7DFFC608891
:10D8900000040014FFF788F8A07BE17BFFF7A4F8F1
:10D8A00010BDC046D22100402E27000004200040B9
:10D8B00030B5051C0024281C0006000E082819D1CC
:10D8C000281C0106090E3248405C00280AD00120BD
:10D8D000F7F738FD0320FDF77FFB0220F6F712F87B
:10D8E000012403E00120F6F70DF80224201C0006B5
:10D8F000000E4BE00120F5F799FD281C0006000EF4
:10D90000F6F72AF8011C081C0006000E002806D1B4
:10D910000121281C0006000E002800D102210A1C4B
:10D920001C480270081C0006000E032822D1281C87
:10D930000106090E1848405C011C49001748405A6E
:10D940000004001407F0DAF8F7F724FB281C01069E
:10D95000090E0F48405C002807D00220FDF73CFB71
:10D960000220F5F7CFFF01240AE00020F5F7CAFFF7
:10D97000022405E00120FDF72FFB0220F5F7C2FF8E
:10D980000020F5F753FD201C0006000E30BDC046F8
:10D99000971D0040D72100408D1D0040401700001A
:10D9A00010B5021C0023101C01280FD002280DD036
:10D9B00003280BD0042809D0052807D0062805D055
:10D9C000072803D0082801D0002803D1111C0E48D5
:10D9D000017001230C480078FFF758FD0B490860DF
:10D9E000181C00280BD00A4C2079FFF761FF207427
:10D9F0000020A0732079011C2220F8F7C9FA012029
:10DA00000021FFF7F7FB10BDD621004004200040A5
:10DA1000D221004000B502200021F8F75BFC054A46
:10DA200001200021F8F712FC034A14200321F8F723
:10DA30000DFC00BD71220040E002000010B5041C86
:10DA40000F48007800280BD00120F6F709F90120D3
:10DA5000F6F726F9201C0006000EF6F711F90EE085
:10DA6000201C0006000EF6F7FBF8201C0006000E36
:10DA7000F6F716F9201C0006000EF6F701F910BDA6
:10DA8000EE21004000B50520F8F798FA0006000ED8
:10DA9000002801D1012000E0002000BD00B5284889
:10DAA0000078002801D1FFF789FC2648007801287A
:10DAB00042D0254925480180FFF76CFE002818D088
:10DAC00023480078F5F748FF0006000E002809D12A
:10DAD000FFF7D8FF002805D0082003210122FFF717
:10DAE0004BFD12E01A480078011C0120FFF720FCD2
:10DAF0000BE0082003210122FFF73EFD0006000E87
:10DB000001281CD10120FFF735FE104800880004D1
:10DB10000014021C01200221FFF78CFB01200221CE
:10DB20000022FFF725FC0B480078002801D00228CE
:10DB300002D10120F5F770FF01210248017000BDFC
:10DB4000D2210040D3210040E2FF0000D421004058
:10DB5000D6210040A11D004000B5174800780028DC
:10DB600012D002200321F8F7B5FB0020FDF734FAAC
:10DB70000120FFF763FF11480078002801D0022838
:10DB800002D10020F5F748FF0D480078012802D0A7
:10DB9000FFF74AFC0BE00B4A00200321F8F756FB85
:10DBA0000948F7F78DFF02200021FFF723FB002132
:10DBB0000148017000BDC046D3210040A11D0040B6
:10DBC000D92100400D270000E803000010B5041C17
:10DBD000201C0078082813D001285ED1201C407832
:10DBE00032280AD0382801D00D2856D12D48007887
:10DBF000011C012001F044FA4FE001F075FA4CE0FD
:10DC0000201C4078012817D0032835D0002844D1A3
:10DC100001212548417081700078011C890023484A
:10DC2000405802680021081CF8F710FB204A142015
:10DC30000321F8F70BFB30E01E480078002801D1E3
:10DC400000202BE017480078022810D0012824D1AA
:10DC5000144C194A0021081CF8F7F8FA144A142049
:10DC60000321F8F7F3FA20780130207015E0032043
:10DC7000002101F005FA10E000210B484170017805
:10DC8000013101700078011C8900084840580028C3
:10DC900003D00021081C01F0F3F9012010BC08BCDE
:10DCA0001847C046A12200409F2200408821004022
:10DCB000C9290000A0220040F329000030B5041C4F
:10DCC000201C0078082835D0012800D070E1201CE5
:10DCD000407832282BD0382802D00D2800D067E1B8
:10DCE000B5480078002800D162E1B44800780028E7
:10DCF00004D00320002101F0C3F959E100250EE012
:10DD000001F04AFAAE48F7F7DBFE02200321F8F7EC
:10DD1000E1FAC820F7F7D4FE01352D062D0E281C98
:10DD20000006000E0328EBDB01F0DEF940E101F014
:10DD3000DBF93DE1201C407801283BD0022874D05B
:10DD4000032800D121E1002800D031E10120F5F7BE
:10DD500049FF9C48F7F76CF90020F5F791FB01218A
:10DD6000994801700021081CFDF768F90220F5F7B9
:10DD7000C9FD01219548017000218F4801708F482D
:10DD8000017093480078011C89009248405802684D
:10DD900000200121F8F75AFA01200221F8F79AFA37
:10DDA00001F0C8F900218C4801700021012001F028
:10DDB00067F9FDE085480078002801D10020F8E0EF
:10DDC000201C81788448017083480078011C8900F8
:10DDD00082484058C06A406806F0DCFF0106090E20
:10DDE0007F48017001200021F8F774FA7A48007822
:10DDF000011C890079484058C06A426814200021FB
:10DE0000F8F724FA74480078011C890073484058D8
:10DE1000C06A4078011C0120FDF710F96E480078B7
:10DE2000011C022001F02CF9C2E0684800780028AB
:10DE300001D10020BDE002F07DFF012800D08DE07F
:10DE4000022002F09FFF051C63480078011C890036
:10DE500062484058C06A4078011C281C08400028CD
:10DE60000DD0604A25200221F8F7F0F900215A4828
:10DE70000078021C920059488058017049E04F48D0
:10DE8000017801310170584A25200221F8F7DEF9A6
:10DE9000012151480078021C9200504880580170BE
:10DEA00002F052FF06F080F84B490A78141CA400D7
:10DEB0004A490B599860D86A0078052806D14B4921
:10DEC0000833186805F0F4FE186008E0484992002D
:10DED000424882580832106805F0EAFE10603E4859
:10DEE0000078011C89003D4843589868414A111C3C
:10DEF00007F048F800D99A601A2002F02FFF051C9D
:10DF00000006000E344909780A1C920033498958EA
:10DF100048703948F7F7D4FD2F4801780131017076
:10DF20002D480078021C92002C498958002904D001
:10DF3000011C012001F0A4F83AE001211E48017003
:10DF40001E480078031C2D4A0021081CF8F77EF9B2
:10DF50002B4A14200321F8F779F929E01E480078AC
:10DF6000011C022001F08CF81D480078112808DA05
:10DF70001430244A0221F8F769F91948017801316F
:10DF800001700F48F7F79CFD12E000210F48017067
:10DF90000F480178013101700D480078011C89009B
:10DFA0000C484058002803D00021081C01F068F8F4
:10DFB000012030BC08BC1847A3220040A422004026
:10DFC0002C010000ECFFFFFF84220040A222004051
:10DFD0009F220040882100409D220040981F004061
:10DFE0009E220040D9260000D526000033C4B13C53
:10DFF0005AF5B93C0000C84220030000BE260000CC
:10E00000DE290000E126000010B5041C201C007869
:10E01000082813D0012800D0CDE0201C40783228F9
:10E0200009D0382802D00D2800D0C4E003200021F8
:10E0300001F026F8BFE001F057F8BCE0201C407862
:10E04000012821D002284AD0032800D1A0E00028CE
:10E0500000D0B0E001215A4801705A480078011CF4
:10E06000890059484058026800200121F8F7EEF86D
:10E0700001200221F8F72EF90021544801700021F7
:10E08000012000F0FDFF96E04D480078002801D106
:10E09000002091E04D480078011C89004C48405810
:10E0A000C06A406806F076FE0106090E4948017014
:10E0B00001200021F8F70EF944480078011C89007E
:10E0C00043484058C06A426814200021F8F7BEF85F
:10E0D0003E480078011C022000F0D2FF6BE0384877
:10E0E0000078002801D1002066E038480078031C41
:10E0F0009B003748C058002834D0017800292AD026
:10E1000082683549101C05F087FE041C33483449E9
:10E11000231C05F0DFFC314806F03CFE0406240E0B
:10E120000AE02C48007814302E4A0021F8F78EF8C7
:10E130002848017801310170201C0006000E1421CE
:10E14000091A244800788842EBDB1430234A022164
:10E15000F8F77CF803E01F48007801F02DF822481A
:10E16000F7F7AEFC194801780131017017480078C3
:10E17000021C920016498958002904D0011C012074
:10E1800000F07EFF17E00320002100F079FF12E08D
:10E1900000210B4801700B480178013101700948DA
:10E1A0000078011C890008484058002803D000214D
:10E1B000081C00F065FF012010BC08BC1847C046D1
:10E1C000A52200409F220040882100409D2200405F
:10E1D000981F00409E220040333353408822004065
:10E1E000AF260000E1260000E803000030B5041C63
:10E1F000201C007808280AD0012800D042E1201C09
:10E200004078322800D03DE100F06EFF3AE1201C5A
:10E210004078012821D0022876D0032800D11EE1C1
:10E22000002800D02EE1012198480170984800781C
:10E23000011C890097484058026800200121F8F726
:10E2400005F801200221F8F745F8002192480170F5
:10E250000021012000F014FF14E18C480078002810
:10E2600001D100200FE18C480078011C89008B4807
:10E270004058C06A406806F08DFD0106090E8848C6
:10E28000017001200021F8F725F883480078011C6F
:10E29000890082484058C06A426814200021F7F77C
:10E2A000D5FF7D480078021C92007C488058017898
:10E2B00000290CD0C06A4078011C0320FCF7BEFE88
:10E2C00075480078011C022000F0DAFEDAE074489C
:10E2D000007800F071FF7348F7F7F2FB6E480178A1
:10E2E000013101706C480078021C92006B4989581A
:10E2F000002904D0011C012000F0C2FEC2E003206E
:10E30000002100F0BDFEBDE060480078002801D18A
:10E310000020B8E002F00EFD012800D088E05E4841
:10E320000078011C89005D484058C06A007800F000
:10E3300063FF0106090E58480078021C92005748F6
:10E34000805828300170192002F008FD011C081CBB
:10E3500002F02AFE504909780A1C92004F49895858
:10E360004860486800F06EFE4B4909780D1CAD000E
:10E370004A494A595060D06A0078052808D1506847
:10E38000494905F095FC494905F030FC506004E02E
:10E390005068474905F08CFC50605068454B191C8B
:10E3A00006F0F0FD00D953605068434B191C06F08D
:10E3B000E9FD00D2536052684048414905F08AFBAC
:10E3C0003E4806F0E7FC0406240E0AE034480078D4
:10E3D00014303C4A0021F7F739FF31480178013108
:10E3E0000170201C0006000E1421091A2C48007828
:10E3F0008842EBDB1430314A0221F7F727FF294826
:10E40000F7F75EFB2448017801310170224800785B
:10E41000021C920021498958002904D0011C0120C6
:10E4200000F02EFE2EE00320002100F029FE29E05E
:10E4300019480078011C022000F022FE18480078DC
:10E440000C2808DA14301F4A0221F7F7FFFE14489F
:10E450000178013101701C48F7F732FB12E000210E
:10E460000A4801700A4801780131017008480078B3
:10E47000011C890007484058002803D00021081CCF
:10E4800000F0FEFD012030BC08BC1847A622004069
:10E490009F220040882100409D220040981F00409C
:10E4A0009E220040E8030000000040BF0000404101
:10E4B0000000E0BF00007041000070C188220040F1
:10E4C000A7260000E1260000BC02000010B5041CD5
:10E4D000201C0078082813D0012800D0EEE0201C72
:10E4E0004078322809D0382802D00D2800D0E5E045
:10E4F0000320002100F0C4FDE0E000F0F5FDDDE0C8
:10E50000201C407801281FD002286FD0032800D19A
:10E51000C3E0002800D0D1E001206A4CA072A078AE
:10E52000011C890068484058026800200121F7F763
:10E530008DFE01200221F7F7CDFE00202070002182
:10E54000012000F09DFDB9E060480078002801D16D
:10E550000020B4E05B4C2078011C89005C484058E6
:10E56000C06A406806F016FC0006000E60700120CC
:10E570000021F7F7AFFE2078011C8900544840586D
:10E58000C06A426814200021F7F760FE2078021C60
:10E5900092004F488058017800290CD0494CC06A3D
:10E5A0004078011C0320FCF749FD2078011C022063
:10E5B00000F066FD82E0434C607800F0FDFD4548C8
:10E5C000F7F77EFA2078013020702078021C920044
:10E5D0003F498958002904D0011C012000F050FD5A
:10E5E0006CE00320002100F04BFD67E03748007825
:10E5F000002801D1002062E002F09CFB012836D106
:10E60000304C2078011C890031484058C06A00789D
:10E6100000F0F2FD0206120E2078031C9B002C482D
:10E62000C058011C2A310A70283000F0EBFE011C92
:10E63000081C03061B0E284A23200221F7F706FEBA
:10E640002448F7F73DFA2078013020702078021C2A
:10E6500092001F498958002904D0011C012000F0B4
:10E660000FFD2BE00320002100F00AFD26E0154CF1
:10E670002078011C022000F003FD60780F2808DAE2
:10E680001430164A0221F7F7E1FD154801780131EF
:10E6900001701448F7F714FA10E0002112480172D3
:10E6A0000178013101700078011C8900064840584A
:10E6B000002803D00021081C00F0E2FC012010BC5F
:10E6C00008BC18479D22004088210040A722004036
:10E6D000981F0040E8030000A1260000E12600008A
:10E6E0009E220040BC0200009F22004030B5041C66
:10E6F000201C0078082813D0012800D02AE1201C13
:10E700004078322809D0382802D00D2800D021E1E5
:10E710000320002100F0B4FC1CE100F0E5FC19E14D
:10E72000201C4078012821D0022876D0032800D16F
:10E73000FDE0002800D00DE10121884801708848E3
:10E740000078011C89008748405802680020012198
:10E75000F7F77CFD01200221F7F7BCFD002182487C
:10E7600001700021012000F08BFCF3E07B48007871
:10E77000002801D10020EEE07B480078011C8900D0
:10E780007A484058C06A406806F004FB0106090E4A
:10E790007748017001200021F7F79CFD724800784E
:10E7A000011C890071484058C06A42681420002149
:10E7B000F7F74CFD6C480078021C92006B488058BB
:10E7C000017800290CD0C06A4078011C0320FCF7B6
:10E7D00035FC65480078011C022000F051FCB9E0CE
:10E7E0006348007800F0E8FC6248F7F769F95E4892
:10E7F0000178013101705C480078021C92005B498D
:10E800008958002904D0011C012000F039FCA1E046
:10E810000320002100F034FC9CE0504800780028E0
:10E8200001D1002097E002F085FA012868D14E4816
:10E830000078011C89004D484058C06A007800F0FB
:10E84000DBFC0106090E48480078051CAD0047486E
:10E850004259101C29300170474B141C0C3420689D
:10E86000191C05F0D9FA206010321068191C05F047
:10E87000D3FA106040493C480078021C92003B48A3
:10E880008258131C1433186805F0C6FA18603A4908
:10E89000131C1833186805F0BFFA18603649131CAA
:10E8A0001C33186805F0B8FA18603349131C20337C
:10E8B000186805F0B1FA18602F492432106805F085
:10E8C000ABFA10602D4A25200221F7F7BFFC29483A
:10E8D000F7F7F6F8244801780131017022480078F2
:10E8E000021C920021498958002904D0011C0120F2
:10E8F00000F0C6FB2EE00320002100F0C1FB29E060
:10E9000019480078011C022000F0BAFB1848007872
:10E91000112808DA14301A4A0221F7F797FC144834
:10E920000178013101701748F7F7CAF812E00021A9
:10E930000A4801700A4801780131017008480078DE
:10E94000011C890007484058002803D00021081CFA
:10E9500000F096FB012030BC08BC1847A8220040FC
:10E960009F220040882100409D220040981F0040C7
:10E970009E220040E8030000000040409D26000069
:10E98000E1260000BC02000030B5051C281C007800
:10E99000082800D14FE2012800D03EE3281C40782F
:10E9A000322800D144E2382802D00D2800D034E3C8
:10E9B0009148007802280AD0012800D02DE30121D7
:10E9C0008E4801700021081C00F05AFB25E300244A
:10E9D00004E1201C03061B0E9B008948C058C16A35
:10E9E0000A7801780220F8F70DFA201C03061B0EA6
:10E9F0009B008348C258906805F000FB0106090E91
:10EA0000D06A02780220F8F739FA201C0106090EB4
:10EA100089007B484058406800F04AFD0106090E15
:10EA2000201C0206120E920075488058C06A0278B7
:10EA30000220F8F7EBFA201C0106090E8900704845
:10EA400040582930007800F01BFD0106090E201CFB
:10EA50000206120E92006A488058C06A02780220AC
:10EA6000F8F70AFB201C0206120E92006448805838
:10EA7000C16A0978052900D1ADE0C06806F074FAD2
:10EA800000F016FD0106090E201C0206120E92006F
:10EA90005B488058C06A02780220F8F755FB201CBA
:10EAA0000106090E890056484058006906F05CFAD4
:10EAB00000F0FEFC0106090E201C0206120E920058
:10EAC0004F488058C06A0278102002430220F8F7AD
:10EAD0003BFB201C0106090E89004948405840694B
:10EAE00006F042FA00F0E4FC0106090E201C0206C2
:10EAF000120E920042488058C06A027820200243D9
:10EB00000220F8F721FB201C0106090E89003C4871
:10EB10004058806906F028FA00F0CAFC0106090E88
:10EB2000201C0206120E920035488058C06A0278F6
:10EB3000302002430220F8F707FB201C0106090ED3
:10EB400089002F484058C06906F00EFA00F0B0FC6A
:10EB50000106090E201C0206120E92002848805859
:10EB6000C06A0278402002430220F8F7EDFA201C28
:10EB70000106090E890022484058006A06F0F4F99F
:10EB800000F096FC0106090E201C0206120E9200EF
:10EB90001B488058C06A0278502002430220F8F7D0
:10EBA000D3FA201C0106090E890015484058406A16
:10EBB00006F0DAF900F07CFC0106090E201C0206C2
:10EBC000120E92000E488058C06A027860200243FC
:10EBD0000220F8F7B9FA01342406240E201C01069D
:10EBE000090E890006484058002800D0F1E60024AC
:10EBF000044804700DE1C046AA2200409F22004054
:10EC0000981F0040C4240040201C03061B0E9B00DC
:10EC1000DC48C058C16A0A7801780020F8F7F2F899
:10EC2000201C03061B0E9B00D648C258906805F0B6
:10EC3000E5F90106090ED06A02780020F8F71EF9FE
:10EC4000201C0106090E8900CE484058406800F09B
:10EC50002FFC0106090E201C0206120E9200C94864
:10EC60008058C06A02780020F8F7D0F9201C01060D
:10EC7000090E8900C34840582930007800F000FC94
:10EC80000106090E201C0206120E9200BD48805893
:10EC9000C06A02780020F8F7EFF9201C0206120E75
:10ECA0009200B8488058C16A0978052900D1ADE0C2
:10ECB000C06806F059F900F0FBFB0106090E201CA4
:10ECC0000206120E9200AF488058C06A02780020F7
:10ECD000F8F73AFA201C0106090E8900A9484058A5
:10ECE000006906F041F900F0E3FB0106090E201C63
:10ECF0000206120E9200A3488058C06A02781020C3
:10ED000002430020F8F720FA201C0106090E8900B2
:10ED10009C484058406906F027F900F0C9FB0106FD
:10ED2000090E201C0206120E920096488058C06AF6
:10ED30000278202002430020F8F706FA201C010682
:10ED4000090E89008F484058806906F00DF900F0DF
:10ED5000AFFB0106090E201C0206120E9200894824
:10ED60008058C06A0278302002430020F8F7ECF99E
:10ED7000201C0106090E890082484058C06906F02F
:10ED8000F3F800F095FB0106090E201C0206120E96
:10ED900092007C488058C06A0278402002430020DC
:10EDA000F8F7D2F9201C0106090E89007548405871
:10EDB000006A06F0D9F800F07BFB0106090E201C62
:10EDC0000206120E92006F488058C06A02785020E6
:10EDD00002430020F8F7B8F9201C0106090E89004B
:10EDE00068484058406A06F0BFF800F061FB010631
:10EDF000090E201C0206120E920062488058C06A5A
:10EE00000278602002430020F8F79EF901342406BE
:10EE1000240E201C0106090E89005A48405800287B
:10EE200000D0F1E601215848017000F05DF9F4E0EE
:10EE300000F05AF9F1E0281C4078012822D002287D
:10EE400048D0032800D1CCE0002800D0E5E0012024
:10EE50004E4D287300206873A878011C89004C4827
:10EE60004058026800200121F7F7F0F90120022143
:10EE7000F7F730FA0020A87328700021012000F075
:10EE8000FFF8CAE043480078002801D10020C5E01F
:10EE90003E4D2878011C89003A484058C06A4068B5
:10EEA00005F078FF0006000E687001200021F7F7DA
:10EEB00011FA2878011C890032484058C06A42681B
:10EEC00014200021F7F7C2F92878011C022000F075
:10EED000D7F8A2E02F480078002801D100209DE05B
:10EEE0002A480078021C920026488058002839D011
:10EEF000017800292FD04078002807D0012126482A
:10EF000001702648264904F0E5FD03E02348254921
:10EF100004F0E0FD214805F03DFF0406240E0BE05F
:10EF20001A4D68781430204A0021F7F78FF9281C11
:10EF30000130017801310170201C0006000E1421FF
:10EF4000091A1A4800788842EADB1430134A022171
:10EF5000F7F77CF903E01548007800F02DF9144824
:10EF6000F6F7AEFD09480178013101700078021C06
:10EF700092000449895800291CD0011C012000F08E
:10EF80007FF84AE0981F0040C42400409D220040C2
:10EF900088210040A9220040AB2200408822004086
:10EFA000932600008A260000E12600009E220040F1
:10EFB000E80300001B48007800280DD001211A4802
:10EFC00001701A4A0021081CF7F740F9184A14206A
:10EFD0000321F7F73BF920E00320002100F050F86F
:10EFE0001BE00021134881720078011C890012483F
:10EFF0004058002804D00021081C00F041F80CE023
:10F000000221094801700D4A0021081CF7F71EF97A
:10F010000B4A14200321F7F719F9012030BC08BC72
:10F020001847C046AB220040AA22004075260000C7
:10F03000602600009F2200408C2100404B260000EB
:10F040003626000000B5021C0C4B101C191C04F0E5
:10F050002FFE04F0D3FF021C101C052105F0D4FF85
:10F06000081C021C000400140521484305F046FD5D
:10F07000021C191C04F0D0FE021C00BD000020413F
:10F0800030B50C1C051C82B00D4900A808220B7875
:10F090000370491C401C521EF9D1082100A80170C0
:10F0A000291C012068440170211C02206844017061
:10F0B00000A90520FBF7FCFF0006000E02B030BDE2
:10F0C000882A000000B5FCF78BF8064B1870052065
:10F0D000FCF776F8002018760021081CFFF7D0FF17
:10F0E00000BDC0468722004010B50021104C201CF6
:10F0F000B2300170201CB5300078FCF761F80220B6
:10F100000021F7F7E7F8201CB53000780021FEF762
:10F1100071F80020F4F766FD2079011C0120FEF74C
:10F1200007F9608800040014F5F73AFF10BDC046E7
:10F13000D221004030B4002021E00021021C15063D
:10F140002D0EAD00134A5259516000231370002355
:10F150005370516091600024131C28331C700024EC
:10F16000131C29331C700024131C2A331C70D1601B
:10F17000116151619161D16101300006000E011CE5
:10F180000A06120E9200034989580029D5D130BCD5
:10F190007047C046981F004000B5054A0021081C72
:10F1A000F7F754F8034A14200321F7F74FF800BD8E
:10F1B000F8260000E326000010B5041C0AE0201C1D
:10F1C0000006000E14300A4A0021F7F73FF8013418
:10F1D0002406240E201C0006000E1128EFDB201C44
:10F1E0000006000E1430034A0221F7F72FF810BD75
:10F1F000E1260000DD260000F0B5041C7B488544B4
:10F2000000200190002712E0381C00040014203078
:10F2100001F0A4FD0190019801F0C6FE391C0A041A
:10F220001214920002A9885001373F043F14381C81
:10F23000000400147928E7DB201C0006000E0528D6
:10F2400029D12127239804F0DBFB009021251CE025
:10F25000381C01040914890002A8405804F0D0FBAE
:10F26000061C002803D13D1C2D062D0E12E0009C2B
:10F27000301C211C05F086FE04D2301C00903D1C81
:10F280002D062D0E013F3F043F14381C00040014CE
:10F290000028DDDA2BE00027029804F0B1FB009093
:10F2A00000251FE0381C01040914890002A84058F9
:10F2B0004F4904F053FC04F0A3FB061C002803D1C3
:10F2C0003D1C2D062D0E12E0009C301C211C05F06B
:10F2D00059FE04D2301C00903D1C2D062D0E013726
:10F2E0003F043F14381C000400142228DADB414894
:10F2F0000078031C9B004048C258D06A007805285B
:10F3000035D106990C32106804F028FC10600E9973
:10F3100038480078021C920037488258131C10337A
:10F32000186804F01BFC18601299131C1433186839
:10F3300004F014FC18601699131C1833186804F0B4
:10F340000DFC18601A99131C1C33186804F006FC95
:10F3500018601E99131C2033186804F0FFFB186016
:10F3600022992432106804F0F9FB106035E01A99F4
:10F3700020480078021C92001F488258131C0C334E
:10F38000186804F0EBFB18602E99131C10331868F2
:10F3900004F0E4FB18604299131C1433186804F05D
:10F3A000DDFB18605699131C1833186804F0D6FB5F
:10F3B00018606A99131C1C33186804F0CFFB18609E
:10F3C0007299131C2033186804F0C8FB18607699F2
:10F3D0002432106804F0C2FB1060281C0106090EDC
:10F3E00049000648405A06498D44F0BDA0FDFFFF84
:10F3F000000040409D220040981F0040D82300009C
:10F400006002000070B4011C002230E0101C0306F2
:10F410001B0E081CC45C101C03061B0E01331B06CC
:10F420001B0E1CE0181C05062D0E081C455D2E1C2D
:10F43000201C0006000EB0420ED2101C0606360E2E
:10F44000081C8555181C05062D0E081C4455101C5B
:10F450000406240E081C045D01331B061B0E181C39
:10F460000006000E0328DDDB01321206120E101C0E
:10F470000006000E0328C9DB081C407870BC7047EA
:10F4800000B5011C081C04F08FFD021C0649101C6D
:10F4900004F0C2FC054904F0A9FB021C04F0AEFD17
:10F4A0000006000E00BDC0460000204100000040E4
:10F4B00010B5021C101C1D4B191C04F0F9FB021C9A
:10F4C00004F09CFD05F01AFB021C191C04F0A4FCBE
:10F4D000021C002311E0181C0106090E89001448C3
:10F4E0004458101C211C05F04DFD03D1181C0006CA
:10F4F000000E1AE001331B061B0E181C0006000E3E
:10F500003D28E8DB0A480468101C211C05F03AFD80
:10F5100001D2002009E007480468101C211C05F0F6
:10F5200031FD01D23C2000E01E2010BD0000004053
:10F5300004060000F406000010B581B041480068E0
:10F54000F6F77CFD002872D13E48006800A9F6F766
:10F55000D3FD14213C4801803C480078012819D093
:10F56000002864D13A48018809023948018000A87E
:10F570000078021C36480188114301803448008815
:10F580003449884253D1012130480170002132486A
:10F5900001804CE030480288101C002804D100A8EB
:10F5A0000078011C2D48018000A80178131C2C480C
:10F5B0000068C154284901320A80284909880B1C77
:10F5C000254A12889A4232D10339013000F0E4F919
:10F5D000031C22480088011C21480068401821496A
:10F5E000415C1A1C120AFF242240914206D11E4996
:10F5F000405C191CFF221140884203D0022000F019
:10F6000009F911E015480088011C1548006800F050
:10F6100045FA0006000E002803D1052000F0FAF894
:10F6200002E0042000F0F6F80021084801700648C6
:10F630000088002802D100210448017001B010BCEC
:10F6400008BC1847D41D00400E050040AC22004005
:10F65000F821004055FF0000F4210040F621004051
:10F66000A8210040FEFFFFFFFFFFFFFF10B5164C73
:10F67000201CDF300078FBF7A3FD206805F0FEFBBF
:10F68000606805F0FBFB1148F4F772FD1049114862
:10F69000016002200021F6F71DFE201CDF300078FB
:10F6A0000021FDF7A7FD201C2E300078011C012051
:10F6B000FDF73EFEA08D00040014F5F771FC00205C
:10F6C000FEF7BCF910BDC046A8210040802500000F
:10F6D000C18B00008805004070B50E1C041CA1B051
:10F6E000301C0006000E802801DD002050E0FF21C4
:10F6F00000A801705521012068440170301C0106EA
:10F70000090E03310906090E022068440170301CFD
:10F710000206120E03206844211C05F04BFB351C29
:10F720000335301C0106090E201C00F035F9021CBF
:10F73000101C000AFF2108400006000E291C01359C
:10F740002D062D0E0B061B0E00A9C854101CFF2100
:10F7500008400006000E291C01352D062D0E0A0654
:10F76000120E00A98854002409E0201C0106090E8D
:10F7700000A8405CF4F7D4FC01342406240E281CB5
:10F780000106090E201C0006000E8842EDD3012060
:10F7900021B070BD10B4031C0022181C0260081CAC
:10F7A0000478181C026822430260181C02681202C6
:10F7B000181C0260081C4078041C181C02682243B4
:10F7C0000260181C02681202181C0260081C807873
:10F7D000021C181C01681143016010BC7047C04630
:10F7E00010B4031C0022181C0260081C0478181CAA
:10F7F000026822430260181C02681202181C026090
:10F80000081C4078021C181C01681143016010BCE0
:10F810007047C04600B5021C002006490968087000
:10F82000101C044909684870022102480068FFF76B
:10F8300053FF00BDAC210040021C081C0006000E56
:10F84000022805D1101C4078002801D1012000E0D9
:10F850000020704710B5041C82B0081C0006000E82
:10F8600006280FD100A8211C0131FFF793FF01A842
:10F87000211C0431FFF7B4FF0199009801F0E4FC6A
:10F88000012000E0002002B010BC08BC1847C046B0
:10F8900030B50C1C051CC1B01F4901A81F4A0B78CC
:10F8A0000370491C401C521EF9D1201C0006000E9A
:10F8B00004282CDD01A8FF21184A05F093FA00A8BE
:10F8C000291C0131FFF766FF201C0206120E043AC4
:10F8D00001A8291C043105F06DFA009910488142F5
:10F8E00000D2009001200021F6F7F4FC0D4A009BA5
:10F8F00014200221F6F7AAFC201C0206120E043A7C
:10F90000009801A901F0A8FD0006000E00E000200B
:10F9100041B030BC08BC1847902A0000000100002C
:10F9200000000E002926000000B5021C81B0081C52
:10F930000006000E042822D100A8111C0131FFF797
:10F9400029FF00981049091802D01049091816D14A
:10F9500001200021F6F7BEFC0D4A009B1420022175
:10F96000F6F774FC009801F0BBFC6420F6F7A8F8E9
:10F97000084A22200221F6F769FC012000E000205D
:10F9800001B008BC1847C0460000F1FF0000F2FFBC
:10F990001E2600001B260000F0B4164B1A1C1FE0A8
:10F9A000141C240B051C2E7835096C400F252C40A7
:10F9B000271CBF00104CE459120162400D4C22403C
:10F9C000141C240B74402C40251CAD000A4C6459B7
:10F9D00012016240074C2240013001390906090E2C
:10F9E0000C1C2406240E002CDADC5A40101CF0BC3F
:10F9F0007047C046FFFF00009823000010B5FBF7DA
:10FA0000EFFB1D4C211CDF3108701C491C480160B4
:10FA10000620FBF7D5FB0120FEF710F8022000219D
:10FA2000F6F758FC174A04200321F6F70FFC164896
:10FA300005F0ECF92060802005F0E8F960602068AE
:10FA4000002807D1114A00200321F6F7FFFBFFF73A
:10FA50000DFE10E00E480068002807D10D4A002076
:10FA60000321F6F7F3FBFFF701FE04E00A48F4F781
:10FA70007FFB01F0E1FB10BDA821004039F500003B
:10FA8000880500400F26000000040000FA25000051
:10FA9000AC210040E625000000E1000070B50E1C1E
:10FAA000051C00241DE0201C0104090C89001248DB
:10FAB00040580178281C407881420FD1301C010445
:10FAC000090C0339281C0130221C13041B0C9B0059
:10FAD000094AD258526805F06DFA0BE0013424044B
:10FAE000240C201C0104090C8900034840580028FC
:10FAF000D9D1002070BDC046B021004030B50D1CEA
:10FB0000041C211C34480171291C41710079FDF746
:10FB1000BDFC32490860201C0006000E08281AD1DE
:10FB2000201C0106090E2E48405C00280CD0012044
:10FB3000F5F708FC0320FBF74FFA0220F3F7E2FE8B
:10FB40000121284801703BE00120F3F7DBFE022190
:10FB50002448017034E0281C0006000E032826D13A
:10FB6000201C0106090E2048405C011C49001F486A
:10FB7000405A0004001404F0C1FFF5F70BFA201CF2
:10FB80000106090E1648405C002809D00220FBF748
:10FB900023FA0220F3F7B6FE0121124801700FE0AC
:10FBA0000020F3F7AFFE02210E48017008E00120AB
:10FBB000FBF712FA0220F3F7A5FE002109480170B5
:10FBC0000B480078011C2220F6F7E2F90120002101
:10FBD000FDF710FB30BDC046D2210040042000409C
:10FBE000971D0040E22100408D1D0040401700009D
:10FBF000D621004000B501F017FA0006000E0C28CF
:10FC000013D00A480078042805D0002803D1042125
:10FC10000648017002E000210448017001210448F7
:10FC200001700248007801F07FF900BDE321004037
:10FC30009C24004000B509480078062803D006211E
:10FC40000648017002E000210448017001210448C7
:10FC500001700248007801F013F900BDE621004070
:10FC60009C24004000B50B480078032811D00A48B6
:10FC70000078012803D001210748017002E000212B
:10FC8000054801700121054801700348007801F022
:10FC9000D1F800BDE9210040EA2100409C24004049
:10FCA00000B501F0C1F90006000E0C2817D001F0D4
:10FCB000BBF90006000E042811D00948007803287B
:10FCC00003D003210648017002E0002104480170BE
:10FCD0000121044801700248007801F025F900BDB7
:10FCE000E32100409C24004000B501F09DF900068E
:10FCF000000E0C2814D00B4801780131017009481E
:10FD00000078012805D0022803D0FFE7002105482C
:10FD100001700121044801700248007801F004F9E3
:10FD200000BDC046E32100409C24004030B50025C2
:10FD30002C1C01F079F90006000E0C284BD0264847
:10FD40000078022805D0032803D0042801D0012818
:10FD50000AD122490978002902D020490D7002E019
:10FD600001221E490A700124022811D003281BD049
:10FD7000042825D0012827D118480078002803D06E
:10FD8000032001F007FB1FE0022001F003FB1BE052
:10FD900012480078002803D0032001F0F1FA13E0A4
:10FDA000022001F0EDFA0FE00C480078002803D0A3
:10FDB000002001F0DBFA07E0042001F0D7FA03E0AD
:10FDC0000648007801F0C4FA201C002803D0012066
:10FDD0000021FDF70FFA30BDE3210040E42100408F
:10FDE00000B51C480078002832D11B480078012853
:10FDF00012D0022810D000281FD1184801780131F4
:10FE0000017016480078012817D0022815D0FFE7A6
:10FE100000211248017010E0104801780131017092
:10FE20000E480078022808D0012803D102210B488F
:10FE3000017002E0002109480170012108480170A9
:10FE40000648007801F01CF801200021FDF7D2F9E6
:10FE500000BDC046EE210040E5210040E621004003
:10FE60009C24004000B533480078002828D00120A9
:10FE7000F5F7FAF830480178013101702E48007822
:10FE8000032105F09DF8011C2B4801702A480078D9
:10FE9000012807D0022809D000280AD1022001F049
:10FEA000D3F806E0022001F0CFF802E0032001F0D1
:10FEB000CBF82248F5F704FE0020F5F7D5F834E03A
:10FEC0001F480078002803D000211D48017002E07F
:10FED00001211B4801701B48007803280DD005281C
:10FEE00003D0062811D0002814D103211548017031
:10FEF0001448007800F0C4FF17E005211148017094
:10FF00001048007800F0BCFF0FE00D48007801F0C9
:10FF10001FFA0AE00A480078002803D0032001F005
:10FF200039FA02E0022001F035FA01200021FDF744
:10FF300061F900BDEE210040E82100402C010000E5
:10FF4000E7210040E62100407047C0467047C046A8
:10FF5000011C081C252811D026280FD027280DD0D9
:10FF600028280BD0292809D02A2807D02B2805D0EB
:10FF70002C2803D02D2801D024280FD11648028820
:10FF8000120115480280081C0206120E243A1204BF
:10FF9000120C114801881143018002E000210E4833
:10FFA00001800D4800880D49091808D002390BD08E
:10FFB00003310ED100210848018001200AE0002110
:10FFC00005480180022005E000210348018003204C
:10FFD00000E000207047C046FA210040DF7AFFFFB2
:10FFE00010B5041CDC480078002816D1201C01281C
:10FFF0000FD0022809D01C2802D0042800D0A9E183
:020000040001F9
:100000000121081CFDF774F9A4E10021D348017017
:10001000A0E10121D14801709CE1201C332805D0CA
:100020004A2803D0FFE70120F6F7FAF8201C000663
:10003000000EFFF78DFF022813D0032818D00128E7
:1000400025D1C74A14200221F6F700F90120F7F75D
:1000500017FE0020FDF78EFB01200021FDF748F977
:1000600015E0FDF7D3FB01200021FDF7C3F80EE0FA
:10007000BB4A14200221F6F7E9F80120F7F700FE49
:100080000120FDF777FB01200021FDF731F9201C4D
:10009000012800D1E9E0022800D1D9E005286AD082
:1000A00006286CD00D2863D00E287DD00F287BD079
:1000B000102879D0112877D0122875D0132873D042
:1000C000142871D015286FD0162800D194E0172875
:1000D00000D17FE0182800D1A0E0192800D1A5E0C8
:1000E0001A2855D01B2859D01D2839D01E2846D093
:1000F0001F2840D030283BD0312844D0322834D07B
:10010000332800D1E9E039285ED03A2840D03B2896
:1001100044D03C2870D03D285CD03E287ED03F287B
:1001200000D183E0402800D1ACE0412844D04228EF
:1001300042D0432840D044283ED045283CD04628D1
:100140003AD0472838D0482836D0492834D04A28D1
:1001500000D19EE0622800D1FAE0042800D0F9E046
:1001600001200021FDF7C4F8F4E0FEF7ABFFF1E059
:10017000F7F774FCEEE00120FBF7D0FBEAE0022089
:10018000FBF7CCFBE6E00021081CFCF7DBFFE1E01D
:10019000012000210022FDF74DF8DBE00121081CC1
:1001A0000022FDF747F8D5E0201C0106090E0E39A4
:1001B0000120FDF7BDF8CDE0201C0106090E4139F4
:1001C0000120FDF7B5F8C5E0012003210022FDF76D
:1001D000CFF8BFE063480078032807D0042808D090
:1001E000012800D0B6E0FFF7A1FDB3E0FFF73AFE2B
:1001F000B0E0FFF7ABFEADE05A480078032807D027
:10020000042808D0012800D0A4E0FFF76DFDA1E08C
:10021000FFF7E6FD9EE0FFF797FE9BE05148007870
:10022000012800D096E0FFF73BFD93E04D480078B1
:10023000032807D0042808D0012800D08AE0FFF75F
:10024000D9FC87E0FFF7F6FC84E0FFF70BFD81E0C7
:100250000020454C2077002000F048FFA079021CC8
:1002600001200221FDF784F874E001203E4C207744
:10027000012000F03BFFA079021C01200221FDF7C4
:1002800077F867E03849087949790022FDF774F971
:1002900060E03648007804285CD101200021F6F7A0
:1002A0008DF833480078002809D0002130480170CB
:1002B000304B1422101C0221F6F744F808E001210B
:1002C0002B4801702C4B1422101C0221F6F73AF82F
:1002D0002748007800F06CFF3CE0224800780328B3
:1002E00038D1264801780131017024480078032173
:1002F00004F066FE011C2148017001200021F6F780
:100300005DF81E48007801280AD002280FD0002886
:1003100013D11B4B1422101C0221F6F713F80CE02A
:10032000184B1422101C0221F6F70CF805E0164BAE
:100330001422101C0221F6F705F810480078011C61
:100340002120F5F725FE0D48007800F0FBFE01E0C6
:10035000FFF754FB10BDC046D3210040EE21004002
:10036000F4240000E0210040D22100409924004004
:10037000E6230040ED240000E7240000E5230040D0
:10038000DE240000D4240000CA240000F0B51F1CA5
:10039000161C0C1C051C82B04C48007800281DD18E
:1003A000281C0106090E4A480078884216D1201CF4
:1003B0000106090E4748007888420FD1301C01061B
:1003C000090E45480078884208D1381C0106090EFC
:1003D00042480078884201D1002075E000213B4866
:1003E0000170291C3A480170211C3A480170311CE7
:1003F00039480170391C394801700120F3F716F8AB
:10040000002000F02FFAFF213548017035480170B7
:10041000032100A80170281C0006000E02F05EFFF8
:1004200001A9087000AA1078031C013B1370002872
:1004300002D008780128EED001A80078012801D167
:10044000012041E0032100A80170201C0006000EDD
:1004500002F044FF01A9087000AA1078031C013BB8
:100460001370002802D008780128EED001A8007887
:10047000012801D1012027E002F0B8FB201C000672
:10048000000E391C0906090E02F0AEFF0006000E30
:10049000012801D1012017E0281C0006000E311CA4
:1004A0000906090E03F044F80006000E012801D1E8
:1004B000012009E0291C0A480170211C094801702B
:1004C0000020F2F7B3FF002002B0F0BD9C240040F2
:1004D0009824004099240040AB240040AC24004004
:1004E000A9240040AA24004010B5011C081C8078F3
:1004F000032808D010286BD0002869D1081C0330CD
:1005000002F05CFD64E033480078042834D003280E
:100510005ED1072000F064FD0006000E2E4C207016
:100520000B2000F05DFD0006000EA070082000F01A
:1005300057FD0006000E6070102000F051FD00060F
:10054000000EE070012001F0ABFB0006000E2071F0
:10055000192000F045FD0004000CE0801E4882B028
:100560006946082302780A70401C491C5B1EF9D1B9
:1005700002F0D0FD02B02BE0062000F043FD0006A3
:10058000000E144CE0760F2000F03CFD0006000E3B
:100590002077122000F036FD0006000E60770D2057
:1005A00000F030FD0006000EA077072000F02AFDC5
:1005B0000006000EE077094882B0694607230278FA
:1005C0000A70401C491C5B1EF9D102F0D9FD02B033
:1005D00010BDC0469A240040CC230040B524004002
:1005E00010B5011C80201C4A107002205070102091
:1005F00090703F20D070BF201071C02050718020BB
:1006000090710120D07110201072081C01280CD0AC
:10061000022813D000281DD180200F4948720020E5
:1006200088722C200C24C87210E0C0200A4948723D
:10063000002088722C200C24C87207E08020064914
:1006400048720020887220200C24C872211C0248A5
:10065000F5F75CFB10BDC046E823004010B5011C57
:1006600081202E4A107000205070002090701020C1
:10067000D070002010710020507100209071012076
:10068000D0718120107200205072002090721120D1
:10069000D072081C01281ED000283ED100201F491E
:1006A000087340204873172088730120C873812085
:1006B000087400204874002088741220C874002038
:1006C0000875002048754E2088754F201824240492
:1006D0002414C8751BE000201049087300204873DB
:1006E000162088730020C873812008740020487485
:1006F000002088741220C8740020087500204875F6
:100700005E2088754F20182424042414C875201CEA
:10071000010409140148F5F721FB10BD282400400D
:1007200010B5011C8120164A1070802050700020E6
:1007300090700320D070081C01280ED000281ED114
:1007400000200F4908711020487110208871002086
:10075000082424042414C8710BE0FF200849087100
:10076000EF204871FF208871FF20082424042414FE
:10077000C871201C010409140148F5F7EFFA10BDF7
:100780002824004000B50A1C011C081C0106090EA3
:1007900004480143101C0206120E812001F034F9B6
:1007A00000BDC0460001000000B5011C081C020687
:1007B000120E8120002101F027F900BD00B5011CB7
:1007C000081C0206120E1020024303480243882030
:1007D000002101F053F900BD0090000000B5031C9A
:1007E0000022181C002800D00122081C002801D07B
:1007F00010200243101C0206120E8A20002101F074
:100800003DF900BD10B5031C181C002800D00124C0
:10081000081C0006000E0321084000010006000E1F
:1008200000210143101C0006000E0F22104000069C
:10083000000E0143201C0206120E1202081C0006C4
:10084000000E02438A20012101F018F910BDC046B4
:1008500000B5011C081C0206120E8A20022101F0BC
:100860000DF900BD00B5011C081C002805D00128A9
:1008700003D10020F4F75EFD0BE00020F4F75AFDF1
:100880000120F5F71DF90120F4F754FD0120F5F7DB
:1008900017F900BD30B5051C281C002801D0012027
:1008A0000443081C002801D008200443101C002821
:1008B00001D010200443181C002801D0402004431C
:1008C000201C0206120ED720002101F09DF830BD39
:1008D00000B5021CD720012101F096F800BDC046EA
:1008E00000B5021CD720022101F08EF800BDC046E1
:1008F00033B50098012815D0022815D0032815D04B
:10090000042815D0052815D0062815D0072815D09D
:10091000082815D0092815D00A2815D00028FFD19D
:10092000032412E0042410E005240EE006240CE069
:1009300007240AE0082408E0092406E00A2404E069
:100940000B2402E00C2400E00D240198012817D0AC
:10095000022817D0032817D0042817D0052817D04D
:10096000062817D0072817D0082817D0092817D02D
:100970000A2817D00B2817D00028FFD1002514E033
:10098000012512E0022510E003250EE004250CE00D
:1009900005250AE0062508E0072506E0082504E00D
:1009A000092502E00A2500E00B25201C0106090E9E
:1009B000281C0206120ED72001F026F802B030BD26
:1009C00011B50098012805D0022805D00028FFD1D4
:1009D0001C2402E01D2400E01E24081C01F0C0F9C4
:1009E000211C0906090E021CD72001F00DF801B0E8
:1009F00010BDC04611B50098042807D0062807D0BE
:100A0000072807D00328FFD11F2404E0202402E098
:100A1000212400E02224081C01F0A2F9211C09066F
:100A2000090E021CD72000F0EFFF01B010BDC04638
:100A300011B5009801280DD002280DD003280DD043
:100A400004280DD006280DD007280DD00028FFD18E
:100A500015240AE0162408E0172406E0182404E010
:100A6000192402E01A2400E01B24081C01F078F984
:100A7000211C0906090E021CD72000F0C5FF01B099
:100A800010BDC04611B50098022805D0052805D034
:100A90000028FFD1232402E0242400E02524081CA0
:100AA00001F05EF9211C0906090E021CD72000F096
:100AB000ABFF01B010BDC04611B50098052803D0AA
:100AC0000128FFD1262400E02724081C01F048F962
:100AD000211C0906090E021CD72000F095FF01B069
:100AE00010BDC04611B50098042805D0052805D0D2
:100AF0000328FFD1282402E0292400E02A24081C2E
:100B000001F02EF9211C0906090E021CD72000F065
:100B10007BFF01B010BDC04611B50098052807D075
:100B2000072803D00628FFD12B2402E02C2400E064
:100B30002D24081C01F014F9211C0906090E021CC1
:100B4000D72000F061FF01B010BDC04611B500987C
:100B5000012807D0022807D0032807D00028FFD19A
:100B60002E2404E02F2402E0302400E03124081C6D
:100B700001F0F6F8211C0906090E021CD72000F02E
:100B800043FF01B010BDC04611B50098012807D041
:100B9000022807D0032807D00028FFD1322404E020
:100BA000332402E0342400E03524081C01F0D8F896
:100BB000211C0906090E021CD72000F025FF01B0F8
:100BC00010BDC04600B5011C081C01F0C9F8021C8C
:100BD000D720362100F018FF00BDC04600B5011C2B
:100BE000081C01F0BDF8021CD720372100F00CFFD3
:100BF00000BDC04600B5011C081C01F0B1F8021C84
:100C0000D720382100F000FF00BDC04611B5009884
:100C100001280DD002280DD003280DD004280DD0B6
:100C200006280DD007280DD00028FFD10E240AE099
:100C30000F2408E0102406E0112404E0122402E04E
:100C4000132400E01424081C01F08AF8211C090672
:100C5000090E021CD72000F0D7FE01B010BDC0461F
:100C600010B52B480078002851D02A480078002879
:100C700003D0011C0020FFF73BFE27480078002826
:100C800003D0011C0120FFF733FE24480078002820
:100C900003D0011C0220FFF72BFE2148007800281A
:100CA00003D0011C0320FFF723FE1E480078002814
:100CB00003D0011C0420FFF71BFE1B48007800280E
:100CC00003D0011C0520FFF713FE18480078002808
:100CD00003D0011C0620FFF70BFE15480078002802
:100CE00013D0011C0720FFF703FE0A4C207A011CD9
:100CF0000820FFF7FDFD607A011C0920FFF7F8FDD1
:100D0000A07A011C0A20FFF7F3FD01F05DF910BD88
:100D1000C4240040D4230040D6230040D523004003
:100D2000D7230040D8230040D9230040DA230040D5
:100D3000DB23004000B5002000F024F8002801D09B
:100D4000002000E0012000BD00B5182000F006F8EA
:100D5000011C0148084000BDFFFF000000B5021C57
:100D60001C2007490870C020487000208870101CA3
:100D7000C87004210248F4F7F1FF00F017FE00BD2F
:100D80002824004000B5021C1D2007490870C0201F
:100D9000487000208870101CC87004210248F4F7C5
:100DA000DDFF00F003FE00BD2824004000B5011C5B
:100DB000081C0206120E9D20042100F025FE00BD35
:100DC00000B5011C081C002805D00022101C111CB5
:100DD000FFF718FD04E00021081C0922FFF712FDAF
:100DE00000BDC04630B5002416E0201C0106090EE7
:100DF000C9000E48405800F0C9F8051C201C010627
:100E0000090EC9000A48405C011C2A1C9C2000F005
:100E1000FBFD01342406240E201C0106090EC90026
:100E20000348405C0028E0D130BDC046A82C00003B
:100E3000A42C000030B5011C10480078012808D00F
:100E4000022806D0032803D00028FFD1072501E09F
:100E500000212425081C012803D00028FFD10324E9
:100E600000E02624281C0006000E211C0906090E9D
:100E700000231A1CFFF78AFA30BDC046A7240040A1
:100E800030B5011C26480078002802D002241A251B
:100E90003AE024480078012818D002282BD00028F6
:100EA00029D1081C00280ED0012806D0022807D01E
:100EB000062808D10024032526E00224042523E087
:100EC00002240E2520E0002404251DE0081C002833
:100ED0000ED0022806D0032807D0062808D1002407
:100EE000262511E002240E250EE0012403250BE047
:100EF0000024032508E00124081C0006000E062833
:100F000001D1262500E00325201C0006000E291C27
:100F10000906090E03220023FFF738FA30BDC04648
:100F2000EE210040A624004010B5011C00F07CF822
:100F30000006000E0C2800D100210422081C002805
:100F400014D0022809D003280AD004280BD0052881
:100F50000CD001280AD1022409E002240E2206E066
:100F60000924032203E01B24032200E00D24201C9B
:100F70000006000E111C0906090E034A1278131C04
:100F80000122FFF703FA10BDAC24004000B5021C9B
:100F90000449101C02F08CFE03F030F8011C081C00
:100FA00000BDC046FFFF7F4B00B5021C101C04496A
:100FB00004F02AF8081C03F0A1FD011C081C00BD68
:100FC000FFFFFF0000B5021C0449101C02F070FE78
:100FD00003F014F8011C081C00BDC046FEFFFF4AC8
:100FE00000B5021C0B200649087000204870101C38
:100FF000887003210248F4F789FE00F0ADFC00BDC3
:10100000E823004000B5021C1120064908700020AA
:101010004870101C887003210248F4F777FE00F036
:101020009BFC00BDE8230040014800787047C046A3
:101030009B24004000B5011C081C0206120EBD20B6
:10104000002100F0E1FC00BD00B5011C081C0206F7
:10105000120EBD20012100F0D7FC00BD00B5BD205F
:101060000421194A00F0D0FCBD200521174A00F0E8
:10107000CBFCBD200621164A00F0C6FCBD2007218E
:10108000144A00F0C1FCBD200821134A00F0BCFC4A
:10109000BD200921114A00F0B7FCBD200C21104AE7
:1010A00000F0B2FCBD200D210E4A00F0ADFCBD20C9
:1010B0000E210D4A00F0A8FC002001F0C1F801202B
:1010C000FFF7C2FF00BDC046406D0100008C01006B
:1010D00000AB0100C0CA010000EA01008009020063
:1010E000C029020000440200405E020000B5011C5D
:1010F000081C00280ED011494A78081C25300270BF
:10110000012008710878CA7C097D0B1C1A21FFF7A1
:101110003DF911E00A4800781A2802D10421084854
:1011200001700120054B18711878191C25310978B8
:10113000DA7C1B7DFFF72AF900BDC04698240040E9
:10114000BD24004010B5011C081C012805D0022850
:1011500005D0002804D1002402E0084C00E0084C2F
:1011600008480078002808D00220FFF771FB201CF7
:1011700000F004FD201C00F009FD10BDFFFF3F0042
:10118000FFFF7F00C424004000B5011C0648007822
:10119000042808D105480078002804D0081C00065F
:1011A000000E01F04FFA00BD99240040C424004015
:1011B00000B5011C06480078042808D1081C002846
:1011C00002D001F059FB02E0002001F08BF900BDD4
:1011D0009924004010B4031C0022181C0260081C53
:1011E0000478181C026822430260181C026812026C
:1011F000181C0260081C4078041C181C026822435A
:101200000260181C02681202181C0260081C807818
:10121000041C181C026822430260181C0268120297
:10122000181C0260081CC078021C181C01681143BD
:10123000016010BC7047C04600B51D201C21002372
:101240001A1CFFF7A3F800BD70B50D1C041C211C6F
:10125000012001F0A1FC291C022001F09DFC0020CE
:10126000022101F099FC002001F0A2FC0028FAD133
:101270001848211CF4F7B8FE00241CE0201C0028AC
:101280000BD0201C00040014042103F0BDFE011C3F
:10129000002902D11048F4F7A7FE201C0004001416
:1012A000103001F085FC061C0C48311CF4F79CFE44
:1012B000013424042414281C042103F0A5FE081C76
:1012C000211C090409148142D8DB0348F4F78CFE81
:1012D00070BDC046542E0000522E00004C2E00005F
:1012E00010B5041C0320062101F056FC042014490B
:1012F00001F052FC0520134901F04EFC0620124972
:1013000001F04AFC07200E4901F046FC08200D4977
:1013100001F042FC211C0D480143092001F03CFC76
:101320000220002101F038FC0020012101F034FCF2
:10133000002001F03DFC0028FAD1012010BDC0467C
:10134000AA0A00AA55050055AA0A0080000000302C
:1013500000B5011C081C002804D0012802D101F0AE
:10136000D9FA01E001F074FB00BDC04600B5011CD4
:10137000081C0206120E8E20012100F07FFB00BD2A
:1013800000B5011C081C0206120EBF20012100F04E
:101390003BFB00BD00B5021C101C0006000E05281A
:1013A00010DC8E20084908700020487001208870E9
:1013B0000020C87000200871101C487106210248E6
:1013C000F4F7A4FC00BDC046E823004000B5021CB1
:1013D000074B101C002800D0064B081C002801D029
:1013E000102003431A1CBB20002100F00DFB00BDA0
:1013F000001100000111000000B58E200021012223
:1014000000F03CFB8E200121022200F037FB8E20F1
:101410000221012200F032FB8E200321002200F085
:101420002DFB8E200421012200F028FB8E200521B7
:10143000012200F023FB8E200621012200F01EFB7A
:101440008E200721FF2200F019FB8E20082109229F
:1014500000F014FB00BDC046F0B5171C0E1C81B097
:101460006424011C012001F097FB381C0106090EC1
:10147000022001F091FB00250EE000A8311CFFF7CF
:10148000A9FE281C0006000E1030009901F084FB14
:1014900001352D062D0E0436381C0006000E0421E1
:1014A00003F0B2FD081C291C0906090E8142E4DB89
:1014B0000320032101F070FB0420194901F06CFBAB
:1014C0000520184901F068FB0620174901F064FB6C
:1014D0000020164901F060FB002001F069FB00903C
:1014E000009800280ED00098114908401149884200
:1014F00008D00A20F4F7E4FA013C24042414201C48
:101500000028E9D1201C00040014002802D0009813
:10151000002801D0002000E0012001B0F0BDC0464D
:10152000AA0A00AA55050055AA0A00A0190000023F
:10153000FFFF000008010000F0B5011C0327081C94
:1015400001280CD0022813D0032815D0002816D16A
:101550000120FFF787F90021174801702BE0174899
:101560000078002800D01A2701240026351C06E048
:1015700002240126351C02E00226341C012501212B
:101580000F480170201C0006000E391C0906090EC8
:101590002A1C1206120E331C1B061B0EFEF7F6FE4B
:1015A0000006000E002803D101210348017002E06B
:1015B000002101480170F0BDC4240040EE2100402C
:1015C0009C24004000B50B1C021C101C012811D0EB
:1015D000022813D0032815D0042817D0052821D0BD
:1015E000062817D0072819D000281ED1191C354805
:1015F00001801AE0191C3448018016E0191C334898
:10160000018012E0191C324801800EE0191C31489B
:1016100001800AE0191C3048018006E0191C2F489F
:10162000018002E0191C2E4801802E480078002815
:1016300047D0101C012814D0022819D003281ED02E
:10164000042823D0052836D0062826D007282BD0FA
:10165000002836D11B480088011C002000F04CFEF9
:101660002FE019480088011C012000F045FE28E009
:1016700016480088011C022000F03EFE21E01448BC
:101680000088011C032000F037FE1AE01148008892
:10169000011C042000F030FE13E00F480088011CFC
:1016A000062000F029FE0CE00C480088011C0720F1
:1016B00000F022FE05E00A480088011C052000F029
:1016C0001BFE00BDBC230040BE230040C0230040E1
:1016D000C4230040C2230040C8230040C62300406A
:1016E000CA230040C424004010B5021C0B1C101C6F
:1016F0000406240E1F480355101C012811D002288F
:1017000013D0032815D0042817D0052821D0062887
:1017100017D0072819D0002824D10A1C16480270B7
:1017200020E00A1C154802701CE00A1C14480270D4
:1017300018E00A1C1348027014E00A1C12480270D8
:1017400010E00A1C114802700CE00A1C10480270DC
:1017500008E0081C084AD071081C1072081C50725E
:10176000081C90720B480078002801D0FFF778FA27
:1017700010BDC046AD240040D4230040D623004015
:10178000D5230040D7230040D8230040D923004070
:10179000DA230040C424004000B50B1C021C191CB5
:1017A000101C0206120E02488154FFF759FA00BDC0
:1017B0009D24004070B5141C0D1C061C2C4800789C
:1017C000002854D00F20032101F04EFF0006000E28
:1017D000002805D10F20032100220123FEF7D6FDAA
:1017E000301C012812D002281BD0032828D004283E
:1017F00035D000283BD1002000F0B0F9281C0206AB
:10180000120E0020012100F083F930E0002000F0EA
:10181000A5F9281C0206120E0120002100F078F91B
:1018200025E00F20032100220123FEF7AFFD012058
:1018300000F094F9201C0006000E00F097F916E065
:101840000F20032100220123FEF7A0FD022000F05B
:1018500085F9201C0006000E00F088F907E0002141
:10186000081C082200F054F9002000F077F970BD40
:10187000C424004010B50C1C011C2248007800282C
:101880003FD0081C012817D002281FD003282CD0D5
:10189000002836D101211C4801700223181C0421A4
:1018A0000122FEF773FD032000F0CCFD002000F0C4
:1018B000BFFDFFF797FA24E0201C0006000E002170
:1018C00000F0D8FD012000F0CBFD1AE0201C00063E
:1018D000000E002100F0CEFD9C200721082200F020
:1018E00093F8022000F0BCFD0BE06F20FFF75EFADA
:1018F000201C0006000E012100F0BCFD082000F0B5
:10190000AFFD10BDC42400409C24004010B4031C53
:101910000022181C0260081C0478181C026822436C
:101920000260181C02681202181C0260081C407831
:10193000041C181C026822430260181C0268120270
:10194000181C0260081C8078021C181C01681143D6
:10195000016010BC7047C04610B581B01424F3F785
:10196000BDFC0006000E002808D00120F4F7A8F8FE
:10197000201C013C2406240E0028F0D1201C002845
:1019800008D007480621F4F78FF900A80549FFF7AA
:10199000BDFF01E004480090009801B010BDC046B2
:1019A000682400406B240040FFFFFF0010B581B0A9
:1019B000002000901424F3F78BFC0006000E002892
:1019C00008D00120F4F77CF8201C013C2406240EEA
:1019D0000028F0D1201C002808D008480821F4F77E
:1019E00031F900A80649FFF7F5FB01E00548009032
:1019F0000120F4F765F8009801B010BD8024004084
:101A000084240040FFFFFFFF10B5041C201C1A4B6C
:101A1000187000205870081C0004000C000AFF24F5
:101A200020400006000E9870081C0004000CFF21E6
:101A300008400006000ED870101C000EFF21084060
:101A40000006000E1871101C000CFF210840000653
:101A5000000E5871101C000AFF2108400006000EFD
:101A60009871101CFF2108400006000ED871082153
:101A70000148F4F773F910BD2824004010B5041C88
:101A8000201C0F4B187000205870081C9870101CF8
:101A9000000CFF2108400006000ED870101C000A40
:101AA000FF2108400006000E1871101CFF2108409D
:101AB0000006000E587106210148F4F727F910BD01
:101AC000E823004030B5051C0024231C281C0028F6
:101AD00000D00123081C002801D010200343101C53
:101AE000002800D001248E2008490870002048708A
:101AF000002088700020C870201C0871181C4871D4
:101B000006210248F4F702F930BDC046E823004040
:101B100010B5041C0023201C002801D0602303E022
:101B2000081C002800D03023101C0006000E0F21D6
:101B300008400006000E0343181C0206120E8820FF
:101B40000121FFF79BFF10BD00B5011C081C020618
:101B5000120E88201421FFF791FF00BD01B5009AF5
:101B600092200021FFF78AFF01B000BD01B5009A65
:101B700092200121FFF782FF01B000BD00B5021CD9
:101B80008A200321FFF77AFF00BDC04600B5021C82
:101B90008A200421FFF772FF00BDC04670B5061C05
:101BA00000252C1C301C002800D00124081C002813
:101BB00001D010200443101C002801D02020044331
:101BC000181C002800D00125281C0206120E120243
:101BD000201C0006000E02439C200021FFF74EFF50
:101BE00070BDC04600B5011C081C0206120E9C20E8
:101BF0001321FFF743FF00BD00B50A1C011C081CA0
